:020000040000FA
:040000006FD00400B9
:101000006F009044000000000000000090200020CD
:10101000A4220020A9BDF9F55C23002000000000F7
:10102000000000005C230020902000200000000051
:101030000000000090200020000000009020002010
:101040000000000090200020902000209020002030
:101050009020002090200020B82B0020902000201D
:10106000000000009020002090200020EC230020B1
:1010700090200020C22300209020002090200020FB
:101080009020002090200020902000209020002020
:101090009020002001A04111B7170040985F3AC688
:1010A000945F3247E39CE6FE3245410182800111A4
:1010B00013078008F337078093F787083EC20100C3
:1010C0000100B7170040930570052380B70413068D
:1010D00080FA2380C7040100010083C6B70493F699
:1010E000F60DA385D704238007049246F3A6068055
:1010F0000100010093760502D5CEF336078093F602
:10110000860836C4010001002380B7042380C70489
:1011100001000100B70614007D89558D88C70100C4
:1011200001000100010023800704A246F3A6068007
:101130000100010073370780137787083AC6010062
:1011400001002380B7042380C704010001000100CF
:1011500001003727004093061005A303D7802380A2
:101160000704B247F3A70780010001009307800836
:10117000F3B7078093F787083ECE01000100B71749
:101180000040130770052380E704130780FA2380CB
:10119000E7040100010003C7B70413670708A3852C
:1011A000E70423800704F247F3A70780010001004A
:1011B0000561828093760504BDC6F336078093F6F9
:1011C000860836C8010001002380B7042380C704C5
:1011D00001000100B7061400938606047D89558D31
:1011E00088C7010001000100010023800704C246F6
:1011F000F3A6068001000100733707801377870884
:101200003ACA010001002380B7042380C70401000B
:1012100001003727004093062005A303D7802380D1
:101220000704D24781B773370780137787083ACC12
:10123000010001002380B7042380C70401000100DE
:1012400098471367070C98C723800704E24719BF24
:101250000111814601468145114506CE6D24930753
:101260008008F3B7078093F787083EC601000100A6
:10127000B7170040130770052380E704130780FAAF
:101280002380E7040100010003C767041367170008
:101290002383E70423800704B247F3A707800100F4
:1012A0000100F2400561828041118146014681457D
:1012B0001145912C13078008F337078093F78708AF
:1012C0003EC401000100B7170040130670052380DB
:1012D000C704930680FA2380D70401000100FD555E
:1012E0002396B70223800704A245F3A505800100D9
:1012F000010073370780137787083AC601000100A1
:101300002380C7042380D7040100010003C76704BA
:10131000136717002383E70423800704B247F3A76A
:1013200007800100010001A0BD473305F50201005F
:101330007D1575FD8280411122C426C206C6AA848D
:10134000014463179400B2402244924441018280D8
:1013500005041305803E4204C13F4180DDB7000013
:101360009305000273A04580824573901534924026
:101370002242B2424243D2436244F2440255925561
:101380002256B2564257D2576258F25806499649E9
:10139000264AB64A464BD64B664CF64C065D965DE1
:1013A000265EB65E465FD65F09617300203041114C
:1013B000B7170040985F3AC6945F3247E39CE6FE59
:1013C000324541018280B71700401307000323888C
:1013D000E7028547171700002326F7F47300203033
:1013E000411122C406C6370400201C408297F5BF75
:1013F00037370040834747009146BD8B6389D7004C
:1014000099466394D700834757407300203097165E
:10141000000083C6F6F39387160017160000A30991
:10142000F6F203478700973700009387E75CB6978B
:101430002380E700B7E70400BC4F0946894517152C
:1014400000000345C5E98297C9B723030480154707
:101450002303E48001002302A48082808307648048
:10146000E3CE07FE23030480828083076480E3CEFB
:1014700007FE03454480828083076480E3CE07FE35
:101480002302A4808280411126C44AC24EC006C6EF
:101490001377F50BAD47AA892E8995446306F700AB
:1014A00019456537653F8D444E854537FD59FD1417
:1014B00063983401B240A2441249824941018280BA
:1014C000135509011375F50F453F2209CDB70111D9
:1014D00026CC06CEB704080051371545BD37713705
:1014E00069372AC6A53F32459377150089EB136506
:1014F00015001375F50FF240E24405618280FD147A
:10150000E9FC0145CDBF397126DC4ADA4ED852D606
:1015100056D45AD25ED006DE62CE66CCB7E700E083
:101520007D5783AA070022C603AA470023A0E71815
:1015300023A2E718B7170040130770052380E704BC
:10154000130780FA2380E70483C74704930B75FFD2
:10155000B684E20793FBFB0F8546AA892E8B32895E
:1015600037240040E187015763FA76016308D5000C
:101570008946130700026313D5000157D98F93F7EB
:10158000F70FB71C00402382FC0411472303E480BB
:101590001305F00F5D3D094CD135636D7C11B70526
:1015A0000700DA9537870700795563F2E504B387BA
:1015B0009500636EF702370B0800A94733EB65010E
:1015C0006399F90689E48144513D26850DA0DA85A9
:1015D0000945553D05090345F9FFFD14050B693D16
:1015E00081C49377FB0FFDF7DD3569FD7D55B71796
:1015F0000040130770052380E704130780FA238057
:10160000E70403C74704418B2382E704F250B7E79E
:1016100000E023A0571123A24711E254324452594B
:10162000C259325AA25A125B825B724CE24C21615F
:101630008280A5476395F90685691309F00FB30603
:101640009900B3742B01B6941349F9FFB374990050
:10165000856B33796901416B9387F9FFB3F72701F4
:1016600099E363FC340193D94900C147E3E637FFAE
:1016700099BF0569C1697D19D9B71305800D6388C4
:101680006901130500026384790113051008CA85F6
:10169000DD3B353D21DD4E99B3843441D9B7DA8540
:1016A0002D45D533CA94E30099F205097D3BA30F7C
:1016B000A9FED5BF9387F9FF93F7F70F6361FC0C81
:1016C00083C71C0413073008631FF704370708009B
:1016D000636BEB04B3079B00B706100063F5D704F8
:1016E000334BEB0089476393F9068980D549E38C36
:1016F00004ECDA850945413B11090327C9FF9147ED
:101700002320E48003076480E34E07FE2303348133
:10171000FD17EDFBFD14110B81C49377FB0FE9FF5F
:101720007D3371F5E1B5B717004003C75704B7071C
:1017300008001377070219E3B78707007955E378A4
:10174000FBEA33079B00E3FFE7F855B58547E382E3
:10175000F9F2DA852D45053B9389F4FFE38504E62C
:10176000293393F7390091EB83260480032709007E
:1017700093074900E39AE6E43E89CE84F1BFB5477A
:101780006396F9001305900BC93135BDB1471305B8
:10179000B00AE38BF9FE99476391F904B705080095
:1017A000B365BB002D45C53181448D4BA1497539C9
:1017B00063967401832704802320F9008504E3984D
:1017C00034FF8327048013172B016355070023126E
:1017D000F900D5BB2322F900FDB39D476399F902B7
:1017E00081451305B0044531BD442320090023225F
:1017F0000900FD599D3993F77400CA9703C7070084
:10180000FD14398D2380A700E39634FF6DBBA147FB
:101810006392F9046D398144630D0B008D47930485
:10182000C0036308FB009304000563048B01930469
:1018300040041375C507E30895D81945393139397E
:101840000545213126850D3909453D314931E31CD6
:1018500005D669BB91476399F90013056006F53613
:10186000F53E130590090DB7E38F09D4F154A9BBD8
:10187000BD660147173600001306C644938606A6C8
:1018800085458347060093F7F70F91C382800507CC
:10189000E3F9E6FE973700002386B742DDB77D16F1
:1018A0006206618693178601E18763D407000145CC
:1018B0008280931726003307F500AE9718439C43A8
:1018C00063E7E7007D16E37FF7FC7D5582800545E1
:1018D0008280FD15E205E18513978501618793F705
:1018E000F50F63480700FD15139725002A97584305
:1018F00065D7138517006205618582803308B502BC
:101900001C4283A80600B335B502C29733B5070160
:10191000AE98469585486367B5006394A50063E378
:10192000070181480C43C6950CC388C21CC2828043
:1019300081471397870161876343B70082801397BC
:1019400027002A97232007008507E5B7814701472D
:1019500093968701E18663C5B60013351700828030
:1019600093962700AA9694428507558FD5B793D7AB
:1019700055408A07AA979C4305453315B5007D8DD0
:10198000828017F3FFDFE702C33B2A84993705C53E
:10199000931725003E940327C4FF814711EB7D1563
:1019A00016053E954205418517F3FFDF6700A33B0F
:1019B00005838507E5B70145C5BF814713978701B3
:1019C00061876343C700828013972700B386E500D1
:1019D00094422A97850714C3D5B77D16620661869F
:1019E000014793178601E18763D507001335170078
:1019F000828093172600B306F500AE9794429C436D
:101A00007D16B58F5D8FF1BF8A05AA950147636387
:101A1000B500828083A6C5FFF11593D71600D98F34
:101A20009CC11397F601E5B72A8301480147014598
:101A30006343D7008280B387050183A80700B307FB
:101A400006019C43C697AA976384F80033B5170133
:101A50000507B3080301620723A0F8006187110896
:101A6000C1BF2A8301478147014563C3D7008280F4
:101A70003388E50083280800330EE600032E0E00AD
:101A80003388A8403308C8416384080133B508018E
:101A90008507B308E300E20723A00801E1871107E7
:101AA000E9B717F3FFDFE702C3290111B286B28459
:101AB0002E86AA850A8575372A84A6850A857935F2
:101AC00033348000060413351500018D056117F3CA
:101AD000FFDF6700432917F3FFDFE702032441110B
:101AE000AA89AE8A328BB68402C202C402C60144FD
:101AF000131C8401135C8C4163499C02939B14006A
:101B0000FD1B0549138CF4FFF15C33048901620469
:101B10006184634D740592478E04CE9423AEF4FE27
:101B2000410117F3FFDF6700C32213192400B30B31
:101B30002B01014A93172A00D69783A50B008843EF
:101B40007800340050005D3B050A93178A01E18755
:101B5000F11BE351FCFE92474E9905042320F90046
:101B6000A2473EC2B24702C63EC459B7131A890102
:101B7000135A8A41131D240093178A01E18763CF0A
:101B8000970092470A044E941CC0A2470509137996
:101B9000F90F3EC2B24702C63EC485BFB3079A03DF
:101BA00013152A0056950841780034005000050AA4
:101BB000EA97DA978C439933C1B70000197106C2CE
:101BC00012C416C61AC81ECA22CC26CE2AD02ED2BD
:101BD00032D436D63AD83EDA42DC46DECAC0CEC26D
:101BE000D2C4D6C6DAC8DECAE2CCE6CEEAD0EED29D
:101BF000F2D4F6D6FAD8FEDA97050000938505727E
:101C00008841E700050092402242B2424243D2435B
:101C10006244F244025592552256B2564257D25768
:101C20006258F25806499649264AB64A464BD64B60
:101C3000664CF64C065D965D265EB65E465FD65FE8
:101C40000961730020300000972100209381813BBF
:101C500017510020130101BB17F5FFFF1305C53A0B
:101C6000970500209385053A171600201306C6FD38
:101C700063FAC5008322050023A0550011059105D4
:101C8000E3EAC5FE17A5010013054553971500208B
:101C90009385C5FB171600201306C66563FAC500B9
:101CA0008322050023A0550011059105E3EAC5FE36
:101CB0001715002013050564974500209385854C72
:101CC0006377B500232005001105E36DB5FEFD42E5
:101CD000739002BC8D4273904280B72200009382C1
:101CE000828873900230970200209382A23193E29F
:101CF000320073905230974200009382A2F47390A6
:101D000012346FC0E42F73002030397101436EC666
:101D100019A0397141536AC866CA62CC5ECE19A057
:101D2000397101535AD056D252D44ED64AD826DAF7
:101D300022DC06DE33016140828241114AC026C2A4
:101D400022C406C68282B24D4101024D924C224C01
:101D5000B24B4101024B924A224AB2494101024927
:101D600092442244B240410182803D432A876373FA
:101D7000C3029377F700BDEFADE5937606FF3D8A8A
:101D8000BA960CC34CC30CC74CC74107E36BD7FED4
:101D900011E28280B306C3408A069702000096963D
:101DA0006780A6002307B700A306B7002306B70085
:101DB000A305B7002305B700A304B7002304B700A9
:101DC000A303B7002303B700A302B7002302B700A1
:101DD000A301B7002301B700A300B7002300B70099
:101DE000828093F5F50F93968500D58D9396050126
:101DF000D58D61B79396270097020000969686824C
:101E0000E78086FA9680C1171D8F3E96E374C3F86B
:101E1000A5B73367B500FD530D8B79E7B7877F7F93
:101E20009387F7F710419441B372F6003363F600DD
:101E3000BE92B3E262006397720C6318D6065041FB
:101E4000D441B372F6003363F600BE92B3E262008F
:101E50006398720A631BD60410459445B372F6006A
:101E60003363F600BE92B3E262006391720A631EAE
:101E7000D6025045D445B372F6003363F600BE92E5
:101E8000B3E26200639A72086311D6021049944962
:101E9000B372F6003363F600BE92B3E2620063935E
:101EA00072085105D105E30FD6F613170601939773
:101EB0000601631CF7001357060193D7060133058B
:101EC000F7409375F50F91E982804183C183330513
:101ED000F7409375F50F91E182801377F70F93F731
:101EE000F70F3305F74082800346050083C60500DF
:101EF000050585056313D60065FA3305D640828053
:101F000011059105E312D6FE014582802105A10548
:101F1000E31CD6FC014582803105B105E316D6FCF1
:101F2000014582804105C105E310D6FC0145828050
:101F3000B717004003C777051377E70FA38BE704B4
:101F4000130700F8A38DE7043D47238CE70413072C
:101F50005003A38CE70403C7A7051377D70F238D7E
:101F6000E7048280B717004003C7E7020D894111DB
:101F70001377C70F498F93068008F3B6068093F650
:101F8000860836C601000100930670052380D70439
:101F9000930680FA2380D704010001002387E7021B
:101FA00023800704B247F3A7078001000100410125
:101FB000828041112A83014E930E407E130F001937
:101FC000930F400663E56E12930800191303400651
:101FD000B3781503854E0D4FA14F337365020D89FC
:101FE0001335150063EFBE121308F6FF7946729899
:101FF0004208135808013307C70213D61700BE075B
:1020000032976146B3F6C60213068070B386C602E5
:102010003697A166F58F42075D8FB716004083C7DC
:10202000F60293F70708A303F1000346710083C784
:10203000F60293F70708E394C7FE83477100B716CB
:10204000004093F7F70F6388071293078008F3B7F0
:10205000078093F787083EC401000100B7170040CE
:10206000930670052380D704930680FA2380D70453
:102070000100010023AA070383C6170393E606089D
:10208000A388D70223800704A247F3A70780010093
:1020900001001166B71700407D16D45BC85F9385B9
:1020A0004703A98EF18EF5FA93068008F3B60680F1
:1020B00093F6860836C6010001009306700523805A
:1020C000D704930680FA2380D7040100010098C149
:1020D00003C7170313670704A388E70223800704D5
:1020E000B247F3A7078001000100410182807D1300
:1020F0003368E3039308E016630E08003368F303C4
:102100009308D016630808009378330093B818003A
:102110009388D81633081E01131E0801135E0E01A2
:1021200055B56393E50305486386080001486303DA
:1021300003002A8871087298FD15131E0801C20554
:10214000135E0E01C18179BD13F8150063F4BF0061
:102150007908D5B713381800E5BF83C7F60293F79F
:102160000708A303F1000346710083C7F60293F743
:102170000708E394C7FE8347710093F7F70FF1DF79
:10218000E9B531714AD966CB06DF22DD26DB4ED7B1
:1021900052D556D35AD15ECF62CD6AC96EC7AA8CCA
:1021A00002D8EF00901C2A8993078008F3B70780B4
:1021B00093F787083EDA01000100B71700401307C4
:1021C00070052380E704130780FA2380E7040100E9
:1021D000010003C7F7021377770FA387E70203C74E
:1021E000F70213678700A387E70223800704D2570B
:1021F000F3A70780010001000545AD33130780C137
:102200003347E902116A93070AE893065002BD6951
:10221000930BA004814A014B1304800893047005BA
:102220007D1AB347F9023307D7023EC0FD873ECC83
:10223000938709A69309803E3347F7023AC27D8708
:102240003AC4334739038549B399990193D9394041
:10225000B306D702B30B7703B3C6F602B3CBFB02C8
:1022600036C6FD8636C893D6FB4136CEB7460F003C
:10227000938606243349D9028566938606FAB39677
:102280009601B389E902130760553309D902930611
:102290000010B389E9023349D902B3C9F902931690
:1022A000390036CA37190040FD8636D0930D09042F
:1022B00093D7F9413ED2F336048093F6860836DC94
:1022C00001000100930770052380FD00930680FA4A
:1022D0002380DD00010001008346390593F6860F57
:1022E000A309D9048346390593E61600A309D90446
:1022F00023800D00E256F3A6068001000100130CB6
:1023000080FA116DF336048093F6860836DE0100FC
:102310000100930770052380FD0023808D010100DB
:10232000010083463905216693E60602A309D90414
:1023300083560905B3E6A6012318D9048356090577
:10234000D18E2318D90423800D00F256F3A60680FF
:10235000010001008346390593F60602638A0618D8
:1023600003463905218A6DDE0818EF001004733624
:10237000048013768608B2C20100010023809D000C
:1023800023808D0101000100B717004003C6370507
:102390001376F60DA389C70403C637051366060234
:1023A000A389C704835609052166B3E6A60123184D
:1023B000D90483560905D18E2318D90423800D0032
:1023C0009646F3A60680010001008346390593F680
:1023D00006026386061483463905A18AEDFE97003E
:1023E0000020E78040CBAA8636D497000020E78003
:1023F00080CAA256E30AD5FE835609054255B3E6C4
:10240000A6012318D904C12783463905A18AEDDE28
:10241000035609058346290582473376CA00B30669
:10242000DA0293D5F641B296B388F640E24733B864
:10243000C6002E983308F840A247B3B616013308F9
:10244000D84063C70701631DF800924763FA17017C
:10245000C247634DF80E63950701B24763E8F80E73
:10246000894663E7660FF2469315180013D3F80107
:102470005E8613951800B365B30042D646D4EF606C
:10248000213A3258050B137BFB0F6347000163129F
:102490000838A258638F083613081500B336A80011
:1024A000B69513D6F5013298B336C800AE961358D8
:1024B0001800FE06B3E6060173360480137686081C
:1024C000B2C60100010023809D0023808D01010020
:1024D00001000356C902B296C206C1822316D90270
:1024E00023800D00B646F3A606800100010019BD49
:1024F000F336048093F68608B6C0010001002380FD
:102500009D0023808D01010001008346390593E67B
:102510000602A309D90423800D00864605BDF336C3
:10252000048093F68608B6C40100010023809D0054
:1025300023808D01010001008346390593E60602E0
:10254000A309D90423800D00A646A5BDE30D0BF019
:10255000F336048093F68608B6C80100010093069E
:1025600080FA23809D002380DD0001000100834666
:10257000390593F5FC0F93F6860FA309D90483461A
:102580003905CD8EA309D90423800D00C646F3A6D4
:10259000068001000100130580FA03463905930601
:1025A00039051D8A631496297336048013768608CC
:1025B000B2CC01000100130680FA23809D00238025
:1025C000CD000100010003C606001376F60D23803E
:1025D000C60003C60600136606022380C6008356A3
:1025E00009051166D18E2318D90483560905216681
:1025F000D18E2318D90423800D00E646F3A6068069
:1026000001000100130680FA8346390593F606029D
:102610006388062483463905130C3905A18AFDDA3F
:1026200008186123F336048093F68608B6D00100BB
:102630000100930680FA23809D002380DD000100C5
:10264000010083460C00116693F6F60D2300DC00B2
:1026500083460C0093E606022300DC00835609053E
:10266000D18E2318D904835609052166D18E2318EB
:10267000D90423800D008656F3A6068001000100D0
:10268000130680FA8346390593F606026385062011
:1026900083463905A18AEDFE97000020E780A09FC0
:1026A0002A8C97000020E780009FE30C85FF83566B
:1026B000090511664255D18E2318D9042923834672
:1026C000390513063905A18AFDDAF336048093F63D
:1026D0008608B6D401000100930680FA23809D008D
:1026E0002380DD00010001008346060093F6F60D0D
:1026F0002300D60023800D00A656F3A60680010015
:1027000001008356090503462905D247B376DA004E
:102710003306CA021305800C9355F6413696330DE5
:10272000F6408257333CD6002E9C3336A601330C3C
:10273000FC40330CCC403308850392564E86B335AB
:10274000A5033305A503C295EF60810D63468001A3
:10275000631E0C16630C0D16130615003335A60008
:102760002E959356F5013696B335D600AA959396D5
:10277000F50105828585D18E6346B000639D051AFB
:10278000638B061A0356C90215823305D600333609
:10279000C500B2956348B000639105241306F00F9D
:1027A000637DA622894663F3561593078008F3B725
:1027B000078093F78708BED6010001003717004055
:1027C000930770052300F704930780FA2300F704AA
:1027D000010001008356C70289678117D58FC207A0
:1027E000C1832316F70223000704B657F3A7078017
:1027F00001000100FA506A54DA544A59BA592A5A67
:102800009A5A0A5BFA4B6A4CDA4C4A4DBA4D296126
:1028100082801308F5FF3335A800FD152E95135659
:10282000F5013298B336C800AA9651B1F336048048
:1028300093F68608B6CA0100010023809D0023801C
:10284000AD000100010083463905CD8EA309D904EE
:1028500023800D00D646F3A606800100010035BB9B
:10286000F336048093F68608B6CE0100010023807B
:102870009D002380CD00010001008346390593E6C9
:102880000602A309D90423800D00F646F3A60680AC
:102890000100010095BBF336048093F68608B6D29A
:1028A0000100010023809D002380CD000100010074
:1028B0008346390593E60602A309D90423800D0057
:1028C0009656F3A60680010001006DBB9306F5FF46
:1028D00033B5A600FD152E959355F501AE96B3B50B
:1028E000B600AA951396F501858269B5F336048082
:1028F00093F68608B6D801000100930680FA23807B
:102900009D002380DD00010001008356C902056699
:10291000011693F6F60FD18EC206C1822316D90294
:1029200023800D00C656F3A6068001000100850A2B
:1029300093FAFA0F49B233E6B60045C20356C9020C
:102940003305D0403338A000B305B040B38505410E
:1029500015826345B000D1E16371A608894663F032
:10296000560593078008F3B7078093F78708BEDA08
:1029700001000100B7170040130770052380E7042A
:10298000130780FA2380E7040100010003D7C70280
:102990007D8B2396E70223800704D65781BDF3364B
:1029A000048093F68608B6DC01000100930680FAE5
:1029B00023809D002380DD00010001008356C902B1
:1029C0000566011693F6F60FD18EC206C182231654
:1029D000D90223800D00E656B9B793078008F3B7F4
:1029E000078093F78708BEDE01000100371700401B
:1029F000930770052300F704930780FA2300F70478
:102A0000010001000356C70293975600B297C20710
:102A1000C1832316F70223000704F657C1BB914771
:102A200063EEB70217870100130707B08A05BA954E
:102A30009C41BA978287B717004003A7470B1345FD
:102A4000F5FF698F23AAE70A03A7070B698F23A85D
:102A5000E70A03A7070A798D23A0A70A8280B71780
:102A6000004083A6470B1347F5FFF98E23AAD70A28
:102A700083A6070B558D23A8A70A83A6070A758F7F
:102A800023A0E70A8280B717004003A7470B498FAE
:102A900023AAE70A03A7070B1345F5FF45BFB7179E
:102AA000004083A6470B1347F5FF758F23AAE70A5B
:102AB00003A7070A598D4DB7B717004003A7470B67
:102AC000498FEDB7914763EEB702178701001307EF
:102AD000E7A68A05BA959C41BA978287B717004046
:102AE00003A7470D1345F5FF698F23AAE70C03A73A
:102AF000070D698F23A8E70C03A7070C798D23A086
:102B0000A70C8280B717004083A6470D1347F5FF37
:102B1000F98E23AAD70C83A6070D558D23A8A70CE1
:102B200083A6070C758F23A0E70C8280B71700409F
:102B300003A7470D498F23AAE70C03A7070D1345E9
:102B4000F5FF45BFB717004083A6470D1347F5FFB4
:102B5000758F23AAE70C03A7070C598D4DB7B7173C
:102B6000004003A7470D498FEDB7B71700408847CE
:102B7000420541819377050491EB9377F501375531
:102B8000E801130505803345F50282809377050C33
:102B9000130700046397E7009377F50137459C1C02
:102BA000CDB72165130505D0828037E700E01C43CF
:102BB0005443A183E206D58F1CC1FD572320F7188B
:102BC0002322F718828013178500B7E700E023A0BF
:102BD000E710618123A2A7108280B7F700E0884741
:102BE000CC478280814737370040A14663C4C70085
:102BF000328582800345B740E38EA6FE3385F5001B
:102C00000345050085072304A740CDB7970700209B
:102C10009387476A9C43173700201307A7563E95B2
:102C2000636EE500174700201307C79D6368A70080
:102C3000170700202320A7683E858280FD57EDBF3F
:102C4000411122C406C62A840D372947B307E5027D
:102C5000B2408D83B3D7870222449507B3D7E702EA
:102C600037370040C207C1832316F7004101828035
:102C7000716541111305052006C6D937B7370040E5
:102C8000130770F82381E7000D47A381E7001307BE
:102C90000004A380E70005472387E700B240410115
:102CA000828037370040834727001A0593F7F703E0
:102CB000C98F93F7F70F2301F7008280B7370040E1
:102CC00003C7170019C9D98DA380B70003C7070030
:102CD000136787002380E700828093C5F5FFF98D95
:102CE000A380B7008280B73700402147B736004045
:102CF00091E1828003C6B700E30CC7FE05050346D9
:102D0000F5FFFD15C2052384C600C181D5B7411169
:102D100022C406C62A84913D2947B307E502B24082
:102D20008D83B3D7870222449507B3D7E70237379D
:102D30000040C207C1832316F740410182807165BC
:102D400041111305052006C6D937B73700401307D0
:102D500070F82381E7400D47A381E7401307000483
:102D6000A380E74005472387E740B24041018280C6
:102D7000CC41411106C6328503C6150083C5050046
:102D800022064D8E42068D654186138875A2630C1E
:102D90000611634BC804138845A26300060D634AFD
:102DA000C800938535A26301B60823900600294622
:102DB0004DA0138855A26305060D938565A2E31601
:102DC000B6FE8D451D4663E6E5081146198E63F390
:102DD000C7003E86B7E704002390C600FC479795DE
:102DE00001009385A5379DA0138895A26303061162
:102DF000634E060D1388A5A263000613938505A5EF
:102E0000E315B6FA99451D4663E5E504198E63F3AB
:102E1000C7003E86B7E704002390C600FC4797052D
:102E200000209385A5491DA09D451D4663E3E5024D
:102E30002146198E63F3C7003E86B7E70400FC47BE
:102E40002390C600970500209385C54ABA958297BE
:102E50000146B240328541018280AD451D46E3EA1C
:102E6000E5FE3146198E63F3C7003E86B7E70400DE
:102E70002390C600FC47977501009385256FF9B72D
:102E8000B1451D46E3E7E5FC3546198E63F3C700FF
:102E90003E86B7E704002390C600FC479775010003
:102EA0009385C56D65B78D451D46E3E4E5FA11468A
:102EB000198E63F3C7003E86B7E704002390C6006F
:102EC000FC47979501009385252A49B78D451D46F6
:102ED000E3E1E5F81146198E63F3C7003E86B7E7D4
:102EE00004002390C600FC4797950100938585292F
:102EF000B1BFA5451D46E3EEE5F42946198E63F3FF
:102F0000C7003E86B7E704002390C600FC479775CC
:102F100001009385E5641DBFB5451D46E3EBE5F271
:102F20003946198E63F3C7003E86B7E70400239045
:102F3000C600FC47977501009385856101BFB7E71F
:102F4000040003A3071397060020938626D9414661
:102F5000A54517050020130565CF02832D4559EFC0
:102F600003C5050009476317E50803A8450041119B
:102F700006C6034718003285034608002207416849
:102F8000518F930828FE6308170363E9E8000518CA
:102F9000630307052390060029451DA8130648FE74
:102FA000630BC7021518E31707FF15463E87637BBF
:102FB000F602154705A83E8691C30546B7E704000B
:102FC000FC472390C6004206CC45418282970145CA
:102FD000B240410182801306700F3E876374F60091
:102FE0001307700FB7E704002390E600FC471316A1
:102FF0000701D9BF23900600054582808280416782
:1030000079176304E504411122C406C685472A8462
:10301000639FF500B7E7040022852244B24003A372
:103020008713970500209385A52D410102838947C9
:103030006399F500B7E7040083A7070B85458297DE
:1030400071D9B2402244410182808280797122D4B8
:1030500052CC2E842A8A9775010093856554177582
:1030600001001305A55506D63AC626D24AD0B68425
:1030700032894ECEEF501146A68517750100130513
:10308000E554EF5031452945EF50114983478400FD
:1030900093F70702E1E78349040089470545324772
:1030A0006396F908544083C7160083C60600A2073A
:1030B000D58FC166138616FE638CC7028D16638F8B
:1030C000D7068D669386269029456391D706B7E784
:1030D0000400A285225403A34714B250F249A686E5
:1030E0004A86925402595285624A85474561028355
:1030F0002D450DEF9307700F354563E99702B7E74C
:103100000400FC4748441306700FCA858297814922
:10311000970700209387871F9C43014581CB9C43E1
:1031200091C74E852686CA8582970145B2502254A2
:1031300092540259F249624A456182802D457DF7D9
:103140009307700F3545E3E397FEB7E70400FC47AC
:1031500048441306700FCA8582975DBF2145F9B7B1
:10316000411122C437E404008327841326C2AA84B1
:10317000416506C697050020938585187D158297C1
:103180008327C40A170500001305A5E785888297E1
:1031900095C0032304132244B240924497060020B2
:1031A000938686C54146C545170500201305C5B35E
:1031B00041010283B2402244924401454101828090
:1031C00019C59707002023A3A71401458280454510
:1031D00082801147636AA70A977601009386063BAF
:1031E0000A0536951841411106C63697AE87B28555
:1031F00002871307700F6145639DE700B7E704007E
:10320000FC471306700F170500201305E51682977B
:103210000145B2404101828005476145E39BE7FEDD
:10322000B7E70400FC470546170500201305050D08
:10323000F9BF1307700F6145E39DE7FCB7E7040092
:10324000FC471306700F1705002013056522C1B750
:103250001307700F6145E39EE7FAB7E70400FC47E8
:103260001306700F17050020130505304DB71547DD
:103270006145E390E7FAB7E70400FC4715461705F8
:1032800000201305250861B709458280411126C237
:10329000B7E4040083A7C41322C44AC006C62E8420
:1032A000970500209385C5052A898297058905C55C
:1032B00097070020938747A383D7A70BA28503A373
:1032C000440D2310F4002244B24092444A8502493E
:1032D000014641010283B2402244924402494945D9
:1032E000410182809707002023840702970700206E
:1032F00023A20702B717004003A7070CB706C0FFB9
:10330000FD16758F23A0E70C03A7070DB706400035
:10331000558F23A8E70C03A7070C3D9B23A0E70CC0
:1033200003A7070D1367070123A8E70C8280B717CF
:10333000004003A5470C83A7470C5981134515008E
:10334000C18B058999E3136525009707002083C782
:1033500027FC6380A70297070020238BA7FA11C9D7
:1033600097070020938707FB03A30700630303006D
:103370000283828011456FE0DFE0411193962500C2
:10338000AA852D4506C697F0FF1FE780C017B240FB
:10339000014541018280011122CC06CE3714004044
:1033A00026CA4AC84EC652C483447405034AB405AB
:1033B0008349840503499405EFE09FB78347A4053B
:1033C00093F4F40F137AFA0F93E71700230DF40424
:1033D00093F9F90F1379F90FB717004003C7A70541
:1033E000058B6DFF03D5C705A38D4705238C3705D6
:1033F000A38C2705A38B9704F2406244D244424930
:10340000B249224A0561828041119397050122C485
:1034100006C626C2C1872E8463DC0700B7E4040019
:10342000FC54829719C1BC5482972165218D3DA01F
:1034300093F7150013C5150095E393F7250085C78D
:10344000FD35B7E70400BC4F1306000A8945170590
:1034500000200345A5EC829713452400B240224486
:103460009244410182809397250163D50702B7E416
:10347000040083A7C41E8297F53DBC4C37F60200BA
:10348000130606E0896517050020034525E98297A4
:10349000096569BF939715010145E3D107FC1775CD
:1034A000010013056519EF50B117B7E70400BC4FD1
:1034B00013060064916517050020034525E68297F1
:1034C0001165ADB72D71232A9110FD74E98C232C61
:1034D000811023282111232631112A84AE893289B3
:1034E000930600100A86A6852D45232E111097F00D
:1034F000FF1FE780400113154401B7E70400FC47B4
:1035000051810A0513962900CA850A958297A685D6
:1035100085660146254597F0FF1FE780C0FE0A86B5
:10352000A68593060010294597F0FF1FE780A0FDB0
:103530008320C11103248111832441110329011126
:103540008329C11015618280B7F7070003C70701FF
:10355000411106C622C426C24AC0A547631AF70015
:103560009537B2402244924402490145410182808C
:1035700013942500AA843289A286AA85014625458E
:1035800097F0FF1FE78020F8A2864A86A685294586
:1035900097F0FF1FE78020F7E9B71D71A2CC37E451
:1035A00004005C5C485886CE4946977501009385B7
:1035B0002504829701E9177501001305A504EF5052
:1035C000310601A0B7F600E0795798CAFD57DCCA6A
:1035D0000567B7E700E023A0E7101306F00290C2EA
:1035E00023A0E71801000100370700201847130641
:1035F000000481459706002023A0E6D24157A38A04
:10360000E7403C440808829797170020938787DE9D
:103610003EC8856713870760231AE1001D673ACC0F
:1036200037070105130707103ACE9387B7D313075F
:10363000B00F2310E1022312F102054797F7FFFFB5
:103640009387E7592301E1023ED8170700001307CB
:1036500007D397070000938747D4B7F50700BAC28E
:103660003EDC17070000130767EE970700009387FB
:10367000A7D081463000E1051945BAC43EDE97F077
:10368000FF1FE78040E818088147994630003E96C2
:103690000346060085070507A30BC700E398D7FE7E
:1036A000C24791C70357410185676373F70001A0C3
:1036B000B7E7040083A7470A08088297AA8501C9CB
:1036C00017750100130545F5EF50C16001A0F640E4
:1036D000664425618280411126C2B7E4040083A7B5
:1036E000040806C622C417050000130525D28297D8
:1036F00017040020130484C22300A4003128DD36FF
:1037000003450400224403A38405B24092441306F7
:103710000032896541010283797106D622D41307EC
:103720008008F337078093F787083EC20100010045
:10373000B7170040930570052380B704130680FA7D
:103740002380C7040100010083C6F70293F6A60F89
:10375000A387D702238007049246F3A606800100C0
:10376000010073370780137787083AC4010001000E
:103770002380B7042380C7040100010003C7F702B8
:1037800013672700A387E70223800704A247F3A754
:103790000780010001000545EFE0CFFCE13E014755
:1037A00081468147054685451305407EEFE07F80D1
:1037B00037E404003C446800514681458297B707CE
:1037C000C0A83EC8B787E803938707D03ECA97F7DB
:1037D000FF1F9387C7BD3EC67C5868008297B250D2
:1037E0002254456182804111977501009385054BF4
:1037F00017750100130585DC06C6EF50A14D17753E
:10380000010013056562EF50E14CB24029454101CA
:103810006F50815041119775010093856549177567
:1038200001001305A5D906C6EF50C14A177501005E
:103830001305455EEF50014AB240294541016F50E2
:10384000A14D411122C406C6834705002A849DC3A9
:10385000977501009385854B17750100130505D6F3
:10386000EF5041474C401775010013052570EF508C
:1038700061461DA058411DE79775010093850549D4
:1038800017750100130585D3EF50C144177501006A
:103890001305456FEF5001442244B24029454101D0
:1038A0006F508147A1679386D7036311D70297753D
:1038B00001009385A54517750100130525D0EF502C
:1038C0006141177501001305E56CE9B7ED079775C0
:1038D00001009385A54317750100130525CE6319D3
:1038E000F700EF50213F177501001305E56B5DB739
:1038F000EF50413E4C40177501001305E56C85BF44
:103900004111977501009385E53B1775010013057B
:10391000E5CA06C6EF50013CB240294541016F504F
:10392000A13F797122D426D24AD02E842A8981459A
:10393000B2844800714606D6EFE02FC397F7FF1F09
:103940009387076BDC4783D70700231421012313D8
:10395000F100EF2030069547A305F1009307401FC3
:103960003EC6FD572305A100230AF100EF20D01623
:103970002686A2854800EF20D006B25022549254E9
:10398000025945618280970700202392079C970780
:103990000020238D079AB7E70400BC47411106C6F3
:1039A000414681451385012E8297EF10D06AEF10B2
:1039B00050480145EF30C01803C7C12F9307F00AE4
:1039C000631DF7009307F0F889451385C12F238EF7
:1039D000F12EA38E012EEF300043EF30E0528145EF
:1039E000370504009707002023AE079497070020AF
:1039F00023980794970700202385079497070020B2
:103A0000239D07929707002023980792970700208D
:103A1000239707929707002023980792EF20003BF7
:103A20000145EF300045977501009385252C1775EA
:103A300001001305A5B8EF50E12917750100130522
:103A4000E55EEF502129B240294541016F50C12C5C
:103A5000411122C406C626C293F715002E84638D39
:103A6000070C814617F6FF1F1306065685451705F6
:103A700000200355258CEF80B00D05C5977501001A
:103A80009385852717750100130545B3EF508124F1
:103A900017750100130505C9EF50C1232945EF50E3
:103AA000A12797750100938525251775010013053A
:103AB000E5B0EF502122177501001305E5C7EF505F
:103AC00061212945EF50412517F5FF1F1305455288
:103AD0005C4505472390E700EFF0E01D9775010076
:103AE0009385852117750100130545ADEF50811EA3
:103AF00017750100130585C5EF50C11D2945EF500D
:103B0000A121930710F8238EF12E9707002083D769
:103B10002782A38EF12E1385C12FA1839145238F78
:103B2000F12EA38F012EEF30002E13451400B2406A
:103B3000224492444101828093F72500D1CB17F7AC
:103B4000FF1F0357E77F51C397F6FF1F9386867FBA
:103B50009442977701009387674F17F6FF1F03463C
:103B6000467E81451385012EEF40D00BAA8431CDCE
:103B7000977501009385051F17750100130505A4AE
:103B8000EF504115A685177501001305A5BDEF502F
:103B900061142945EF50411897F7FF1F2392077AC8
:103BA000930710F8238EF12E97F7FF1F83D74778DE
:103BB000A38EF12EA183238FF12E91458D4713857E
:103BC000C12FA38FF12EEF3000241345240085B7B9
:103BD00093F74500B1CF977501009385A518177528
:103BE00001001305A59DEF50E10E177501001305A7
:103BF00025B9EF50210E2945EF500112930720F807
:103C0000238EF12E97F7FF1F83D72773A38EF12EF4
:103C1000A183238FF12E8547A38FF12EEF20C06B58
:103C20001385C12F9145EF30001E1345440001B7A5
:103C300093F785008DCF977501009385A5121775B1
:103C400001001305A597EF50E10817750100130552
:103C500065B4EF5021082945EF50010C97F7FF1F7D
:103C60002390076EEF40F00813458400C9B593F721
:103C70000501A5C3854517F5FF1F0355056CEF002A
:103C8000B152977501009385E50D17750100130575
:103C9000E592EF502104177501001305E5B0EF50D0
:103CA00061032945EF504107930730F8238EF12E29
:103CB00097F7FF1F83D76768A38EF12E1385C12F57
:103CC000A1838D45238FF12EEF30E01313450401BE
:103CD000B9BD93F70502B5C39775010093858508B3
:103CE000177501001305858DEF40D17E1775010012
:103CF0001305C5ADEF40117E2945EF50E101930753
:103D000040F8238EF12E97F7FF1F83D7E762A38E2B
:103D1000F12EA183238FF12E8547A38FF12E97F7E4
:103D2000FF1F239B0760EF20205B1385C12F914568
:103D3000EF30600D13450402DDBB93F70504CDC7DA
:103D40009775010093850502177501001305058716
:103D5000EF405178177501001305C5A8EF40917722
:103D60002945EF40717B83C7C12F1307700A638811
:103D7000E7041307800A6386E7061307600A639760
:103D8000E702930760F8238EF12E97F7FF1F83D782
:103D9000075BA38EF12EA183238FF12E8547A3838A
:103DA000F130B1451385C12FEF30E005EF20C0524F
:103DB0001345040497F7FF1F239307588DBB930700
:103DC00070F8238EF12E97F7FF1F83D74757A38EE6
:103DD000F12EA183238FF12E8547A380F1309945E1
:103DE000D1B7930780F8F1BF93F705080145E38049
:103DF00007D4977501009385E5F617650100130553
:103E0000E57BEF40316D177501001305259FEF40ED
:103E1000716C2945EF4051709307A0F8238EF12E65
:103E200097F7FF1F83D74752A38EF12EA183238FCD
:103E3000F12E8547A38FF12E97F7FF1F239607508A
:103E4000EF2080491385C12F9145EF20D07B13458A
:103E50000408F1B9411122C497750100938545EC1E
:103E60002A84176501001305657506C6EF40916643
:103E70004C40177501001305E50CEF40B16529456D
:103E8000EF409169034704009307F00F6319F702AD
:103E9000977501009385C5E8176501001305057244
:103EA000EF4051634C40177501001305A50AEF4020
:103EB00071622244B240294541016F40F165B24030
:103EC00022444101828085CD411122C41765010041
:103ED0001305C56E2E8497750100938565DF06C6B0
:103EE000EF40515FA285177501001305E511EF4002
:103EF000715E2244B240294541016F40F1618280E8
:103F0000411122C426C22E84AA849775010093858C
:103F1000E5DC176501001305656A06C6EF40915B95
:103F2000177501001305050FEF40D15A2945EF40E1
:103F3000B15E97750100938565DA97F7FF1F239BA4
:103F4000973E1765010013056567854497F7FF1FC6
:103F50002390873E97F7FF1F239D973C97F7FF1FFE
:103F60002397873EEF40115797F5FF1F83D5253ED6
:103F7000177501001305850AEF40D1552945EF401B
:103F8000B15997F7FF1F2383973CEF10806A228572
:103F9000EF20103B0545EF20D06D97F7FF1F93876B
:103FA0002705DC4703D70700C167FD176312F70237
:103FB0002244B7E70400B240924403A3870517F5F3
:103FC000FF1F034525361306000A8545410102837C
:103FD000B2402244924441018280011122CC37E454
:103FE00004005C5C06CE26CA3546977501009385B1
:103FF000E5E4177501001305657C829701E91765F3
:10400000010013052560EF40B16101A097F7FF1F84
:10401000938707653EC4B7F507008567938707C098
:10402000814617F6FF1F13062630E10519453EC6E7
:1040300097E0FF1FE780204D7C44194697F5FF1F4E
:104040009385852E138541278297340017F6FF1F2D
:104050001306862D977501009385053417750100A9
:1040600013050535EF408014AA8415C99775010022
:10407000938545CE1765010013054554EF409145E2
:10408000A68517750100130565DCEF40B14429458D
:10409000EF409148F2406244D24405618280EFA033
:1040A000602B17750100130565D1EF30C02FEF703D
:1040B000A019EF00313817F5FF1F130525F0EF00A9
:1040C000112517750100130565D0EF007138AA841A
:1040D000EF30700AEFC0805DEF20D157EF4090269F
:1040E000EF30B069EFE0703A97750100938585C6AF
:1040F000176501001305854C89C8EF40B13DA685C1
:10410000177501001305C5D649B7EF40B13C1775C7
:104110000100130525D8EF40F13B2945EF40D13F81
:10412000EFE0101DEFB040476305050E85453705EC
:104130000400EF10B049977501009385A5C117657C
:1041400001001305A547EF40F1381775010013056D
:10415000E5D5EF4031382945EF40113C97F7FF1F77
:10416000938747D983D7070017F7FF1F2311F71E3F
:10417000854717F7FF1F230BF71CEF10C068EF10E0
:10418000404B17F5FF1F0355851CEF20701B97F759
:10419000FF1F83C7971BB9EFA303010083274417B1
:1041A00013067100854513055030829797750100FD
:1041B000938545BA1765010013054540EF409131DD
:1041C000177501001305C5D0EF40D1302945EF40E8
:1041D000B134977501009385E5B7176501001305A4
:1041E000E53DEF40312F17750100130565D4EF4011
:1041F000712E71BD977501009385C5B517650100D6
:104200001305C53BEF40112D177501001305C5CFF0
:1042100065BF977501009385E5B317650100130528
:10422000E539EF40312B17750100130525E0EF400C
:10423000712A2945EF40512E0145EF20904351BF8F
:10424000411122C437E404008327041A06C682976A
:10425000EF20D0178327040817F5FFFF1305857F8C
:10426000829797F7FF1F238FA70A17F5FF1F1305E4
:1042700025D8EF2040332244B2404101B9BBB7E713
:104280000400FC471171A2DDCAD986DFA6DBCED7B8
:104290002E8432892E86AA851385C12F8297138793
:1042A000C12F83470700930680029387E70793F7A0
:1042B000F70F63E4F676BA898A07176701001307D8
:1042C000E737BA979C43BA9782878D479775010065
:1042D000938585AA176501001305452E630BF4002D
:1042E000EF40511F176501001305C567EF40911E90
:1042F000FDA2EF40311E1765010013052568EF4050
:10430000711D2945EF405121930720F811469385EF
:10431000C12F4A85238EF12EA38F012EEFF06FE07F
:104320002A840DC597750100938505A517650100C1
:104330001305C528EF40111AA28517650100130562
:10434000A567EF4031192945EF40111D9775010010
:10435000938585A21765010013054526EF40911747
:104360001765010013058566EF40D1162945EF401A
:10437000B11A4165930730FA05469385C12F7D1523
:10438000238EF12EEFF0EFD92A840DC59775010029
:104390009385859E1765010013054522EF40911313
:1043A000A2851765010013052561EF40B11229456B
:1043B000EF409116B7E70400BC4F0566130606C828
:1043C000A14517F5FF1F0345E5F58297FE506E5492
:1043D000DE544E59BE591161828091476301F40247
:1043E0009775010093854599176501001305051D13
:1043F000EF40510E1765010013058560C5BDB7E795
:104400000400FC4F914517F5FF1F0345A5F1829766
:104410009775010093854596176501001305051AE8
:10442000EF40510B176501001305455FEF40910AFE
:104430002945EF40710EEF10306A9145E1A28547A2
:104440006301F402977501009385059317650100D8
:104450001305C516EF401108176501001305855DAA
:1044600071B597F7FF1F239A27EDB7E7040005669C
:10447000BC4F130606C8C145A9B78D476301F402B6
:10448000977501009385458F176501001305051386
:10449000EF405104176501001305855B81BD93074B
:1044A00040F811469385C12F4A85238EF12EA38FA4
:1044B000012EEFF00FC72A84E30A05F0977501007B
:1044C0009385858B176501001305450FEF4091001B
:1044D000A285176501001305254EEF40A17F2945F0
:1044E000EF409103E5B59147E31CF4F8B7E704000A
:1044F000FC4F9305000217F5FF1F0345A5E28297C5
:104500009775010093854587176501001305050B15
:10451000EF40417C176501001305055501BF894730
:1045200063E1870297750100938505851765010092
:104530001305C508EF40017A1765010013050554FE
:1045400075B383C4E12F83C7D12F9775010093857D
:10455000A582A2041765010013054506DD8CEF4016
:104560006177A2851765010013058552EF408176BA
:10457000C2042945EF40417AC1849305D4FF939644
:104580000401C1824A8693F5F50F1385F12FEF10D0
:104590007007E35D90E2930750F8238EF12E83C7F6
:1045A000390022869385C12F85074A85A38FF12E76
:1045B000EFF02FB72A84E30B05E0976501009385A0
:1045C000A57B17650100130565FFEF40A170A2856B
:1045D00017750100130545A209B7894763E18702F2
:1045E000976501009385457917650100130505FD61
:1045F000EF40416E176501001305454BC5B9EF103B
:10460000B04DA2851385C12FEF20E07FC1B38D4748
:104610006301F40297650100938505761765010033
:104620001305C5F9EF40016B176501001305C54976
:1046300075B9B76602000146B7750200054597E0F7
:10464000FF1FE78040EC930760F8238EF12EA38FC5
:10465000012E930700062380F1308947A380F130B3
:1046600023810130A3810130C1472382F1309307B8
:1046700020F9A382F1303146A383A1309385C12F65
:104680004A8523830130EFF0CFA92A84E30005D4C3
:10469000976501009385456E17650100130505F2C6
:1046A000EF404163A285176501001305654335B5E9
:1046B000B1476301F402976501009385E56B1765C7
:1046C00001001305A5EFEF40E16017650100130538
:1046D000E54229B9B7E70400FC4F9305000417F53C
:1046E000FF1F034525C48297EF10103FB14519BF46
:1046F000914763E18702976501009385E567176538
:1047000001001305A5EBEF40E15C176501001305FF
:10471000A540E9BE83C4013083C7F12FA204DD8C1C
:104720008E04B77702006D14BE942286A6851765A5
:1047300001001305A53FEF40E159B7E70400FC472E
:104740002286938511302800829793160401C18236
:104750003000A685094597E0FF1FE780C0DA2A846C
:1047600019C5176501001305253EEF40616B9307DE
:1047700070F819469385C12F4A85238EF12EA380A8
:104780008130EFF00F9A2A84E30205C49765010097
:104790009385855E17650100130545E2EF4081535F
:1047A000A285176501001305253B05BB99476301E9
:1047B000F410976501009385255C176501001305CA
:1047C000E5DFEF402151176501001305653A39BE59
:1047D000914763E18702976501009385E559176565
:1047E00001001305A5DDEF40E14E1765010013053B
:1047F000A539EDBC83C4013083C7F12FA204DD8C41
:104800008E04B77702006D14BE942286A6851765C4
:1048100001001305A538EF40E14BB7E70400FC4762
:104820002286938511302800829793160401C18255
:104830003000A6850D4597E0FF1FE780C0CC2A8495
:1048400019C51765010013052537EF40615D930712
:1048500080F819469385C12F4A85238EF12EA380B7
:104860008130EFF00F8C2A84E30205B697650100D2
:104870009385855017650100130545D4EF408145A8
:10488000A285176501001305653481B99947630155
:10489000F402976501009385254E17650100130505
:1048A000E5D1EF402143176501001305A5333DBC59
:1048B000B7E70400FC4F9305000417F5FF1F0345FD
:1048C00065A68297EF10502199452DBB8D47630156
:1048D000F402976501009385254A176501001305C9
:1048E000E5CDEF40213F1765010013052531FDBAE5
:1048F0001765010013058531EF4081521305C01281
:1049000097E0FF1FE78020A30145EFE00FAA0D45C8
:10491000EF00F001294597E0FF1FE780C0A197E075
:10492000FF1FE780E0925DB499476301F402976549
:1049300001009385654417650100130525C8EF4004
:104940006139176501001305252D4DB203C71130DC
:1049500083C7013022075D8F9166BA96C206116641
:10496000C1821306F6EF8D476363D60297E7FF1FF8
:10497000938707689C4B03C6F12F9386C70039C6FF
:1049800003D607005DCA8907E39CD7FE8947130752
:10499000A0F811469385C12F4A85238EE12EA38F5F
:1049A000F12EEFE01FF82A84E30205A297650100CB
:1049B0009385853C17650100130545C0EF408131A3
:1049C000A285176501001305652601BE03D6070001
:1049D0006302E60A8907E39BF6FE8D474DBF9147C8
:1049E0006302F4029765010093850539176501009C
:1049F0001305C5BCEF40012E176501001305852482
:104A00006FF0DF8EB7E70400FC4F9305000817F541
:104A1000FF1F03452591829739BC97650100938557
:104A2000A53517650100130565B9EF40A12A176583
:104A300001001305A5226FF07F8B2390E70017E597
:104A4000FF1F1305E55AEFE0A02897650100938545
:104A5000A53217650100130565B6EF40A12717655C
:104A600001001305A520EF40E1262945EF40C12AAA
:104A7000814731BF2390070017E5FF1F13054557F6
:104A8000EFE00025976501009385052F176501006C
:104A90001305C5B2EF400124176501001305851EFB
:104AA000D9B7411122C406C6834705002A849DC395
:104AB000976501009385052817650100130505B06A
:104AC000EF4041214C401765010013052559EF4087
:104AD000612075A05841B707CF009387777D631396
:104AE000F706976501009385E52417650100130516
:104AF000E5ACEF40211E1C448356E4008355C400FE
:104B000003C60700176501001305C556EF40811C59
:104B10002945EF4061200357E40097F7FF1F83D733
:104B200007836307F7008355C4000844EFE0AF9B99
:104B30000356E4008355C40008442244B2404101B6
:104B40006FF0EFF3B707CC009387777D631FF70211
:104B5000976501009385051E17650100130505A6DD
:104B6000EF4041171C448356E4008355C40003C63C
:104B70000700176501001305E54FEF40A11522441A
:104B8000B240294541016F402119B707CE009387F4
:104B9000777D6302F702976501009385A519176574
:104BA00001001305A5A1EF40E1124C40176501007B
:104BB0001305854129BFB240224441018280B7E7F5
:104BC0000400FC4741112E8606C622C426C24AC0F4
:104BD0002E842A89AA851385C12F829797650100A3
:104BE0009385451B176501001305459DEF40810E18
:104BF00083C5C12F176501001305C5C1EF40810DA5
:104C00002945EF4061119384C12F83C704004147B8
:104C10009387070693F7F70F6361F74A1767010059
:104C2000130707AC8A07BA979C43BA9782879D47B8
:104C30006303F402976501009385C51517650100AC
:104C40001305C597EF40010917650100130505BD60
:104C5000EF404108F9AA83C7D12FC9C703C7F12F75
:104C600083C7E12F22075D8F83C70130C2075D8FA5
:104C700083C71130E207D98F17E7FF1F2324F76C92
:104C800083C76400976501009385C510176501000F
:104C90001305C59217E7FF1F2305F76AEF4081034D
:104CA00097E7FF1F9387076A8C4317E6FF1F0346AA
:104CB000466917650100130525B8EF40A101294594
:104CC000EF408105A38E012E2244B2409244024956
:104CD000930700F8238EF12E9D451385C12F4101C6
:104CE0006F206012EF30900C238FA12E9357850018
:104CF000A38FF12E935705012A842380F130935717
:104D000085010145A380F130EF30100B2381A130E4
:104D10009765010093850508176501001305058A4D
:104D2000EF30517B03C62130A285176501001305C2
:104D300025B261B7CD476301F40297650100938501
:104D400065051765010013056587EF30B1781765B4
:104D50000100130565B1EDBD37E404007C44414614
:104D60009385D12F1385012E82971385012EEF0095
:104D7000F022EF00100C83C7E13003C7D130A20747
:104D800003238405D98F17E7FF1F231BF75A130648
:104D9000000A89452244B2409244024917E5FF1FA8
:104DA00003454558410102838D476301F40297652D
:104DB0000100938525FE1765010013052580EF305E
:104DC0007171176501001305E5B959B503C4E12FE9
:104DD00083C7D12F976501009385C5FB2204175522
:104DE00001001305A57D5D8CEF30D16EA28517659E
:104DF00001001305E5A8EF30F16D2945EF30D171C1
:104E00000D469385C12F2285EFE0BFB1AA8415C955
:104E100097650100938505F8175501001305057A7C
:104E2000EF30516BA685176501001305A5A6EF307D
:104E3000716A2244B24092440249294541016F30CF
:104E4000B16D97E7FF1F239A874EB7E704001166FD
:104E500003A38705130606E891452DBF8D4763011F
:104E6000F402976501009385E5F2175501001305DB
:104E7000E574EF30316617650100130565BDC9BBE8
:104E800003C4E12F83C7D12F97650100938585F077
:104E9000220417550100130565725D8CEF30916394
:104EA000A28517650100130525A0EF30B1622945E1
:104EB000EF3091660D469385C12F2285EFE07FA6E6
:104EC000AA840DC1976501009385C5EC17550100B3
:104ED0001305C56EEF301160A68517650100130537
:104EE000E59DB1B797E7FF1F23988744B7E7040014
:104EF000116603A38705130606E89305000259BD52
:104F0000894763E18702976501009385A5E81755F6
:104F100001001305A56AEF30F15B17650100130569
:104F2000E5B53DB383C4E12F83C7D12F9765010059
:104F3000938545E6A2041755010013052568DD8C0D
:104F4000EF305159A685176501001305A598EF307C
:104F500071582945EF30515C22869385C12F2685F3
:104F6000EFE03F9C2A84630905169765010093854D
:104F700065E21755010013056564EF30B155A28550
:104F800017650100130545965DB5854763F68714DF
:104F9000834519002244B24092440249B335B0001F
:104FA00097E7FF1F238CB738176501001305059598
:104FB00041016F303152A2852244B24092444A8569
:104FC00002494101C9A299476301F40297650100B2
:104FD000938545DC175501001305455EEF30914F71
:104FE00017650100130545C3A5B103C4E12F83C7AD
:104FF000D12F976501009385E5D92204175501004B
:105000001305C55B5D8CEF30F14CA285176501007F
:1050100013054590EF30114C2945EF30F14F1946FB
:105020009385C12F2285EFE0DF8FAA840DC197659C
:105030000100938525D61755010013052558EF303B
:105040007149A685176501001305C58DCDB397E796
:10505000FF1F239B872EB7E70400116603A3870574
:10506000130606E89305000835B3854797650100E8
:10507000938545D217550100130545546309F40083
:10508000EF305145176501001305058BD1B6EF30A0
:105090007144176501001305A58BEF30B143294515
:1050A000EF3091472244B2409244024997E7FF1FF4
:1050B0002398072841016F30C0439765010093850D
:1050C00065CD175501001305654FEF30B1401765E9
:1050D00001001305A5B8ADBEB24022449244024976
:1050E00041018280411106C622C4EFE09F8393777D
:1050F000F50F95CB2A8497650100938525CB17552D
:1051000001001305A54BEF30F13C9375F40F1765C3
:105110000100130565EEEF30F13B2244B240294512
:1051200041016F30713FB240224441018280411100
:1051300022C491462A841386013E9D652D4506C6EC
:1051400097D0FF1FE780203CB7F7070003C7070190
:10515000A5476313F70001A09306001001469D6563
:10516000254597D0FF1FE780003A2380813E2244E7
:10517000B24091461386013E9D652945410117D3F2
:10518000FF1F670043385171CAD137E904008327F4
:10519000C904A2D52E8686D7A6D32E84AA851385C8
:1051A000C12F829783C7C12F1307700A638DE70C45
:1051B000636CF7001307600A6382E704BE502E5445
:1051C0009E540E596D6182801307800A6382E71234
:1051D0001307900AE394E7FE8D47630BF416976577
:1051E00001009385A5F4175501001305253DEF3007
:1051F000712E176501001305A5F015A08D476306F4
:10520000F40297650100938565F2175501001305B7
:10521000E53AEF30312C176501001305A5E7EF30B3
:10522000712B2945EF30512F51BF8547176501007C
:10523000130505E817E7FF1F2302F710EF30513E73
:10524000B7750200B76602000146054597D0FF1FFB
:10525000E780602B930760F8238EF12EA38F012E39
:105260009307002623A0F130E57793870721239247
:10527000F130B14523830130A383A1301385C12FC1
:10528000EF10703825BF914763E1870297650100F1
:105290009385C5E91755010013054532EF30912379
:1052A000176501001305C5E29DBF83C4013083C7A4
:1052B000F12FA204DD8C8327C9046D142286938507
:1052C0001130280082978E0493160401B7750200EE
:1052D000C1823000A695094597D0FF1FE780A02224
:1052E000930770F8238EF12E9945A380A13079B7EA
:1052F000914763E1870297650100938525E3175580
:1053000001001305A52BEF30F11C176501001305F3
:10531000A5DD31B783C4013083C7F12FA204DD8C32
:105320008327C9046D142286938511302800829743
:105330008E0493160401B7750200C1823000A69551
:105340000D4597D0FF1FE780001C930780F859BFD9
:1053500017650100130505DCEF30912C1305C01211
:1053600097D0FF1FE78020FD0145EFD01F840D453A
:105370007D3B294597D0FF1FE780E0FB97D0FF1FBB
:10538000E78000ED25BD01114EC697E6FF1F83D6CD
:1053900006FCB28917E6FF1F035646F426CA4AC820
:1053A00006CE22CCAA842E89252397E7FF1F83C728
:1053B000E7F9B1CB03C4440083C73400176501008B
:1053C0001305C5DA22045D8CEF30D1104A86A6851C
:1053D0002285EFF03FD1638F090297E7FF1F83C754
:1053E000C7F68DCB6308090297E7FF1F83C707F550
:1053F00095E36244F240B249CA8526854249D244C7
:1054000005616F105020176501001305A5D6EF3018
:105410003121D1B7F2406244D2444249B2490561D8
:1054200082808347550083454500176501001305B9
:10543000A5D2A207DD8D6F30F109176501001305B4
:10544000A5D06F30F11D8D4763F2B70A011126CA4E
:1054500006CE22CC0344350097E4FF1F83C4F4EE4C
:10546000976501009385C5D1B337800017E7FF1F0B
:10547000A30DF7EC09C497650100938525D1176545
:105480000100130525D1EF30F10497E7FF1F83C713
:10549000D7EB63839700252C97E7FF1F83C7F7EAB5
:1054A0009DC385472306F100B7E7040083A747178C
:1054B000700085451305503082971765010013056C
:1054C00065CEEF30F1159967938757EE2316F100FB
:1054D000680085479145A30781002307F100EF107D
:1054E0009012F2406244D2440561828082808947F2
:1054F00063F2B708011122CC06CE26CA83442500E8
:1055000085472A846398F404914763F0B704034500
:1055100045008347340022055D8D97E7FF1F239FD9
:10552000A7DA1D299967938767EE2314F100834753
:10553000340023059100A305F100834744009545FD
:1055400028002306F100EF10100CF2406244D24410
:1055500005618280FDF89967938767EE2314F10057
:1055600097E7FF1F83D787D7A305F1002305010025
:10557000A183F1B782800111996722CCD51717E476
:10558000FF1F1304A4DC2314F1008347040026CA80
:1055900097E4FF1F9384A4DB2305F10083D7040065
:1055A00028009545A305F100A18306CE2306F1004E
:1055B000EF10700503D60400834504001765010051
:1055C0001305C5BFEF300171F2406244D24405615A
:1055D00082809D677971D9172316F10097E7FF1F25
:1055E00083C7C7D606D62307F1009DCBB7E70400D3
:1055F000FC4741469385012E1305F1008297680010
:10560000CD45EF10500097E5FF1F83C525D41765E2
:1056100001001305A5BDEF30E16BB25045618280FA
:10562000B7E70400BC47414681451305F100829766
:10563000F9B7B76702036971938757AA3EC48567B4
:10564000938727E02316F10097E7FF1F938707D082
:1056500083C7070023248112A30701002307F10059
:1056600097E7FF1F9387A7CE83D7070037E404008F
:10567000232611122318F10097E7FF1F938707C60F
:1056800083D70700414648082319F1007C449385DD
:10569000012E8297F1452800E52A2312A1027C44BD
:1056A0002C002810794682973C44130561041306A8
:1056B000900D8145829730109305700F0145EFD012
:1056C0005FB18320C1120324811255618280B7C764
:1056D000A55A01119387C7333EC497E7FF1F83C7BD
:1056E000D7C63EC6B7F7070003C7070106CE22CCD0
:1056F000A5476313F70001A01164930504F0930616
:1057000000100146254597D0FF1FE780C0DF30001D
:10571000930504F0A146294597D0FF1FE780A0DE3E
:1057200097E5FF1F83C575C2176501001305C5BC4A
:10573000EF30415AF2406244056182800111916567
:10574000A1463000938505F02D4506CE97D0FF1F6A
:10575000E78060DB2247B7C7A55A9387C733631238
:10576000F702B24517650100130545ACB335B0002B
:1057700097E7FF1FA38BB7BCEF30C155F24005611F
:105780008280814517650100130585AC97E7FF1FEF
:10579000A38D07BAEF3001541D3FCDB7B7C7A55A47
:1057A00079719387F7353EC6B7E70400FC47AA85B1
:1057B00006D622D4414608088297B7F7070003C7E8
:1057C0000701A5476313F70001A01164930504E8DE
:1057D000930600100146254597D0FF1FE780A0D211
:1057E0007000930504E8D146294597D0FF1FE78054
:1057F00080D1176501001305E5B3EF306162B25047
:1058000022544561828079719165D14670009385FB
:1058100005E82D4506D697D0FF1FE780C0CE32475A
:10582000B7C7A55A9387F73517650100130545AA31
:10583000631EF700B7E70400FC471385012E4146BD
:105840000C08829717650100130585A6EF30415DAE
:10585000B25045618280B7F7070003C70701A5472B
:105860006313F70001A091654111930600100146F2
:10587000938505E8254506C697D0FF1FE780A0C899
:10588000B240176501001305A59841016F304159D9
:10589000C16769768146FD170506139706014183A6
:1058A0006364B7003E8582803307D5000347070055
:1058B000B98F214713F81700858363050800B18F5E
:1058C000C207C1837D171377F70F6DF78506F1B710
:1058D00049C1A547054763FFB7068347150003473E
:1058E00005003168A207D98F13978700A183D98F4C
:1058F000C207C1831308C8550547639D07054111B9
:1059000006C622C426C203442500914763FD8702D0
:10591000930754006399F502A301C5002182230275
:10592000C5009304340091C6A302D500A1822303CD
:10593000D5002A84A685A93F26942300A4002181AE
:10594000A300A4000147B240224492443A85410199
:10595000828005473A858280B7C7A55A011193878F
:10596000E7343EC42AC6B7F7070003C7070106CECF
:1059700022CC26CAA5476313F70001A091642A84AC
:10598000938504EE930600100146254597D0FF1F2E
:10599000E78060B73000A146938504EE294597D093
:1059A000FF1FE78040B6A285176501001305C59665
:1059B000EF304132EFF0FFC7F2406244D24405615C
:1059C000828001119165A1463000938505EE2D4539
:1059D00006CE97D0FF1FE78000B32247B7C7A55A6E
:1059E0009387E7346314F702B24517650100130586
:1059F000258897E7FF1F2393B78EC205C181EF303B
:105A0000612DEFF01FC3F24005618280D147D1457F
:105A1000176501001305C58717E7FF1F2310F78CD3
:105A2000EF30412B17E5FF1F0355458B3537E1BF9D
:105A3000011126CA06CE22CC93F71500AE848DCB79
:105A4000AD67371700409387A7AA1CC3B7E70400C8
:105A5000BC4F13060019854517E5FF1F0345E58771
:105A6000829713C51400F2406244D24405618280DB
:105A700093F7250063850712976501009385858F4D
:105A80002D464800EF30A11997E5FF1F83C5158CFF
:105A9000854793C4240063E1B70489CD97E7FF1FCE
:105AA00083C7A78A85C3854517050020130585F49C
:105AB000EF1060351395040197E7FF1FA38807884F
:105AC000418155B74165054697050020938585F2CC
:105AD0007D15EFF02FE1F9BF17040020034484F196
:105AE0009707002083C717F122045D8CAD67C205BC
:105AF0009387B755C1816306F40863E68702A967F7
:105B00009387A7556306F40897E7FF1F83C7E783CA
:105B10008DE741652E867D1597050020938585EDDF
:105B2000EFF04FDCB9A0B1679387C755630EF4005F
:105B3000B5679387D755E319F4FC170500201305C3
:105B400065EBEF10402C35A0054617050020130526
:105B500065EAEFF05F8397D7FF1F83C7277F91EB3D
:105B60004800EF30213493150501C1814800EFD082
:105B70008F97A285175501001305C57DEF3081155C
:105B800015BF170500201305E5E6EFF09F89D5B78F
:105B900017050020130505E6EFF03F8AD9BF93F7FC
:105BA00045000145E38107EC175501001305C57B4E
:105BB000EF300127EF10003713C544006DB54111D8
:105BC00022C437E404005C5C06C6354697550100E4
:105BD0009385C52617650100130545BE829701E927
:105BE000175501001305C579EF30812301A08327E4
:105BF000041C82972A840545EF802075EF10C16848
:105C0000EF100147EF70B0292285B24022444101D4
:105C100082801567B71700401307575598C3D843BC
:105C20009D66558FD8C3D843FD76758FD8C3D843AA
:105C30001367F70FD8C335671307C7CC98C38280A3
:105C400041111305800406C622C426C24AC097C06B
:105C5000FF1FE780C04585457D55EFC05FDC85456A
:105C60007D55EFC03FE6371400408327840A8D45F9
:105C70001305002093E707202324F40AEFC03FDA3E
:105C8000B7E40400EFD0AF8BC8581309840C130499
:105C9000C40CEF30E11817650100130525B2EF3091
:105CA00021188327C4FF8545414593E70708232E24
:105CB000F4FEEFC03FE18D4513050008EFC09FE003
:105CC000EFC01FFB0145EFC0DFFD85450545894756
:105CD00017D7FF1F230EF766EFC05FFE37070004DC
:105CE000B7E700E023A0E710EFD03F8BEFD0BF9ED7
:105CF000F935EFF0BFA4EFF0DFCCEFE06FD48D45C6
:105D00000D65EFC03FDC170500201305A5DE856794
:105D10001CC589672320250140C12326250100C910
:105D20005CC983A7841E829783A704081705000017
:105D3000130545D0829797D7FF1F2380A75ABC4CE5
:105D40001306006485458297E93597C0FF1FE780F9
:105D5000206901458280B7F7070003C70701A547FF
:105D6000AE866316F7009397450191C301A0AA85FB
:105D70000146254517C3FF1F6700E3784111B2862E
:105D80002E86AA852D4506C697C0FF1FE780A077FF
:105D9000B2400145410182809307000463E6C702D7
:105DA0001D71A2CC2A84080886CE32C6EF20316746
:105DB000B2461008A285294597C0FF1FE780A0744E
:105DC000F64066442561828039558280411126C2A1
:105DD000AE848D4522C406C62A84EFC0BFCEB71755
:105DE000004099C803A5C70C418D23A6A70CB2405B
:105DF000224492444101828003A5870C418D23A453
:105E0000A70CF5B78347050003471500A207D98FF4
:105E1000C2076177C187130727206397E70083458F
:105E20002500370504005DB7828097D7FF1F938751
:105E3000675218429C4383D645000345070083C53B
:105E4000C700035646006396A50083D5E700638D1F
:105E5000D502011106CE2386A7002397D700B705E8
:105E6000CF00DC4B9385757D05077D162EC2230080
:105E700001003AC42316C1002317D10099C30A8533
:105E80008297F240056182808280DC4DDC4B81CFBD
:105E9000B7E70400904503A38705914517D5FF1F79
:105EA0000345854B028382806D713C083EC6B7076F
:105EB000E500232291103EC8AA843C08328523269F
:105EC00011103ECA23248110232021112E89EF2096
:105ED00090672A84975501009385C55217450100A4
:105EE0001305C56DEF20115FA2851755010013053D
:105EF0006561EF20315E2945EF201162B705CB00C7
:105F00009385757D6800EF10A043A2856800EF209F
:105F10003059014781467000CA852685EF10C0625E
:105F200015C52A84975501009385C54D1745010075
:105F30001305C568EF20115AA285175501001305F6
:105F4000255DEF2031592945EF20115D8320C110D7
:105F500003248110832441100329011051618280A0
:105F600097D7FF1F9387073F18429C43797122D42C
:105F700006D60348070083C807012A8483D6450054
:105F8000035546006396080183D82701638DD80224
:105F90002388070105072399D7003708CC00DC4B7D
:105FA0001308787D3ACC1307F5FF42CA2308010095
:105FB000231EE100231FD10099C7080832C62EC452
:105FC00082973246A2452285C535B250225445619A
:105FD00082806D713C083EC0B707E5003EC23C08B8
:105FE0003EC423261110232481102322911023174D
:105FF00001002318010023190100231A0100231BAB
:10600000010097D7FF1F83D7A70299E3C167FD1748
:106010002316F10097D7FF1F83D7A70191EB97D7DE
:10602000FF1F938727339C439C43DC4783D707009C
:1060300017D4FF1F1304C4FF584C2317F1008357D4
:106040004400484B2318F10005ED97550100938556
:1060500065421745010013056556EF20B1471755F6
:10606000010013056542EF20F1462945EF20D14A92
:106070008320C11003248110832441105161828048
:1060800097D7FF1F83C737FB89EBB7E70400BC57DF
:1060900082975C4C23AA0700E1BFFD1797D6FF1F2C
:1060A000A38BF6F803560701834704014C470A8582
:1060B000230BF100EF20F03C97D7FF1F9387872930
:1060C0009C430147814688430A866C00EF10C04715
:1060D000AA841DC9975501009385C539174501004C
:1060E0001305C54DEF20113FA68517550100130577
:1060F000653AEF20313E2945EF201142584CB7E771
:106100000400BC57484B69B797D7FF1F83C7B7F246
:10611000F5D7B7E70400BC4F1044854517D5FF1FDE
:10612000034585238297A9B75C4EDC4BA9CBA1C957
:10613000411122C417450100130545482E84975587
:1061400001009385653106C6EF20D138A285175529
:10615000010013056536EF20F1372945EF20D13BCB
:10616000B7E704002244B24003A3870517D5FF1FF9
:106170000345851E13064006914541010283828036
:10618000411122C417D4FF1F130484E81C4C06C617
:1061900089C7DC4399C34C488297584CB7E7040041
:1061A000BC57484B82975C4CB240224423AA07005C
:1061B0004101828017D7FF1F13076712834707002B
:1061C0009306F00B850793F7F70F63E9F60097D670
:1061D000FF1F2386F610034507008280930700F80F
:1061E000FDB7835745006386070E01114AC817D9CA
:1061F000FF1F1309E9E352C4032AC90106CE22CCCA
:1062000003274A0126CA4EC656C2F15721EF13078B
:10621000D00DFD576368C704B7E9040083A70907D9
:106220002A841305860042054181B284AE8A829792
:10623000232AAA000325C9015C499DEF9755010057
:106240009385851F1745010013054537EF209128D9
:10625000175501001305852EEF20D1272945EF2082
:10626000B12BDD57F2406244D2444249B249224A3E
:10627000924A3E850561828093874400B705CF002E
:106280002319F5009385757D3105EF10600B03250B
:10629000C901834564003105EF2090200325C90121
:1062A0002686D6853105EF20D01D7146A2854A8508
:1062B000EF20F116504419CA83A78905854517D5E3
:1062C000FF1F034565098297814769BFEFF07FD0C3
:1062D000E5BFFD573E858280411126C297D4FF1F3E
:1062E000938404D5D84C22C437E404003C54484B72
:1062F00006C68297DC4C0323C4052244B240924474
:1063000023AA070017D5FF1F034505058545410151
:106310000283411126C297D4FF1F9384A4039C409B
:1063200006C622C44AC0C9CBDC43D9C75CC123001E
:10633000B5002A84975501009385450B1745010048
:106340001305C527EF2011192945EF20F11C9C40AA
:1063500023A4070023A2070097D7FF1F938747CBEB
:10636000DC4FDC4B81C72955EFF09FE197D7FF1F2A
:10637000938707CCDC4FDC4B91C3B93F37E904006E
:106380008327C905894517D5FF1F0345E5FC82977B
:106390008327C905914517D5FF1F0345E5FB829764
:1063A0009C4003A347016309030022852244B240B5
:1063B0009244024941010283B2402244924402497C
:1063C000410182800111328506CE22CC26CA2E845C
:1063D000EF207017AA84975501009385650417452F
:1063E00001001305A51DEF20F10E030784000356DD
:1063F000640083554400A686175501001305C50D9A
:10640000EF20510D2945EF20311197D7FF1F83C78A
:1064100087C0639897000145EFF09FD681450A85B4
:10642000CD3DF2406244D244056182806D712324E7
:106430008110232611102322911093F745002E84FA
:10644000638507123C083EC0B707E5003EC23C0822
:106450003EC4231701002318010023190100231A49
:106460000100231B010097D7FF1F83D767BA99E369
:10647000C167FD172316F10097D7FF1F83D767B9B0
:1064800091EB97D7FF1F9387E7EC9C439C43DC4736
:1064900083D7070017D7FF1F130787B72317F1000C
:1064A000544F835747002318F100DC4A95EF975566
:1064B0000100938525FB1745010013052510EF20EA
:1064C000710117550100130525FCEF20B100294586
:1064D000EF209104134544008320C1100324811050
:1064E000832441105161828097D7FF1F83C7B7B2C1
:1064F0002555ADCBFD1717D6FF1FA30EF6B003D65B
:10650000060183470701CC460A85230BF100EF20E3
:10651000407797D7FF1F9387E7E39C4317D7FF1F69
:10652000130707AF97660100938686C888430A86DB
:106530006C00EF106001AA8451DD9755010093852E
:1065400065F21745010013056507EF20A178A685C0
:1065500017550100130505F4EF20C1772945EF20F9
:10656000A17B2685EFF0DFC1B5B793F725009DC36A
:10657000B7E70400BC474146814528088297255566
:10658000EFF01FC028089305F00FEFF09FD81345D8
:10659000240099B793F7150001459DDFEFF07FA325
:1065A0001345140015BF5C4D411106C688C317D7AB
:1065B000FF1F2321F7DAB7E7040083A707081705B1
:1065C00000001305E5E68297B24097D7FF1F2385A9
:1065D000A7D801454101828001119307700F23164E
:1065E000F10006CE97D7FF1F83C7D7D78DE7B7E750
:1065F000040083A7870D17D6FF1F0346A6CE6C00A5
:1066000017D5FF1F035545D682973335A00097D77E
:10661000FF1FA389A7D4F24005618280411193979F
:10662000050122C406C626C2C1872E8463D4070290
:10663000B7E40400FC5417D5FF1F0345A5CA829791
:1066400019C1BC5482972165218DB24022449244E5
:106650004101828093F715008DC7B7E7040083A737
:10666000471A17D6FF1F1306A69E97F5FF1F93859F
:10667000654D17D5FF1F0345E5C6829713451400E6
:10668000E9B793F7250099CFB7E70400BC4F13068D
:106690000064894517D5FF1F0345C5C4829713457C
:1066A000240065B793F785009DC7B7E7040003A8EA
:1066B000871A1307401F97D7FF1F83C7A7C28146BA
:1066C00013064006994517D5FF1F0355E5C90298E3
:1066D000134584009DBF93F745000145BDD7B7E43E
:1066E000040083A7041817D5FF1F0355E5C7829739
:1066F000BC4C13060064914517D5FF1F034585BEAA
:1067000082971345440091B797D7FF1F83D7C7C51A
:106710006396A70217D7FF1F2319B7C417D7FF1F08
:106720002316C7C417D7FF1F2313D7C42E861755A8
:106730000100130565F6BE856F20C159175501008C
:10674000130505F76F20C16D03574500011106CEF3
:1067500022CC97D7FF1F83D727C1175501001305F8
:1067600025F56310F706C167F91717D7FF1F232D0B
:10677000F7BE37E4040097D7FF1F23A907BE7C4C60
:10678000894517D5FF1F0345E5B582977C4C914598
:1067900017D5FF1F034505B5829797D7FF1F83C7FE
:1067A000D7BA95C78547A307F10083274417130677
:1067B000F1008545130550308297175501001305E8
:1067C000A5E4EF20E165F24062440561828097D73D
:1067D000FF1F83C7A7B7175501001305A5E7F5F3FA
:1067E0008547A307F100832744171306F100854569
:1067F00013055030829717550100130525E3D1B7D3
:106800007D15954763E0A71A17570100130787DC2A
:106810000A053A951C41011122CC06CE26CABA9728
:106820002E84828717550100130505E9EF20415F8B
:106830000DA203C725009947631DF7002E85EFF0D1
:10684000BFF083456400175501001305E5E7EF200D
:10685000614897D7FF1F238A07AE1755010013051C
:1068600065E8E9B703C7250095476317F702C167D5
:1068700017D7FF1F035747AFF91703D5A5006307C5
:10688000F702B7E7040083A7C717829717550100DF
:10689000130545E6EF20C158854717D7FF1F23068C
:1068A000F7AA17550100130565E749B797D7FF1FEA
:1068B000239CA7AA83D7E500B7E40400096617D78D
:1068C000FF1F2314F7AA83D705011306069017D5D7
:1068D000FF1F034525A117D7FF1F2319F7A883D74B
:1068E0002501A14517D7FF1F2313F7A8BC4C82979A
:1068F000BC4C13060064914517D5FF1F0345859EC8
:1069000082970356E4008355A40017550100130530
:10691000A5DFEF20213C49B7175501001305C5E05D
:1069200031B783C525009147639AF502854717550E
:1069300001001305E5E0A307F100EF20614EB7E782
:10694000040083A747171306F1008545130550304F
:106950008297F2406244D244056182809947639EE7
:10696000F5002285EFF05FDE8345640017550100D6
:10697000130585D5EF200136E9BF9547639FF500E4
:106980008347140017550100130585DBE39007EAE0
:1069900017550100130585DC51BD1755010013057E
:1069A00065DCC9BF82806D712324811023261110FC
:1069B00023229110328401CD89476306F50283209A
:1069C000C110032481108324411051618280175526
:1069D00001001305E5D9AE84EF208144A285268508
:1069E000EFE0EF9DE9BFB7E70400FC47280082977E
:1069F00017550100130585D8EF2081428347810098
:106A000039C01307000B638EE7001387A7051377C0
:106A1000F70F8D4663E9E602A2852800EFE0AFF6A6
:106A200079BF8547E3FD87F883459100174501004D
:106A30001305C5ECB335B00097D7FF1F2380B7907F
:106A4000EF204129ADBF03479100A207D98F3567D9
:106A50001307D755638DE7066366F7022D671307A3
:106A6000B7556381E70631671307C7556386E704A7
:106A700029671307A7556392E702A2852800EFE074
:106A8000DF9B35BF39679306E7656383D70663E904
:106A9000F6001307E7556388E704A285280089B745
:106AA0003D679306F755638AD7041307F766E396A5
:106AB000E7FEEFE01FB221B70146A2852800EFE014
:106AC0009F8CF5BDA2852800EFE0BF95CDBD89471D
:106AD000E3F787EE9305E4FFC205C1811305A1002A
:106AE000EFC06FA0E9BDA2852800EFE0DF95C1BD32
:106AF000A2852800EFE0BF9FD9B5EFE0DFA7C1B5C1
:106B0000411122C417C4FF1F13044456AA86175606
:106B100001001306A6AD2285C14506C6EF2041310E
:106B20000357440097C7FF1F938747552393E700F8
:106B3000035764002394E700B2402244410182805D
:106B4000011106CE22CC6D3F37E404008327841464
:106B500017C6FF1F13068651D54501458297832727
:106B600084179305F1001305503082978347F10095
:106B7000A1C7A3070100832744171306F100854529
:106B80001305503082978327441717C6FF1F13063B
:106B9000E64ECD451305703082978547A307F10077
:106BA000832744171306F10085451305503082975B
:106BB000F2406244056182808327441717C6FF1F95
:106BC0001306C64BCD4513057030D5B7130101DE52
:106BD000232C812037E4040083270408232E11206E
:106BE000232A912023282121232631211705000063
:106BF000130505A3829717C9FF1F1309A96E9947AB
:106C000085442300A9002318F100975501009385BE
:106C1000E5A693074006174501001305259A23149E
:106C2000F1102304910097C9FF1F93894972EF2047
:106C3000610A83D50900175501001305E59BEF2074
:106C400061092945EF20410D03D50900EFF05FEB05
:106C500083274417300085451305503082978327DA
:106C6000441717C6FF1F13066641CD451305703044
:106C700082978327441717C6FF1F1306263EB54584
:106C80001305603082978327441710088945130540
:106C9000103182978327441730028945130520312C
:106CA000829783274415930500320D4582978327E9
:106CB00044159305003211458297A30191002302E8
:106CC000910023049100232401102308010083274D
:106CD00084163002914513057040829783278416ED
:106CE00013063100854513050040829783278416DB
:106CF000500085451305104082978327841610089D
:106D000085451305204082978327841630008545EA
:106D1000130550408297832704157D55829783275A
:106D200044137D5582977D55EFC08FC38327440C54
:106D30008297EFC0CFA08327841417C6FF1F1306C6
:106D4000E632D5450145829789471306700F814584
:106D500008082302F100EFB04F818D471306700F32
:106D6000814528022308F100EFB02F8091472304CA
:106D7000F11097C7FF1F93876757984383C7470052
:106D80003AC42306F100EFE0DF8A5000854505454F
:106D9000EFC02FC410089305700F0945EFC06FC3F3
:106DA00030029305700F0D45EFC0AFC2300095451E
:106DB0001145EFC00FC2C16717C7FF1F1307C75A9E
:106DC000F9171CC32322070017C5FF1F13054551E0
:106DD000EFC00FBF8327C41D17C5FF1F130505583C
:106DE00082973C4803450900854582978320C1214D
:106DF0000324812183244121032901218329C120E6
:106E00001301012282800111C16726CA06CEAA841D
:106E100022CC17C5FF1F03552555F9176306F50446
:106E200037E40400832784122E862315B10001471E
:106E30008146ED4582977C440356A1002AC6A6856B
:106E400082972C0017C5FF1F03550552EFC00FC4D2
:106E500001CD1755010013056583EF10717C832761
:106E6000C412ED4528008297F2406244D244056185
:106E70008280011106CE22CC2DC9854717C7FF1F7E
:106E8000A303F71E97C7FF1F2380071E37E40400E4
:106E9000832784179305F1001305503082978347A9
:106EA000F100A9CBA3070100832744171306F100C3
:106EB00085451305503082978327441717C6FF1F57
:106EC0001306C619B5451305603082978547A30799
:106ED000F100832744171306F10085451305503050
:106EE0008297F24062440561828097C7FF1FA38C9E
:106EF000071649BF8327441717C6FF1F1306061638
:106F0000B54513056030E9BFC16717C5FF1F0355BD
:106F1000A545F9176307F500B7E7040003A3C717F2
:106F20000283828001118547A307010017C7FF1F55
:106F3000230AF742B7E7040083A7471706CE1306D4
:106F4000F1008545130550308297F240056182803B
:106F5000EFA21FDD2A8408452E89B28909C900C124
:106F6000970500009385C5746105EF008101814498
:106F70007D5AEF10C00963C3A4048144EF10200AB6
:106F800063C6A40497F7FF1F938787BC9C43DC4725
:106F9000B307F94091872302F40063810904832732
:106FA000C900B307F4409587A302F4001C4C89C7BD
:106FB0009C4799C3228582976FA0DFD95C441397C1
:106FC00014008504BA972390470165B71C481397AE
:106FD00014008504BA97239007004DB783278900D2
:106FE0000547B307F4409587A302F40083570400D4
:106FF000638EE7028DC309476384E7040D47E39777
:10700000E7FA97570100938727CA1CCC97570100CE
:10701000938787CA11A897570100938767901CCC64
:10702000975701009387C7905CC849B797470100FD
:107030009387077C1CCC974701009387677CEDB74B
:1070400097570100938707CB1CCC97570100938774
:1070500067CBD9BF85E1EFA25FCE004618448347D6
:10706000940075839D8B6315F700EF00501C48C496
:107070006FA0FFCE8280EFA2BFCA13893500C16422
:1070800042094111AA890144F11413590901054A21
:107090002EC6EF00D077B2456346A40001454101FA
:1070A0006FA05FCB83A7090013171400BA9783D78B
:1070B00007006388B7006394970063742A0105048E
:1070C000C1BF0545E9BFEFA2DFC4AA892E89328B73
:1070D000B6843A8ABE8AEF80204C55C12685EF10CF
:1070E00030368D4763E5A7007D556FA01FC683DB53
:1070F0004400EF00D0772A84EF00B0789307740043
:1071000031443305850263C5A702EF005076EF00D6
:1071100010762A84EF00F07693077400314433052B
:10712000850263CDA702EF0090749307450019A86C
:10713000EF003075330585021307F0179307C0176A
:10714000E357A7FC2D55E3C277FB63000B02D686FD
:107150005286A6854A85EFE0106341BFEF0070724A
:10716000330585029307C5FFF1BF832749001385C7
:10717000C90083D52700EFF01FF071F9B5B7695545
:10718000ADB797F7FF1F2397A79C97F7FF1F93872C
:10719000279C904381470C463307F5004207418303
:1071A0006393B70082805446139847008507C296C0
:1071B0002390E600D5B797F7FF1F938767999C4305
:1071C00003C58700828017F5FF1F0355A5988280AD
:1071D000EFA2BFB6C1671387D7FF6307E5026368F5
:1071E000A700F117630EF50001456FA05FB7138785
:1071F000E7FF630EE500FD171D8D13351500F5B78C
:10720000EF40003D7D15D5BFEF40801AE5BFEF4050
:10721000E018CDBFEFA27FB24111AA8401442EC66F
:10722000EF00F05FB2456346A400014541016FA045
:107230001FB39C48131514003E9583570500E38740
:10724000B7FE0504E9BF03485500814693F7F60FE2
:1072500063E5070181473E85828058459397560034
:10726000BA9703D727006316B70003D70700E304D4
:10727000C7FE8506E1BF8346450001479377F70FB8
:1072800063E4D700814711A81C4513165700050772
:10729000B29703D60700E313B6FE3E858280EFA2C5
:1072A0003FA893170501C18797FAFF1F938A4A8A5F
:1072B0006355F00883A70A00C0479C4703570400A2
:1072C000198D420541816366F500014422856FA056
:1072D0007FA812052A94DDBFDC4713944900014AB8
:1072E0003E94834744006341FA02014A83475400B5
:1072F0006347FA028509C20993D9090183A70A00E5
:107300009847E3EBE9FCD1B71C4413195A00A68552
:107310003E994A85EFF01FF011ED050AD9B75C449C
:1073200013195A00A6853E994A85EFF0BFEE19E180
:10733000050A6DBFE30009FC51BFAA8481497DBFE6
:10734000EFA2BF9F1C452A8481E79307C5001CC597
:107350001C44231204001CC09307F00F63E9B7001C
:1073600093F5F50F2285EF10B0136FA05F9F9394F4
:107370000501C167C18063F7F500A6852285EF107E
:10738000D015E5B7C18193F5F50F2285EF105011A7
:10739000A6852285EF101012C9BF97E7FF1F9387BC
:1073A000277B884382801C4599C797E7FF1F23A14D
:1073B000A77A014582807D55828097E7FF1F9387DA
:1073C0002779984383474500484792073E95828036
:1073D000EFA2BF96617100451C183EC6B707800139
:1073E0003EC81C183ECA8357440002CE02D002CCCD
:1073F000231EF100834784002A8902D22301F1026F
:107400003C083ED402D6EFF05FFB835705002316FD
:10741000F102EF30706B2307A1025C40035564005A
:10742000F18313F717008347F10252055181F99B4D
:10743000D98FA307F102EFE0702639C5AA8403555E
:107440000500EF80401683D704002AD26800231C71
:10745000F10083D72400231DF1001C4803D6470008
:107460008C43EF1010028347B400CA861746010010
:10747000130686318117A305F4006C004810EFE075
:1074800090305D616FA0BF8D2155E5BF1C45B1CF28
:1074900003C5A700894613576500630BD7028D46C5
:1074A000630ED70285466300D702130740063305F3
:1074B000E50203C7B700418B15CB83C7B700BD8B6F
:1074C0003355F54082801375F5031307803EC5B729
:1074D00009671375F50313070771D1BF3727090033
:1074E0001375F5031307077CD9B701458280EFA216
:1074F000DF8403A98500630509048347B900AE84CE
:1075000093F7070E91CF03459900930520030D8152
:107510000505B305B50288446105EFF0B0320DA052
:107520002E85EFF0BFF62A8401CD11238325C900F3
:10753000B307B54063F887002E94B305A440E1FD7E
:107540006FA0FF818545C1BFEFA22FFF2A8403D51D
:107550000500011132C636C43AC22EC002CA02CC9E
:1075600002CEEF80400482452ACA22852ECCEFF05D
:10757000DFE403570500231EE100EF30F054A2467C
:1075800032469247230FA10036874C08B2862285E7
:107590000146EFF05FB305616FA06FFCEFA2EFF95A
:1075A00061711C183EC6B70780013EC81C183ECA50
:1075B0003C0800453ED4AA8402CC02CE02D002D2BE
:1075C00002D6EFF09FDF8357050035592316F102ED
:1075D000EF30904F2307A10209C48357440091E77D
:1075E00021594A855D616FA08FF7035564005205EC
:1075F0005181EFE0B00A2A8965D58347B40093F73B
:10760000070E89C713058401EFF050258357440006
:10761000231EF100834784002301F1025C400355DF
:107620000900D98313F7070883471102231CA1001F
:1076300093F7F707D98FA300F10283572900231D81
:10764000F1005C40F18313F717008347F102F99BC7
:10765000D98FA307F102EF7010752AD251D1834759
:1076600094006800139757008347B400FD8BD98FAF
:10767000A305F4001C4803D647008C43EF1060605C
:10768000A6871747010013072710740005464C1002
:107690002685EFF05FA32A8929D58347B400A68504
:1076A000FD8BA305F400EFF09FE425BFEFA2EFE808
:1076B000832485FE2A8441112685EFF03FDD834730
:1076C00034FF93F7070E9DC32AC62685EFF05FD0DF
:1076D00019C9834734FFB245FD8BA309F4FE81C568
:1076E0002285EFF0301641016FA06FE76DDD832733
:1076F000C4FF2685829765F9834734FF93F7070E09
:1077000081C72285EFF09015032584FEEFF01FE975
:10771000D9BFEFA28FDF9C4141112A8903C707001F
:1077200089472E8493566700638CF6020D46638268
:10773000C6049307F0076302F7022E85EF10A060DE
:10774000AA848149C16B130C490097E7FF1F9387F7
:1077500027409C43984763ECE90241016FA0AFDEEC
:1077600003D745008547E3FAE7FE2E85EF108061D9
:10777000C1BF03D74500E3F2E7FE2E85EF10A05C02
:10778000AA842285EF10805DC204C98C5DBFDC47EE
:107790000355A900139A49003E9A93170501C18722
:1077A000635DF00083570A006395A70263E57403E5
:1077B0008327CA00034D5A001DA0A1672167A98F26
:1077C0001307F7EFE374F7FE63950900EFF05FA08E
:1077D00071FD85099DBF83278A00034D4A00835DA3
:1077E000A90003576900216A138BC7003AC6814A72
:1077F00033CA4D01631E5D0197E7FF1F9387C735AD
:107800009C43E1DBA2866286814526858297D1B7BB
:10781000A1679387F7EF930C4BFF63F04703B245E3
:107820005A85EFF05F8519CD03278B00104719CAE1
:1078300010436380C4023107D5BFEE856685EFF043
:107840007F9D71FD93861A0093FAF60F130B0B02BE
:1078500055B7835644005C43E3EDF6F622853AC6FD
:10786000EF10603DA1679387D7042A8A035D440027
:10787000324763E897008347D90093E707F8A306E8
:10788000F9001C4766852286E2858297C167084415
:10789000FD17337AFA00529508C02312A40115BFD0
:1078A00097E7FF1F9387C72A9843814715C314475B
:1078B000814763FFD500939745004C47BE9519C992
:1078C00003C7550081476375E600DC451606B2978D
:1078D0003E85828003C745008147E37BE6FE1606AE
:1078E0009C45F5B7EFA2CFC3AA892E8A814497EAB7
:1078F000FF1F938AEA2583A70A00984763E4E40000
:107900006FA04FC5DC471394440001493E9413BB5C
:10791000140083474400634BF900014913BB140072
:1079200083475400634FF9008504F1B70844931767
:1079300059005287DA860146A2853E95829905094B
:10794000C9BF4844931759005287DA860546A28575
:107950003E9582990509E9B7EFA22FBE814517F53B
:10796000FFFF1305255F97E7FF1F2395071EEFF025
:107970007FF76FA0CFBE97E7FF1F9387671D9C43DC
:1079800081CFEFA28FBB814517F5FFFF1305855C03
:10799000EFF05FF56FA0AFBC8280EFA26FB837E465
:1079A00004008327841241112315E100AE89328936
:1079B000368A3A8681460147ED45AA8482972AC6CF
:1079C00021C50356A100D285EF1061258327C4137A
:1079D000CE8526858297058915C58327440D2314F6
:1079E000210101462C00268582972A8401C9B7E728
:1079F000040083A7C712ED45280082972285410124
:107A00006FA04FB54944E5B76554CDBF5C41FD1744
:107A10005CC18280EFA26FB2B7E70400FC5F82977F
:107A200095473305F50281450D816FA04FB3EFA255
:107A3000CFB0B7E70400FC5F829795473305F502A6
:107A40000D816FA0CFB1EFA24FAFB7E7040083A7BE
:107A5000870B0355050082976FA06FB0EFA2EFADC3
:107A6000035505003287AE8617B6FF1F03562667FB
:107A700097E5FF1F9385850EEFF03FF26FA02FAEC5
:107A8000EFA2AFABB7E7040083A7C71782976FA039
:107A90000FADEFA28FAAB7E7040083A7871397E57E
:107AA000FF1F9385A50B829701456FA04FABEFA2F7
:107AB000CFA8B7E7040083A7C71F814517B5FF1FED
:107AC0000355E55D82976FA08FA9EFA20FA7B7E7D7
:107AD000040083A7871397E5FF1F938525098297E5
:107AE00001456FA0CFA7EFA24FA5B7E7040083A77A
:107AF000C71F814517B5FF1F0355656082976FA0AB
:107B00000FA6EFA28FA32E85EF600055EF60900DBA
:107B10006FA0EFA4EFA26FA2EF60D0176FA02FA409
:107B20005C49E1175CC95CC583572501A10723198E
:107B3000F50083570501A1072318F5008280F1475E
:107B40003305F50297E7FF1F938747049C433E9553
:107B500082808D476317F60603D74600854763F298
:107B6000E706EFA28F9D368536842E89EF10A01D83
:107B700039C18357440093140501C18063ED970216
:107B80002285EF10401CFD14231294009307A002DD
:107B9000630EF5009307B0026301F50293079002AC
:107BA000631BF5002285EFC0B07E31A00146CA8577
:107BB0002285EF80000F6FA08F9A2285EF00105969
:107BC000DDBF828097E6FF1F938686FC9C420145BD
:107BD00099CF9843D44217E6FF1F232BE6FA63960A
:107BE000D70097E6FF1F23A7E6FA1385C7FE82801A
:107BF000EFA2AF94E9267144330585029145EF70F9
:107C0000606201E565556FA08F9597E7FF1F23AD73
:107C1000A7F67526330585029145EF70A0607DD1EA
:107C200097E7FF1F23A4A7F6592E97E7FF1F239777
:107C3000A7F4712697E7FF1F2393A7F49747010046
:107C40009387C7B917E7FF1F232EF7F297070000A6
:107C5000938747ED17E7FF1F2324F7F2014565B728
:107C6000EFA2AF8DAA8517E5FF1F130525F1EF10D1
:107C700060216FA0CF8EEFA24F8CEFF07FFEEF1050
:107C8000E02197E7FF1F9387A7F09C4381CF1387DD
:107C9000C7FE09CB83D5C7FF17E5FF1F1305C5EF47
:107CA000EFF0403A6FA0AF8BEFA22F89EFF09FF17A
:107CB00019C9834785002A8493F7070499E7035578
:107CC000E500EFF05FFB6FA08F898347C500930449
:107CD000450117E9FF1F1309A9EB85E38327090075
:107CE0005CC997E7FF1F23A597EA83274900E1FFB7
:107CF00097E7FF1F23A097EAF9B7FD172306F500C2
:107D00006105EF60E07E8307840063CB070483474F
:107D1000840093E707F82304F400B7E704009C5FAE
:107D200082974205A94741813375F5028347840054
:107D300093F707FCC98F2304F4008347D4003E95D2
:107D40001C402318A40089CF984319CB8347C40053
:107D50005040814585073305F50242054181029770
:107D6000832709005CC897E7FF1F23A397E28327B7
:107D7000490089E797E7FF1F23AE97E08347C400D8
:107D8000B9D38355040117E5FF1F1305E5E0EFF0B4
:107D9000602B15BFEF927FFA97E7FF1F93870705C8
:107DA0009C4701448583858B81EFAE84B2853A86FA
:107DB000EF1020142A8409C5EF10200B829408CC00
:107DC00022856F90DFF9EF92BFF541112E8932C6FF
:107DD000AA89712C324713060502CA86970500004E
:107DE000938525D617E5FF1F130545D9EFF09FFAB8
:107DF0002A8429CD9304C50065261946AA852685BF
:107E0000EF00306885452685EF00106517450100B5
:107E10001305859A4E95834505002685EF00506829
:107E20005C4831468145A1075CC85CC48357240186
:107E3000E1172319F40083570401E1172318F40014
:107E40001C4C3E85EF907FF2A30425012285410161
:107E50006F905FF0EF927FEE4111AA842EC632C47C
:107E6000EF100003004DB2452246834784000CC04A
:107E700050C093F7F70393E707042304F400231893
:107E800004002685EF00707E83479400A9462317DF
:107E9000A40013D7370005073307D7029D8B85074A
:107EA0002306F400A306E40083C70401D84885072D
:107EB000230FF7FE17E7FF1F130787CD5843232A29
:107EC0000400930744011DEB17E7FF1F2324F7CCA1
:107ED00017E7FF1F232EF7CA17E4FF1F1304C4CBB5
:107EE0002285EFF0A00B1C44858B5D8D09E5814553
:107EF0002285EFF0201541016F907FE61CC317E744
:107F0000FF1F2329F7C8C9BFEF923FE39705000081
:107F1000938565C40145EFF0DFBE01456F903FE4F6
:107F2000EF92BFE1EFF01FBF6F907FE38347C50083
:107F3000A1E7EF929FE02A840355E500EFF05FD2BE
:107F400015C98347840093F7F7FB2304F4001C4012
:107F500091C7DC4381C74C4001458297EFF09FC633
:107F600017E5FF1F130545C3EFF0400F0355E4006D
:107F7000EFF07FD06F90BFDE8280EF921FDC97E73B
:107F8000FF1F9387E7C097050000938525D217E56B
:107F9000FF1F130565C023A0070023A20700EFE021
:107FA000507E6F90DFDB1C4D91CBDC4381CBEF9299
:107FB000DFD88345070082976F907FDA828097E74A
:107FC000FF1F9387A7BF9C4303C50700828097E7E5
:107FD000FF1F9387A7BE9C4303C51700828097E7C6
:107FE000FF1F9387A7BD9C4303C52700828097E7A7
:107FF000FF1F9387A7BC9C4303C54700828097E778
:10800000FF1F9387A7BB9C4303C53700828097E778
:10801000FF1F9387A7BA9C4303C55700828097E749
:10802000FF1F9387A7B99C4303C56700828097E72A
:10803000FF1F9387A7B89C4303C57700828097E70B
:10804000FF1F9387A7B79C4303C58700828097E7EC
:10805000FF1F9387A7B69C4303C59700828097E7CD
:10806000FF1F9387A7B59C4303C5A700828097E7AE
:10807000FF1F9387A7B49C4303C5B70011E11D45BB
:10808000828097E7FF1F938767B39C4303C5C700B0
:10809000828097E7FF1F938767B29C4303C5D70091
:1080A000828097E7FF1F938767B19C4303C5E70072
:1080B000828097E7FF1F938767B09C4303D5070132
:1080C000828097E7FF1F938767AF9C4303C5270113
:1080D000828097E7FF1F938767AE9C4303D54701D4
:1080E000828097E7FF1F938767AD9C4303D56701A5
:1080F000828097E7FF1F938767AC9C4303D5870176
:10810000828097E7FF1F938767AB9C4303C5A70156
:10811000828097E7FF1F938767AA9C4303C5B70137
:10812000828097E7FF1F938767A99C4303C5C70118
:10813000828097E7FF1F938767A89C4303C5D701F9
:10814000828097E7FF1F938767A79C4388578280A9
:1081500097E7FF1F938787A69C4303D5C7028280BA
:1081600097E7FF1F938787A59C4303D5E70219E193
:108170001305800C828097E7FF1F938727A49C43F9
:1081800003C50703828097E7FF1F938727A39C43BC
:10819000C85B828097E7FF1F9387C7A188438280CF
:1081A00097E7FF1F938747A18843828019E17D5598
:1081B0008280F5DE984265DFFDD917E7FF1F1307C0
:1081C000E7C21847AA877155058B6319072203C5B3
:1081D00007001547E37DA7FC03C737001305F0052B
:1081E0007D171377F70FE364E5FC03C35700E30043
:1081F00003FC83C86700E38C08FA03C7770049458E
:1082000079171377F70FE364E5FA03C7A70011485E
:108210001305F7FF1375F50FE36BA8F803CE97006E
:108220000D481305FEFF1375F50FE362A8F803C8A8
:10823000B7006309080065181378F80F1305600D7F
:10824000E36705F703C5C700794879151375F50F7E
:10825000E36FA8F403C8D7000D457D181378F80F15
:10826000E36705F503D80701930E4017511842083C
:1082700013580801E3ED0EF303C8E7007D181378E7
:10828000F80FE36605F303C827017D181378F80F8C
:10829000E36F05F103C88700C54E75181378F80F12
:1082A000E3E70EF103D86701856E938EBEE06D188B
:1082B000420813580801E3EC0EEF03D847016D188C
:1082C000420813580801E3E40EEF03D88701791838
:1082D000420813580801E36C05ED03C8A7017D1897
:1082E0001378F80FE36505ED03C5B7011D487D154B
:1082F0001375F50FE36DA8EA03C5D7017148791529
:108300001375F50FE365A8EA03D5E7011308E00F3D
:108310007D1542054181E36CA8E803C50702494881
:1083200079151375F50FE364A8E8C85301C937C878
:1083300034005915130858BFE36BA8E603A8870259
:1083400037C53400130555BF5918E36205E717E533
:10835000FF1F2323C58603C6050117E5FF1F232F33
:10836000F5840545E375C5E403D82501D049337686
:108370000603E31E06E203C61501E30A06E217E65A
:10838000FF1F2329B68283C5270001466387A50006
:1083900003C61700F1453306B60283C707039305EA
:1083A000C00272971A071307C70516031A97960893
:1083B0004697B387B70241553E97329742074183AC
:1083C000636EE802EF927F973685EF60D06FEFD053
:1083D000B0212A84EF80B01D2A94EFC090252A9402
:1083E000EF7040072A94EFF0BF802A94EF2050638B
:1083F0002A94EF50406622956F907F968280EF928C
:10840000DF934111A307A100EF80801E9305F100C7
:1084100017050000130565B9EFF0CFCC0145410108
:108420006F90FF93EF92FF8E17E4FF1F1304049CDD
:108430000328840079599368180097E4FF1F23AB41
:10844000149B13781800631E0800BA84BE89368B0B
:10845000328A2E89AA8AEFE01FD67D15269509E576
:1084600031594A856F907F8EEFE0FFD47D152695B8
:10847000A167E357F5FE97E7FF1F938727CE984341
:108480003E8C814B11C70145EFC0B03E933B1500B8
:108490004A85DA865686D285EF7070372A8911CDE3
:1084A0001C44F99B17E7FF1F2326F79483270C0032
:1084B000CDDBE3880BFA82976DB7268597E7FF1F20
:1084C00023A80792EFE0FFCB4146CE8517E5FF1FBB
:1084D0001305459BEF00A174EFA070080325040B62
:1084E000EFA0700A0545EFA070100545EFF03FF1D1
:1084F0008DBF97E7FF1F9387678F9C47858BD5C7F5
:10850000EF92BF8317E5FF1F1305059697E7FF1F3F
:1085100023AE078C97E7FF1F23AC078C97E7FF1F5D
:1085200023AA078CEFE09033EF40C002EFE0F00A9F
:10853000EFE0700F97E7FF1F9387C7899C4381C7C0
:108540000545EF60B03397D7FF1F938767729C4351
:1085500089C741657D15EF50A06BEFC0703AEFA061
:10856000F00097E7FF1F9387679D9C4313971701C0
:1085700063540700EFC0A04597E7FF1F23A40790AF
:1085800097E7FF1F23A2079097E7FF1F23A00790FD
:1085900097E7FF1F23AE078EEFF09F984923EFF078
:1085A000AFBBEFC080676F908FFB828097E7FF1FA4
:1085B0009387C78388438280EF922FF8EF60B07E65
:1085C000EF7080006F90AFF9EF928FF52A849304DB
:1085D000140201112E85B289A685214636C63A8934
:1085E000EF0081611DE1B24638082686CE8513056D
:1085F0009404EF40604321462C084A85EF00C15F98
:108600001335150005616F90EFF40145E5BFEF925A
:10861000CFF29305450617D5FF1F1305655AEFE006
:1086200070226F90CFF3EF924FF141112EC6EFF011
:108630000FC0B24588C141016F906FF2EF924FEECB
:10864000AA842E84EF605078AA8985452285892DD9
:1086500083C7E4011389940899E313890403CE8541
:1086600022853D2D2146930519022285192D97D784
:10867000FF1F9387A7778C432285EF00E068214690
:10868000938584022285F52B6F90CFECEF926FE8F3
:108690003971EFC0E04E9305400645EDEF60D06FB5
:1086A000630E051097D7FF1F83C7475313B71700F3
:1086B00097D6FF1F2384E652014489CFC16417D99E
:1086C000FF1F1309A9729309400EFD14EFF03F98A4
:1086D0006348A408EFF0AFB54169B7290900096AFA
:1086E000FD7A2A8B81447D199389F97B130A0A71DB
:1086F000938A8AC7EFF0BF9563D5A4041304400E94
:10870000B387840217D7FF1F1307476E0324070B95
:108710003E948357C4016386270918403307EB4012
:1087200063EAE900834744008507B3874703D69788
:108730006369F706014681450945EFF0CFE8AA8B4A
:1087400029E1EF20105A8547631FF5048965938559
:10875000057117D5FF1F1305A546EFE0B00EA1A8C0
:10876000B30734030327090BBA9703D7C70163087C
:10877000970003C75700A38207002382E700050480
:10878000B1B79305C5002285EFF05FEB5E852286C9
:108790009735010093858503EFF0CFEB5E85EF0001
:1087A000E06F850481BF97D7FF1F938727649C479D
:1087B0008D83858BC1FF21616F902FD9014685453F
:1087C000094502D002D202D402D6EFF0CFDFAA844C
:1087D0007DD1EFC0203A1389C4002A8481454A859F
:1087E000C1210C4041464A85692983294400638898
:1087F00009084E8502D802DA02DC02DEEF00816A47
:108800002ACE141005462C0808184ECCEF406019EB
:108810001375F50F2DE58355840093E525004A85F2
:108820006D2911460C104A85A9290146973501008A
:10883000938545FA2685EFF0EFE12685EF00006687
:108840005C40B5DB014685450D45EFF0CFD7AA84E6
:108850003DD148401389C400EF00C1642AC64A854F
:10886000C5263246636AC5004C404A85192901462F
:1088700081452685EFF00FDE26850D252DBF83551A
:10888000840071BFEF926FCB97D7FF1F9387075676
:108890009C4719CD93E7870017D5FF1F1305453275
:1088A00017D7FF1F2328F754EFE060786F902FCB86
:1088B000DD9B17D7FF1F232FF752EF2090427DF546
:1088C00017D5FF1F1305C52FEFE04079C5B7EF920D
:1088D0004FC44169AA892E8AB28A368BBA8B8144E9
:1088E00017DCFF1F130C8C50930C400E7D19EFF01A
:1088F0000FF663C4A40001442DA03384940383279E
:108900000C0B3E948357C401638027055A87D68693
:108910005286CE8513050403EFF01FCB11C52380CB
:108920000B0022856F906FC28347F40191CF5A8765
:10893000D6865286CE8513059408EFF0FFC809C588
:1089400085472380FB00F1BF850455B78357450059
:10895000638D0716EF92CFBC01112A84ED2619C54D
:108960008547630AF50405616F90CFBEEFC04021D3
:108970007DF9835744004947ED9BE396E7FEC145E7
:1089800022854524AA842285F52E0357440002CE71
:1089900091472A896317F700228539293C082ACC98
:1089A0003ECEEFC0201D5C55DDDF74084A86A685EB
:1089B000054582974DBF03574400D147E3F5E7FAD9
:1089C000032A0400C169014997DAFF1F938A0A420A
:1089D000130B400EFD19EFF08FE76344A90C2285BD
:1089E000032A04008D26A1452A8922851D2CAA84EC
:1089F0002285D92614402A86AA8978082685CA8520
:108A0000EFF0FFECAA8425D103C7F4018947631571
:108A1000F7008347C101A1DB5546D2851385640069
:108A2000EF00E11F0145EF60103801C583D7C40195
:108A3000B1EB97D7FF1F9387673B9C47935519006E
:108A4000858913D73700058B11CB8983858B639775
:108A5000B70001452EC6EFF0FFE2B2454E85EF604C
:108A6000703C0346C1012A84937519002685EF7076
:108A7000703131C92685EF607037268511C00145F8
:108A8000EF60D061EF20F0258547E31EF5EC83C74A
:108A900054001307F00FE388E7EC8507A382F40086
:108AA000D9B5B304690383A70A0BBE9483D7C40165
:108AB000638937015546D28513856400EF00C113E1
:108AC00071D1050909BF5DDC5DBF8280EF924FA5C2
:108AD000EF60902C11CDC164014417D9FF1F130919
:108AE000E9309309400EFD14EFF06FD6634AA400FD
:108AF00017D5FF1F1305C50CEFE060536F908FA5CE
:108B0000330534038327090B3E958357C5016386DC
:108B1000970023120500EF60702D0504F1B797D779
:108B2000FF1F9387A72C9C478D83858B99EBEF9232
:108B3000CFA017D5FF1F1305A508EFE020526F90B7
:108B40000FA28280EF926F9F97050000938545B436
:108B500017D5FF1F1305C506EFE0A0426F902FA0A9
:108B6000EF92AF9D8841B7E70400BC5B0505420565
:108B70004181829709C585472300F50005056F905F
:108B80000F9E83C7F5FF2E858507A38FF5FE828094
:108B900083C7F5FFFD1793F7F70FA38FF5FE99EB4A
:108BA000EF92AF99B7E70400BC571385F5FF8297A2
:108BB0006F90EF9A82801C41035745008D8FBA95C4
:108BC0001CC12312B5003E85828093D78500A20583
:108BD0001441DD8D835745001387E6FF18C18907CF
:108BE0002312F50013D685004111238FB6FEA38F03
:108BF000C6FE4101828018419307F7FF1CC18357CD
:108C0000450085072312F500A30FB7FE8280835726
:108C100045008D8F2312F5001C41BE950CC12E8599
:108C20008280AA8703D7470008410D8FAA95239217
:108C3000E7008CC38280184108453305A740828035
:108C400083574500035765001D8F1C410845338538
:108C5000A7403305A7408280EF922F8E41112EC688
:108C60002A84EFF0FFFDB2456373B50001A083577E
:108C700044000840BE952312B4003E9541016F9018
:108C80000F8EEF928F8B41112E84B28532C6EFF09A
:108C9000BFFC3246A285EFF0907841016F902F8C97
:108CA000EF92AF892E848545EFF01FFB23008500EE
:108CB0006F90EF8AEF926F8841112317B1008945B9
:108CC000EFF09FF98347E1002300F5008347F100AF
:108CD000A300F50041016F908F88EF920F8693D724
:108CE0008500A2054111DD8D2317B1008945EFF004
:108CF000BFF68347E1002300F5008347F100A3009E
:108D0000F50041016F90AF85EF922F831397850196
:108D100093D78501C166938606F0D98F13D7850056
:108D2000758FD98FA2053707FF00F98D4111DD8DB1
:108D30002EC69145EFF05FF26C001146EFF0306EF9
:108D400041016F90CF81EF825FFF1C41854503C4D5
:108D50000700EFF0DFEB22856F906F80EF82FFFD61
:108D60001C414111894503C7070083C7170023072A
:108D7000E100A307F100EFF09FE90355E100410195
:108D80006F80FFFDEF827FFB1C414111894503C7C6
:108D9000070083C717002307E100A307F100EFF0E6
:108DA0001FE78357E100410113D58700A2075D8DBE
:108DB000420541816F80BFFAEF823FF80C414111BB
:108DC0002A8411466800EFF0906591452285EFF006
:108DD0001FE4B247C166938606F01397870113D547
:108DE0008701598D13D78700758F598DA2073707D3
:108DF000FF00F98F5D8D41016F807FF61C45BE95A8
:108E00000CC18280AE87944391E6584101EF0CC1BA
:108E10005CC1828003C7570013671700A382E70075
:108E2000B687D5B70CC3EDB7AA87084119CD18414D
:108E3000D44398C36313D500D8C32A870346570089
:108E40009376160081E6232007008280944381CA2E
:108E50008C4203A847008CC363930601CCC3799A64
:108E600014C3A302C7003687D1BF1C45DC471D8D44
:108E7000B777DBB6938777DB09853305F5024205C3
:108E800041818280F147B385F50248452E95828065
:108E90008347450085072302F5008280EF82FFE9C2
:108EA0002A8419E06F80BFEB83474400E5DFFD179C
:108EB00093F7F70F2302F400F5F71C4403D72700BC
:108EC00005072391E700DC4399C3228582974C482C
:108ED00089CD83475400898B99E71C4422859C47A0
:108EE0009C439C478297232A0400004023200400CF
:108EF0004DBFEF829FE48357250041112EC691E7B5
:108F00000144228541016F809FE503570500814799
:108F1000F146E307F7FEB385D702404585072E9457
:108F20008345440008C4F5F5B247AA8481E7232AA3
:108F3000040009A81C456C0022859C439C43829731
:108F400048C85DDD85472312F400B24723200400A2
:108F5000231804002319F4005C485CC483D7240060
:108F6000FD172391F40071BFEF823FDD97D7FF1FFC
:108F7000938707C78843232605002324050041055E
:108F8000EFE0C00D6F80BFDDEF823FDB17D4FF1F26
:108F9000130404C51C40411189CF9C472300B50030
:108FA0002AC65CC1EFF05FFC1C40DC4399C332452C
:108FB000829741016F80BFDA034745001DEB584D92
:108FC000AA877D550DCBEF825FD71CC3DC4797D6B0
:108FD000FF1F23A7E6C0F156130507012390D70012
:108FE0009705000093858501EFD0B07901456F802A
:108FF0001FD77D5582808280EF823FD40111614668
:1090000081452800EF807FD697D7FF1F938747BD04
:109010009C4328009305F00FDC473EC6EFF0DFF6D7
:1090200005616F80DFD397D7FF1F938767BB9C4392
:10903000D847A1679387C7026312F70A397106DE22
:1090400022DC26DA80004AD84ED652D456D2328557
:10905000B284EFF05FCFAA892685EFF03FD02318C6
:10906000A4FC2685EFF09FCF2319A4FC2685EFF002
:10907000FFCE83D744000A8A231AA4FC858393F782
:10908000F70F230EF4FC8607BD0793F7073F330164
:10909000F1408A8A01498347C4FD6365F902CE85A0
:1090A000130584FC232C54FDEFF01FEE52811301B5
:1090B00004FCF2506254D2544259B259225A925A84
:1090C000216182802685EFF07FC993171900D6971A
:1090D00005092390A7001379F90F75BF828097D7F0
:1090E000FF1F9387E7AF9C43D847A1679387A702E9
:1090F0006310F70A397106DE22DC26DA80004AD8CE
:109100004ED652D456D23285B284EFF0DFC3AA894C
:109110002685EFF0BFC4FD572318A4FC268523192C
:10912000F4FCEFF0BFC383D744000A8A231AA4FCDF
:10913000858393F7F70F230EF4FC8607BD0793F79B
:10914000073F3301F1408A8A01498347C4FD6365C3
:10915000F902CE85130584FC232C54FDEFF0DFE2E9
:109160005281130104FCF2506254D2544259B25954
:10917000225A925A216182802685EFF03FBE9317D2
:109180001900D69705092390A7001379F90F75BF29
:10919000828097D7FF1F9387A7A49C43D847A167D6
:1091A00089076318F708397106DE22DC26DA8000A9
:1091B0004AD84ED652D456D232853289EFF0BFB853
:1091C000AA894A85EFF09FB9835749000A8A231874
:1091D000A4FC858393F7F70F230CF4FC8607BD07E7
:1091E00093F7073F3301F1408A8A8144834784FD26
:1091F00063E5F402CE85130584FC232A54FDEFF0C9
:10920000BFD85281130104FCF2506254D254425927
:10921000B259225A925A216182804A85EFF01FB4D6
:1092200093971400D69785042390A70093F4F40F26
:1092300075BF828097D7FF1F9387879A9C43D84733
:10924000A1679387E7046312F70A397106DE22DC0F
:1092500026DA80004AD84ED652D456D23285B2840D
:10926000EFF07FAEAA892685EFF05FAF2318A4FC4C
:109270002685EFF0BFAE231AA4FC2685EFF01FAEC3
:1092800083D744000A8A2319A4FC858393F7F70F38
:10929000230EF4FC8607BD0793F7073F3301F14027
:1092A0008A8A01498347C4FD6365F902CE851305A7
:1092B00084FC232C54FDEFF03FCD5281130104FCBC
:1092C000F2506254D2544259B259225A925A2161F0
:1092D00082802685EFF09FA893171900D69705097D
:1092E0002390A7001379F90F75BF828097D7FF1FCE
:1092F0009387078F9C43D847A1679387C704631060
:10930000F70A397106DE22DC26DA80004AD84ED60A
:1093100052D456D23285B284EFF0FFA2AA892685B4
:10932000EFF0DFA3FD572318A4FC2685231AF4FCD5
:10933000EFF0DFA283D744000A8A2319A4FC8583B7
:1093400093F7F70F230EF4FC8607BD0793F7073F4B
:109350003301F1408A8A01498347C4FD6365F902FC
:10936000CE85130584FC232C54FDEFF0FFC1528100
:10937000130104FCF2506254D2544259B259225A99
:10938000925A216182802685EFF05F9D9317190024
:10939000D69705092390A7001379F90F75BF82802E
:1093A00097D7FF1F9387C7839C43D847A167DD07E3
:1093B000631BF702EF827F98797132853284EFF078
:1093C0009F982AC62285EFF07F992311A10222855A
:1093D000EFF07F97B2452300A1022808EFF0DFBA33
:1093E00045616F80DF97828097C7FF1F9387477F14
:1093F0009C43D847A16793878704631BF702EF82DA
:10940000DF93797132853284EFF0FF932AC622858B
:10941000EFF0DF942311A1022285EFF0DF92B24535
:109420002300A1022808EFF03FB645616F803F930B
:10943000828097C7FF1F9387A77A9C43D847A1676D
:109440009387A704631CF700EF823F8F0111280068
:109450008145EFF07FB305616F807F90828097C771
:10946000FF1F9387E7779C43D847A16793875702ED
:109470006311F702EF827F8C01113285EFF0BF8C10
:109480002308A10081452800EFF01FB005616F801F
:109490001F8D828097C7FF1F938787749C43D8478F
:1094A000A1679387E702631FF702EF821F8901110B
:1094B00032853284EFF09F8AAA842285EFF01F8ADA
:1094C000854719E52285EFF01F884205B337A000D4
:1094D00028008145231891003ECAEFF0FFAA0561DC
:1094E0006F80FF87828097C7FF1F9387676F9C43BA
:1094F000D8479947631FF704EF823F84797132851B
:109500003284EFF05F842AC62285EFF03F85231076
:10951000A1022285EFF03F832301A1022285EFF013
:109520009F82A301A1022285EFF0FF812302A10205
:109530002285EFF05F812313A1022285EFF0BF8027
:10954000B2452314A1022808EFF01FA445616F80E3
:109550001F81828097C7FF1F938787689C43D847E6
:10956000A1679387C703631FF704EF820FFD79712B
:1095700032853284EFF02FFD2AC62285EFF00FFEF0
:109580002310A1022285EFF06FFD2311A102228595
:10959000EFF06FFB2302A1022285EFF0CFFAA302C6
:1095A000A1022285EFF02FFA2303A1022285EFF01A
:1095B0008FF9B245A303A1022808EFF0FF9C456193
:1095C0006F80EFF98280EF824FF701112A84EFF06C
:1095D0008FF7AA842285EFF06FF82285EFF00FF85D
:1095E000035744008D4763F5E7002285EFF00FF73E
:1095F0002285EFF0AFF62800A685EFF0FF98056111
:109600006F80EFF597C7FF1F9387875D9C43D8470F
:10961000A167FD076319F700EF822FF23285EFF0A3
:109620009FFA6F80CFF3828097C7FF1F9387475BB6
:109630009C43D847A167E5076311F706EF82EFEF78
:10964000797132853284EFF00FF02AC62285EFF06F
:10965000EFF02285EFF08FF02310A1022285EFF0CA
:10966000EFEF520551812311A1022285230201024D
:10967000EFF06FEDA302A1022285EFF0CFEC230300
:10968000A1022285EFF02FECB245A303A102280826
:10969000EFF09F8F45616F808FEC828097C7FF1F2F
:1096A000938707549C43D847A1679387E7036319BF
:1096B000F700EF828FE83285EFF0FFF06F802FEA3E
:1096C000828097C7FF1F9387A7519C43D847A16704
:1096D000938747046314F702EF822FE6797132858E
:1096E0003284EFF04FE62AC62285EFF02FE7B2452D
:1096F0002808EFF07F8945616F806FE6828097C709
:10970000FF1F9387E74D9C43D847A1679387870244
:109710006316F702EF826FE2797132853284EFF0DF
:109720008FE22AC62285EFF00FE2B2452300A102A4
:109730002808EFF07F8545616F806FE28280EF82BD
:10974000CFDF0111EFF02FE0AA852800EFF0DF83D3
:1097500005616F80CFE097C7FF1F938767489C43E1
:10976000D847A167D1076319F700EF820FDD328573
:10977000EFF0FFFC6F80AFDE828097C7FF1F9387FB
:1097800027469C43D847A167C5076319F700EF82B6
:10979000CFDA3285EFF0BFFA6F806FDC828097C737
:1097A000FF1F9387E7439C43D847A167B907631915
:1097B000F700EF828FD83285EFF07FF86F802FDAD5
:1097C000828097C7FF1F9387A7419C43D847A16713
:1097D000AD076319F700EF824FD63285EFF03FF601
:1097E0006F80EFD7828097C7FF1F9387673F9C43A7
:1097F000D84789476310F702EF822FD401113285D1
:1098000032C8EFF04FD4AA852800EFF0EFF70561DA
:109810006F80EFD4828097C7FF1F9387673C9C437C
:10982000D847A1678D076317F702EF820FD10111A7
:1098300032853284EFF02FD113066100AA844C00E8
:109840002285EF20D00C2800A685EFF0EFF305610C
:109850006F80EFD0828097C7FF1F9387A7389C4304
:1098600081CBDC4391C7EF824FCD82976F802FCFA2
:109870008280EF828FCC79713C08AE843ED2A165A4
:10988000B7070A002A843ED448103C08DD053ED6BE
:1098900036C432C63AC2EFD0BFAA12474810BA85C2
:1098A000EFF00FC032464810B285EFF0AFC0A246CD
:1098B0004810B685EFF0CFBE501001478146A6850F
:1098C0002285EFD07FC845616F806FC9EF82EFC6F8
:1098D00001117C000329C501AE843ECAA165B7070A
:1098E00007002A843ECC48087C00C5053ECEEFD058
:1098F0003FA58345D9004808EFF08FBA50080147CB
:109900008146A6852285EFD03FC405616F802FC5B3
:10991000EF82AFC283C7950093F7F707A384F500E2
:10992000EFF0DFFA6F80AFC3EF822FC179713C088F
:10993000AE843ED2A165B70709002A843ED4481000
:109940003C08938545043ED632C636C4EFD05F9FAF
:10995000A2464810B685EFF0AFB432464810B28543
:10996000EFF04FB5501001478146A6852285EFD014
:10997000BFBD45616F80AFBEEF822FBC83C795002E
:1099800041112A8493F7F707A384F50032852EC688
:10999000EFF0CFBC85672AC4637CF500EF50B04080
:1099A0002246B24509E9114781462285EFF07FEC56
:1099B00041016F80CFBA01478346F501FDB7EF82C1
:1099C0002FB601113C003ECAB7070A003ECC3C004E
:1099D0003ECE83C79500AA89328593F7F707A38403
:1099E000F5002E84EFF08FB785676371F504A165EC
:1099F000AA84938585044808EFD09F942685EF506C
:109A0000903A2A891DE591454808EFF06FA9A6858F
:109A10004808EFF02FAACA854808EFF06FA8014761
:109A200081465008A2854E85EFD01FB205616F8038
:109A30006FB281454808EFF0AFA603490902C1BFE4
:109A4000EF820FAE79711C103ECAB7070F003ECCF3
:109A5000404D1C10AA84AE894808994532C6368903
:109A60003ECEEFD0FF8D32464808B285EFF04FA3CF
:109A700063040902A5454808EFF00F9E2546CA85F4
:109A8000EFF0E019500801478146CE852685EFD0DA
:109A9000BFAB45616F800FAC8355C4024808EFF03F
:109AA0006FA10355E402814515C185478545630FC4
:109AB000F500C167FD179305F00F6309F5007D15EB
:109AC000EF5020749305150093F5F50F4808EFF05B
:109AD0002F9D834504034808EFF08F9C83451403B2
:109AE0004808EFF0EF9B835524034808EFF08F9C64
:109AF000835544034808EFF0EF9B69B7EF82EFA36B
:109B000083C795008146014693F7F707A384F500C4
:109B1000EFF01FF36F80AFA4EF822FA279713E8424
:109B20001C103ECA2E89B7070F00A1653ECCFD056B
:109B30001C10AA84480842C03AC23ECE36C432C67F
:109B4000EFD01F8032464808B285EFF06F95A246ED
:109B50004808B685EFF00F9612474808BA85EFF02F
:109B60006F9502486304080291454808EFF0CF8ED4
:109B70001146A285EFF0A00A500801478146CA8528
:109B80002685EFD07F9C45616F806F9D8945480891
:109B9000EFF08F8C834704002300F5008347140007
:109BA000A300F500D1BFEF82AF9783C795000111E5
:109BB0002A8A93F7F707A384F5003285AE8432C66C
:109BC000EFF0CF9932462A893285EFF0CF9785673B
:109BD000637FF900AA894A85EF50F01C2A8419E9AD
:109BE000114781464A86A6855285EFF09FC80561D8
:109BF0006F804F969387E9FF93F7F70F0547E36868
:109C0000F7FE8347F50195E78947E382F9FE83462E
:109C1000F401528501474A86A685EFF09FC5A167EA
:109C2000D90748083ECC230A010002CEEFF0BFC29C
:109C30007DBF639CE7008947639CF9009307102070
:109C4000231FF500EF50901AD9B70947E391E7FCBD
:109C50008D47E39EF9FA2285EF50D03B97C7FF1F4F
:109C6000938747179C4399E797C7FF1F9387470040
:109C70009C4389C703D50400EF60300C231F040008
:109C80002285C9B7EF826F8B01113C003ECAB7072E
:109C90000B003ECC3C003ECE83C795002A8932851E
:109CA00093F7F707A384F500AE84EFF02F8B93179B
:109CB0000501C187635EF004A1652A849385E502EE
:109CC0004808EFD0EFE7A2854808EFE0BFFE97C74E
:109CD000FF1F9387E7F99C439DEF01449375F40FB1
:109CE0004808EFE0FFFB9355844093F5F50F4808D3
:109CF000EFE01FFB9355044193F5F50F4808EFE0A3
:109D00003FFA014781465008A6854A85EFD0DF8398
:109D100005616F80CF84416585460546A2857D1526
:109D2000EF3070675DD95105EFD04027130440062E
:109D30003344850265B7EF824F800111B7070600F3
:109D40003EC683C7950021642A8993F7F707A38449
:109D5000F500AE8428009305A4040AC40AC8EFD015
:109D60002FDE300001478146A6854A85EFD0CFFD22
:109D7000EFE02FF813049404480822CC230A0100D2
:109D800002CEEFF05FAD05616F707FFDEF725FF99E
:109D9000C1642A89014497C9FF1F93892905130AC1
:109DA0008002FD14EFE0AFAB6345A40001456F7086
:109DB0007FFAB307440303A7C90ABA9703D707007A
:109DC0006306970083D72700638427010504D9BF62
:109DD0000545F1BFEF72DFF42A8A2E8999C123A0CD
:109DE00005008149814497CAFF1F938AEADF614BCE
:109DF000EFE02FAD63C5A4004E856F70BFF53384CF
:109E0000640383A70A003E948357040099E7630420
:109E10000900232089008504E1BF4146D28513054E
:109E20004400EFE0705D65F9A289F5B7EF725FEF6E
:109E300039717C083ED4B7070A003ED67C083ED86C
:109E400083C795002A8A328593F7F707A384F50024
:109E50002E8932C6EFE09FF085676373F5063246C0
:109E6000AA843285EFE03FEE8547AA8963EAA7041A
:109E7000A165938585042810EFD08FCC2685EF50FF
:109E800080722A8429E191452810EFE07FE1A685C0
:109E90002810EFE03FE2CE852810EFE07FE0014799
:109EA00081463010CA855285EFD00FEAA1679387AB
:109EB000770448183EDC230A010202DEEFF0BF9966
:109EC00021616F703FE981452810EFE07FDDA685B5
:109ED0002810EFE03FDE97C7FF1F9387E7279C43DB
:109EE00091C7228563870900EFB0600C83450402A7
:109EF00065B7EFB0200BDDBFEF729FE283C795001F
:109F00004111AA8993F7F707A384F5003285AE843F
:109F1000328AEFE0BFE48567637BF5022A89EF5060
:109F200080682A84914621C18347F50105476383F0
:109F3000E70291C70D47636EF702AD462DA093056A
:109F4000050303250A004146EFE0104B1DE14101E6
:109F50006F705FE09305950803250A004146EFE026
:109F6000B049814679F94A86A6854E85EFF0DF9B98
:109F7000F9BF83250A0013059408EF60600119C139
:109F8000C146D5B797C7FF1F9387C7E49C4399E79E
:109F900097C7FF1F9387C7CD9C4389C72285EF6072
:109FA000A05479FD8547A30FF4002285EF80B05DB2
:109FB0002285EF50A0634E8581464A86A685EFF044
:109FC000BF96A1679387570448003EC4230201004F
:109FD00002C6EFF05F88A5BFEF72BFD383C79500BD
:109FE0004111AA8993F7F707A384F50032852E89DA
:109FF000B28AEFE0BFD685676370F50CAA84EF5094
:10A00000805A2A841DE9416B014A97CBFF1F938B2D
:10A01000EBDD130C400E7D1B19A833048A0383A7C4
:10A020000B0B3E948357C401638D6703050AEFE071
:10A030000F82E344AAFE954639A88357C50163926F
:10A0400097029305050303A50A004146EFE0D03AC5
:10A05000994611E181462686CA854E85EFF0DF8C50
:10A06000A1A883A50A0013050403EF507072C1462E
:10A070007DF12285231E9400EF80F0502285EF5061
:10A08000E05697C7FF1F9387270D9C438DCB230076
:10A0900004022285EFA090614E8581462686CA85FE
:10A0A000EFF09F88A1679387070448003EC423020E
:10A0B000010002C6EFF02FFA41016F701FC98947F6
:10A0C0002300F402D1BF397106DE22DC4AD88000B9
:10A0D00052D456D25AD026DA4ED65ECE2E8A328945
:10A0E0002A8BEFD0DFF30605710541998A8A330187
:10A0F000A140232224FC231404FCEFD05FF2834709
:10A100009A000605350593F7F7072315A4FCA30469
:10A11000FA004A85232624FCEFE05FC4931705016B
:10A12000C1876340F0025681130104FCF25062546F
:10A13000D2544259B259225A925A025BF24B2161CF
:10A140008280AA844A85EFE07FC1AA894A85EFE030
:10A15000FFC0A1659385C5022A89130544FCEFD091
:10A160002F9E2685EFD0AF93854501C94A86CE85BF
:10A17000EFD06F8DAA8B15ED8945130544FCEFE0F8
:10A180003FB2A685130544FCEFE0DFB2CE85130590
:10A1900044FCEFE03FB2CA85130544FCEFE09FB1F9
:10A1A00001478146130644FCD2855A85EFD0CFB9CA
:10A1B0009DBF8145130544FCEFE09FAEA6851305C6
:10A1C00044FCEFE03FAFCE85130544FCEFE09FAECB
:10A1D000CA85130544FCEFE0FFAD8144EFD03FE4B6
:10A1E000E3D0A4FC83A70B0113971400BA9783D57F
:10A1F000070089C5130544FCEFE0DFAB8504F9BF18
:10A20000797106D622D44AD000184ECE52CC56CA06
:10A2100026D25AC8AE893289AA8AEFD05FE00605F5
:10A22000690541990A8A3301A140232A24FC231C91
:10A2300004FCEFD0DFDE83C7990006052D0593F7F8
:10A24000F707231DA4FCA384F9004A85232E24FCD0
:10A25000EFE0DFB093170501C187634FF000528133
:10A26000130104FDB250225492540259F249624A39
:10A27000D24A424B45618280AA844A85EFE01FAEF4
:10A28000A1659385A5022A89130544FDEFD04F8B64
:10A290002685EFD0CF80854519C5CA85EFC0BFFDA3
:10A2A0002A8B0DE98945130544FDEFE07F9FA685C4
:10A2B000130544FDEFE01FA0CA85130544FDEFE040
:10A2C0007F9F01478146130644FDCE855685EFD01A
:10A2D000AFA771B78145130544FDEFE07F9CA685CC
:10A2E000130544FDEFE01F9DCA85130544FDEFE013
:10A2F0007F9C8144EFD0BFD2E3D5A4FC83270B0120
:10A3000013971400BA9783D5070089C5130544FD38
:10A31000EFE05F9A8504F9BFEF723FA283474500E3
:10A32000404DD5E7FD574DC0834694000947636D06
:10A33000D7080346B400854663E8C6088306E400F0
:10A3400063C406085C45F9562390D70097C7FF1FE2
:10A3500083C7C78999E3A304E40097C7FF1F9387C6
:10A3600027919C4381E78947A306F40097C7FF1F05
:10A37000938787DE9C4381E789472306F40097058E
:10A38000000093854505AA8413050401EFC0703FC2
:10A39000FD57231AF40281471CDC014897C7FF1FB1
:10A3A00023A2878497C7FF1F93870784232E040364
:10A3B00004C08043EFD0FFD061463306C50281451B
:10A3C0002285EF709F9A81473E856F705F99FD5798
:10A3D000E5BFEF729F962A8403554502EF50A01CFB
:10A3E00009E5231E04006F709F978357E401E5DFA2
:10A3F000930504FF1715010013058577EFB010636F
:10A40000DDB7EF729F932E89A16541119385E50316
:10A410002A8436C432C6BE843AC2EFC07FF21247E5
:10A420002285BA85EFE0DF8732462285B285EFE0EC
:10A430007F88A2462285B685EFE0DF87630D09009D
:10A4400091452285EFE05F811146A685EFE0207DF2
:10A4500041016F70DF9089452285EFE0EFFF83C7F0
:10A4600004002300F50083C71400A300F500CDB756
:10A47000EF72BF8C83C79500444D054793F7F707EC
:10A48000A384F5001C42411183C70700636DF704E4
:10A490002E842A8985CC03C7D4006309F70217B735
:10A4A000FF1F1307E77C184301CFA386F400EF805A
:10A4B000902B83C7D40089E741657D15EF30407547
:10A4C00083D72403918B99C3EFB0B0624A85A285EC
:10A4D000EFF0CFBFA167C10748003EC423020100CF
:10A4E00002C6EFF04FB741016F707F87EF72FF84B4
:10A4F00003D745008D47AA8441112E8432892E85C9
:10A5000063EDE700EFE09F85AA852300090026851B
:10A51000EFC07FD641016F709F84EFE03F842AC671
:10A520002285EFE0BF83B24585472A862300F900E4
:10A530002685EFC05FD1F9BF397106DE22DC26DA4D
:10A5400080004ED652D456D24AD85AD05ECEAE896A
:10A55000B284AA8AEFD0BFAB060513052502419944
:10A560000A8A3301A140232224FC231404FCEFD0E7
:10A570001FAA83C7990006054D0593F7F707231512
:10A58000A4FCA384F9002685232624FCEFE00FFD1C
:10A5900093170501C1876340F0025281130104FC47
:10A5A000F2506254D2544259B259225A925A025B22
:10A5B000F24B21618280AA8B03AB0400EFC03FCE37
:10A5C00035E983D7440001498544F11793B7170053
:10A5D000A301F4FC834734FCA165BDC79385E50462
:10A5E000130544FCEFC0DFD5A685130544FCEFE05E
:10A5F0002FEBDE85130544FCEFE0CFEB834734FC03
:10A60000114691E30946DA85130544FCEFE06FE754
:10A61000814463080900416B7D1BEFD05F9F63C8D5
:10A62000A40201478146130644FCCE855685EFC03F
:10A63000BFF1A5B7A685130634FCEFF03FEB9334CA
:10A6400015002A89860479B79385C50451BF8327ED
:10A65000C90013971400BA9783D507006386650174
:10A66000130544FCEFE00FE5850445BFEF726FEA88
:10A6700079711C103EC4B7070F003EC61C103EC8BF
:10A6800083C79500AA8A328593F7F707A384F5005C
:10A69000AE893284EFE08FEC93170501C1876350D8
:10A6A000F0062A8A2285EFE06FEB2A895285032B78
:10A6B0000400EFC0DFBE39E5835744008144054400
:10A6C000F11793B71700A303F10083457100DA87F0
:10A6D0002287CA8652862800EFF0BFD20147814602
:10A6E0003000CE855685EFC03FE6A1679387D7033C
:10A6F00048083ECC230A810026CEEFF0CF95456175
:10A700006F70AFE4A28513067100EFF03FDEAA84FC
:10A71000094445DD3544E30A55FB4A85EFF00FE770
:10A720000D4445D50144EFD09F8E634BA400C16B0F
:10A730000144FD1BEFD0BF8D634EA400154471B7DB
:10A74000DC4413171400BA9783D7070063812703EB
:10A750000504D1BFD84493171400BA9703D7070054
:10A7600063197701239027012685EF80C0540144A7
:10A77000A9BF0504C1B7EF72AFDA83C795004111D5
:10A780002A8A93F7F707A384F50032852E8932844D
:10A79000EFE0CFDC93170501C187635BF004AA8962
:10A7A0002285EFE0AFDB2311A1004E85832A040050
:10A7B000EFC0FFAE29E18357440085440144F117FF
:10A7C00093B71700A300F1000348110003572100BD
:10A7D000D6875285CE862686CA85EFF0EFB3A1676D
:10A7E000F10748003EC42302910022C6EFF0AF8675
:10A7F00041016F702FD6A28513061100EFF01FCF15
:10A800002A84894471D18357210011678544BA97FE
:10A81000C2071167C1831307F7EFE367F7FA97B72A
:10A82000FF1F9387275B9C4391C785451305210034
:10A83000EF40300E8355210022858144EFC09F9D5B
:10A8400041D5231005002285EF808048B5BFEF7207
:10A850004FCC83C7950041112A8B93F7F707A38448
:10A86000F50032852E8A3284EFE04FCF9317050131
:10A87000C1876359F004AA8A2285EFE02FCE2A8986
:10A880005685832B0400EFC09FA121E1835744002C
:10A8900081440544F11793B71700A301F100034861
:10A8A0003100DE875A854A87D6862286D285EFF028
:10A8B000AFA6A167ED0748003EC42302810026C66B
:10A8C000EFE07FF941016F704FC8A2851306310098
:10A8D000EFF0DFC1AA84094479D19167CA97C20712
:10A8E0001167C1831307F7EF0544E36AF7FACA85D6
:10A8F000EFC05F92014445F58149EFD04FF263DB31
:10A90000A900984893971900BA9703D7070015E74D
:10A9100023902701EFD0AFF01544E382A9F82685F4
:10A92000EF80003B97B7FF1F9387C74A9C430144C2
:10A93000BDD74A85EF4040769DB785097DBFEF7250
:10A940002FBE79713E847C083EC82E8AB70714005A
:10A95000A1653ECAE5057C08AA89080836C4428973
:10A9600032C6BA8AC6843ECCEFC09F9DCA8508080D
:10A97000EFE00FB332460808B285EFE0AFB3A2466E
:10A98000630E09029D450808EFE00FAD1D468145A5
:10A99000EF70AFBD63870A0691450808EFE0CFABC3
:10A9A0001146A685EFE0A027100801478146D28511
:10A9B0004E85EFC07FB945616F70CFB9B685080885
:10A9C000EFE04FAF1C400808D8439355C701858975
:10A9D00012075183B205D98DEFE0CFAD1C400808B6
:10A9E00083C58700EFE0CFAB1C40080883C5A700F4
:10A9F000EFE00FAB1C40080883C59700EFE04FAABB
:10AA000051BF89450808EFE02FA583C70400230044
:10AA1000F50083C71400A300F50079B7EF724FB0BB
:10AA200083C795004111AA8993F7F707A384F5001E
:10AA30003285AE843284EFE06FB293170501C1878F
:10AA40006357F0042A89032A0400EFC05F8519E9DF
:10AA5000835744000548F11793B71700A307F10087
:10AA6000814621A81306F100A285EFF03FA81DC181
:10AA70001C459DC383D6470001480347F100930757
:10AA80008500D2884A86A6854E85EFF05FEB4101AE
:10AA90006F704FAC0948E9B71D48D9B7EF724FA89E
:10AAA00065715C083EC4B7077B013EC65C083EC8C2
:10AAB00083C795002A8A328593F7F707A384F500A8
:10AAC000AE89EFE04FA88357E100C5C38945280050
:10AAD000EFC01F8781452800EFE08F9CEFC0FF8B00
:10AAE00097B7FF1F938747679C4317B4FF1F034423
:10AAF000E40FAA843334800099C31364240097B709
:10AB0000FF1F9387E7169C4399C31364440097B7CC
:10AB1000FF1F9387272C9C4399C31364840083D51C
:10AB2000040028000149EFE0EF9883D524002800B5
:10AB3000EFE04F9883D544002800EFE0AF97EFD0C7
:10AB40000FC993150501C1812800EFE0AF96A285DA
:10AB50002800EFE02F969C44636CF9000147814682
:10AB60003000CE855285EFC03F9E59616F708F9E39
:10AB7000DC441314490028003E94EFE06F8C8347B7
:10AB800044000347540089070607BA978607E36E17
:10AB9000F5FC835524002800814AEFE0AF918345FE
:10ABA00044002800EFE0CF8F834554002800EFE0F9
:10ABB0002F8F8347440063C9FA00814A83475400BA
:10ABC00063CFFA00050941BF1C4413975A002800BF
:10ABD000BA9783D50700850AEFE0CF8DD9BF032B45
:10ABE000C40093975A0028003E9B83552B00850A8A
:10ABF000EFE04F8C83550B002800EFE0AF8B7DBF5B
:10AC0000EF72AF935C4993E717005CC9EF80203384
:10AC10006F70EF94EF726F922E848145EFF08F9BEF
:10AC200005C183570500FD172310F50009C483579C
:10AC300025002310F400EFF0BFFC01456F702F9248
:10AC400031456DDC23100400D5BFEF726F8D83C7D3
:10AC5000950041112A8A93F7F707A384F5003285FE
:10AC60002E893284EFE08F8F93170501C187635ED1
:10AC7000F004AA89C1452285EFD0BFFA2A8B4E8500
:10AC8000832A0400EFC0AFE121E58357440023117C
:10AC900001000544F11793B71700A300F1008144A8
:10ACA0000348110003572100D6875285CE8622869D
:10ACB000CA85EFE07FE6A1679387170248003EC48C
:10ACC0002302810026C6EFE01FB941016F708F8813
:10ACD00013061100A285EFF07F81AA8409E52311F4
:10ACE0000100094475BF930521005A85EFF09FF2DA
:10ACF000835721002A84CDD797B7FF1F9387870DED
:10AD00009C4391C7854513052100EF408040835542
:10AD1000210026853144EFC0EFCF59D12310050023
:10AD20002685EF70F07A0144A5BFEF720F814111C3
:10AD30002E896C00AA8402C6EFF0CF8909CD035793
:10AD4000050005072310E500EFF09FEB81473E85E6
:10AD500041016F70CF803247954775DBCA852685E4
:10AD6000EF20D008C147E34405FE32448547414601
:10AD70002310F40083570900A6851305440023110E
:10AD8000F400EFD0D0692285C1B7EF627FF983C7A5
:10AD900095004111AA8A93F7F707A384F50032853D
:10ADA000AE893284EFD09FFB93170501C187635EA4
:10ADB000F0042A8AC1452285EFD0BFE6AA845285D5
:10ADC000032B0400EFC0AFCD21E5835744002311CE
:10ADD00001008544F11793B71700A300F100014467
:10ADE0000348110003572100DA875685D28626864C
:10ADF000CE85EFE07FD2A1679387070248003EC46B
:10AE00002302910022C6EFE01FA541016F609FF46D
:10AE1000A28513061100EFF06FED2A8409E52311D6
:10AE20000100894475BF268593052100EFF0FFEFEF
:10AE3000AA845DF5835521002285EFC0AFBD4DF199
:10AE40000149EFD0CF9D635DA90018489317190001
:10AE5000BA9703D707001DE7035721002390E700A7
:10AE6000EFD0EF9B6302250397B7FF1F938787F609
:10AE70009C4389C703552100EF4000222285EF70D3
:10AE80003065B9BF050975BF954499BF05C19307E2
:10AE9000F00F630FF500C547630CF5009307F5FF4E
:10AEA00005453315F50042054181828001458280C8
:10AEB00041657D158280B9E1EF623FE803450603F5
:10AEC0003284EFF0BFFC9305803EB305B502C205A6
:10AED000C18191C90357E402854763F6E700130572
:10AEE0000401EFC020168357E40241677D17638594
:10AEF000E700FD172317F4026F607FE68280EF62A0
:10AF00005FE1004283C79500444D0349140093F765
:10AF1000F707A384F500834704002209116733690A
:10AF2000F900A167B347F90041112A8BAE8A63EC9F
:10AF3000E70C834724001307C00EB91793F7F70FE8
:10AF40006371F70E03473400C14763ECE70C834796
:10AF500044001307E00793C707086373F70A8349A0
:10AF6000840083477400A209B3E9F900856763F997
:10AF7000F908034A6400834754004E85220A336A65
:10AF8000FA00EF40406245C123962403834B34000E
:10AF9000137AFA00239A3403238874032399440311
:10AFA00093890401631A090023A60402239804026A
:10AFB0004E85EFC0A00A1DA0034924004A85EFF08A
:10AFC000FFEC2397A402834744004E85A388F40234
:10AFD000E3810BFEE30F09FCEFC06005EF70907991
:10AFE00081460146D6855A85EFE09FA5A1679387E4
:10AFF00097033EC423020100480002C6EFE0BF856C
:10B0000041016F609FD48544A2862686D6855A85E5
:10B01000EFE01FA3A167938797033EC4230291002B
:10B02000E1BFBD44D5B79144C5B7EF627FCF0111F1
:10B030001C08404D3EC2B7070F003EC41C083EC668
:10B040002A89AE89EFC01F9D585C1C5C634CB70A0F
:10B050006394E50063E8A70A3385A740B3B7A70068
:10B06000B305B7401306803E81469D8DEFD0407BEF
:10B0700093140501C180A1659385C5034800EFC005
:10B080002FAC81454800EFD0BFC183550404480070
:10B09000EFD05FC2835524044800EFD0BFC1814583
:10B0A00099C8C167FD179305F00F6386F4002685E4
:10B0B000EF402015AA854800EFD09FBE03554404F9
:10B0C000814511C9C167FD179305F00F6305F500B0
:10B0D000EF402013AA854800EFD09FBC834564044D
:10B0E0004800EFD0FFBB834574044800EFD05FBB3E
:10B0F000500001478146CE854A85EFC0EFC4056107
:10B100006F605FC5814485BFEF623FC383C7950011
:10B1100093F7F707A384F500EFF03FF16F603FC4AA
:10B12000EF621FC083C795004111404D93F7F707A9
:10B13000A384F5002A8A3285B284AE89EFD01FC27B
:10B140002A8B2685EFD09FC12A892685EFD0BFBFE5
:10B1500093170B0163CA0702E177CA97C207C1833D
:10B16000116763E3E70293070910C207C18313075E
:10B17000B00F637BF70093170901C187AA8A634860
:10B18000F000C54763FA570141016F60BFBCEFC0D3
:10B190008F83E31B25FFF5B763060B0263040902E7
:10B1A000814463870A02B7077F00231064052311D7
:10B1B00024057CC05685EFF07FCD9304803EB30418
:10B1C000950239A0B7077F00232004047CC0814486
:10B1D00003552404EFB0101095CCEFC0BF83269523
:10B1E00093D7F44133379500AE97BA9708DC5CDC0F
:10B1F000CE855285EFF07FE399E023220404A16716
:10B200009387B70348003EC42302010002C6EFE063
:10B210008FE49DBF814701481CDC232E0403C9BF76
:10B22000EF62BFB1EFC0FFE9E1473305F502914599
:10B23000EF30507FE55711C597B7FF1F23A6A79A98
:10B2400081473E856F60BFB1854717B7FF1F230F4A
:10B25000F7988280EF627FAE97B7FF1F938787983A
:10B2600080432DC083570404639EA704835724049E
:10B27000639AB7043689B284EFC0CFF95C5C63C3CC
:10B28000B7046395B7001C5C63EEA70283476404B0
:10B2900063F3F400A6872303F4048347740463F381
:10B2A0009700A687A303F4048357440441677D17DE
:10B2B0006385E70085072312F4043C4481C7CA85EF
:10B2C000268582976F60BFA997B7FF1F93878791E5
:10B2D0009C43014599C303C587008280EF62FFA5A7
:10B2E0000111B70707003EC683C79500584D0AC431
:10B2F00093F7F7070AC8A384F5002A89AE8401CB27
:10B300001C4283C707002304F700EF70D045216477
:10B31000930554022800EFC0AF82EFF0FFFAAA8530
:10B320002800EFD0FF97300001478146A6854A8567
:10B33000EFC08FA113044402480822CC230A010065
:10B3400002CEEFE04FD105616F607FA1EF62FF9EFB
:10B3500001117C003ECAB70707003ECC7C003ECE00
:10B3600083C795002E84AA8493F7F707A384F5007A
:10B37000A165938555024808EFB09FFCEFF0DFF41C
:10B38000AA854808EFD0DF91500801478146A28581
:10B390002685EFC06F9B05616F607F9C97B7FF1F8D
:10B3A000938747849C43094599C303C597008280CE
:10B3B00097B7FF1F938707839C43094599C303C52C
:10B3C000D700828097B7FF1F9387C7819C430145B1
:10B3D00099C303C5A7008280EF629F940111B7074C
:10B3E00008003EC683C79500404D0AC493F7F7078F
:10B3F0000AC8A384F5002A89AE8429C0144285476F
:10B4000003C7060063EEE7068347940009468149B7
:10B41000638EC700B307F740A304E400B339F0001C
:10B4200083C716002305F400EF70F033035724039D
:10B43000058B09C763840900EFA0B06B21649305F5
:10B4400084022800EFB0DFEFEFF05FF5AA85280057
:10B45000EFD01F85EFF01FF7AA852800EFD05F849B
:10B46000014781463000A6854A85EFC0EF8D130461
:10B470007402480822CC230A010002CEEFE0AFBDDF
:10B4800005616F603F8DEF625F8B01117C003ECAEA
:10B49000B70708003ECC7C003ECE83C795002E84C3
:10B4A000AA8493F7F707A384F500A1659385850225
:10B4B0004808EFB0FFE8EFF07FEEAA854808EFD02C
:10B4C0002FFEEFF03FF0AA854808EFD06FFD50083F
:10B4D00001478146A2852685EFC00F8705616F6011
:10B4E0001F8897A7FF1F9387E76F9C43014599C368
:10B4F00003C5B7008280EF625F840111B7070700C0
:10B500003EC683C79500404D0AC493F7F7070AC8A3
:10B51000A384F5002A89AE8405C41C42054783C76D
:10B520000700636AF7040347B400630BF700A30541
:10B53000F400EF7050238347B400A9C3EFD00FD9B4
:10B5400021649305B4002800EFB09FDFEFF07FF98E
:10B55000AA852800EFD0CFF4014781463000A685A8
:10B560004A85EFB07FFE2904480822CC230A010057
:10B5700002CEEFE04FAE05616F606FFEEFD02FDAC5
:10B58000C1B7EF628FFB01117C003ECAB70707000D
:10B590003ECC7C003ECE83C795002E84AA8493F7D0
:10B5A000F707A384F500A165AD054808EFB05FD9A2
:10B5B000EFF03FF3AA854808EFD08FEE500801471F
:10B5C0008146A2852685EFB03FF805616F602FF9AF
:10B5D00097A7FF1F938707619C43094599C303C53C
:10B5E000C7008280EF626FF501117C00AE843ECA15
:10B5F000A165B70707002A843ECCD1057C00480826
:10B600003ECEEFB0FFD3EFF0BFFCAA854808EFD0E5
:10B610002FE9500801478146A6852285EFB0DFF269
:10B6200005616F60CFF3EF624FF183C7950093F729
:10B63000F707A384F500EFF0FFFA6F604FF2EF62B7
:10B640002FEE83C795000329C501411193F7F70732
:10B65000A384F5001C4283C90700854763EC3705C6
:10B6600097B7FF1F938747AF9C432E84AA8495C743
:10B67000EFF01FF689476302F50263000902834772
:10B68000C900638C370123063901EF70D00D835751
:10B690002903898B99C3EFA0D0452685A285EFF0B9
:10B6A0007FF4A167CD0748003EC42302010002C613
:10B6B000EFE06F9A41016F60EFE997A7FF1F938753
:10B6C00067529C431D4599C303C5E7008280EF6222
:10B6D000CFE60111B70707003EC683C79500584D56
:10B6E0000AC493F7F7070AC8A384F5002A89AE8431
:10B6F00005C71C4283C7070093968701E18663C88C
:10B70000060485466385D7048346E7006386F60012
:10B710002307F700EF70300521649305E40028004B
:10B72000EFB01FC2EFF07FF9AA852800EFD04FD706
:10B73000014781463000A6854A85EFB0FFE0350419
:10B74000480822CC230A010002CEEFE0CF90056129
:10B750006F60EFE0EF626FDE01117C003ECAB70759
:10B7600007003ECC7C003ECE83C795002E84AA8481
:10B7700093F7F707A384F500A165B9054808EFB072
:10B780003FBCEFF09FF3AA854808EFD06FD1500877
:10B7900001478146A2852685EFB01FDB05616F60FA
:10B7A0000FDCEF62EFD7AA84014417A9FF1F13092A
:10B7B000A943E149EFC0FF906344A400014519A8E3
:10B7C00033053403832709003E958357250063958D
:10B7D000970011056F600FD80504E9BF032E85009F
:10B7E00063040E1017A3FF1F1303C35E032303009C
:10B7F000631503002943639A060E03234E01631564
:10B8000003001D436393070EEF62AFD0C689428ADF
:10B810003E89BA8AB684328BAE8B2A84A1E903555D
:10B820004E0009E501431A856F602FD2A167A98FE9
:10B83000116763F7E700EFF0DFF68145EFF08FBDAA
:10B840000844B70700E05841F98F18455CC1B707B5
:10B85000001FF98F1CC55C4981C76105EFB010005E
:10B86000E38209FC2285EF70606E6DBF3285EFA028
:10B87000E0620D434DD91C44116703D54700A16711
:10B88000A98F63F7E700EFF0DFF18145EFF08FB8A4
:10B890000323840093164B01D1828347B3000356E0
:10B8A00063008588FD8BA305F300FD777D8E558EA3
:10B8B000FD76FD16B204F18E83274301C58E231257
:10B8C00073012313D3002304530123052301A3048D
:10B8D0004301D9D72285EFB07FBBAA850844B5DDE7
:10B8E0006105EFB02076ADBF1D431A858280EF62FF
:10B8F0002FC30569AA84AE89328A0144FD5A7D1995
:10B90000EFC0EFF06345A40001456F60AFC4D844B9
:10B9100093171400BA9703D70700631B37032390CC
:10B92000570163050A002685EF70E0389C448DC3FB
:10B9300083D76700B3F72701639C3701D28801489A
:10B94000814701478146014681452685EFF01FE981
:10B9500005047DB7EF62CFBC79711C103EC4B707F8
:10B960000F003EC61C103EC883C79500AA8A3285C8
:10B9700093F7F707A384F5002E893284EFD00FBE2A
:10B9800093170501C1876350F006AA892285EFD07D
:10B99000EFBC2A8A4E85032B0400EFB05F9039E597
:10B9A0008357440081440544F11793B71700A3035C
:10B9B000F10083457100DA872287D2864E862800FF
:10B9C000EFE03FA4014781463000CA855685EFB0BD
:10B9D000BFB7A1679387F70348083ECC230A8100CD
:10B9E00026CEEFD05FE745616F60CFB6A285130624
:10B9F0007100EFE0BFAFAA84094445DD5285EFE056
:10BA0000EFB80D445DD50546D2852685EFF03FEEB3
:10BA10002A8445B7EF626FB28355070003462700BB
:10BA200041112A842E8532C62EC4EFE02FB611C5EF
:10BA30003246A2452285EFF09FEB41016F602FB2A5
:10BA4000EF622FAD83C795004111AA8A93F7F707DC
:10BA5000A384F5003285AE893284EFD02FB09317DE
:10BA60000501C1876357F008C1452A8A2285EFD0B6
:10BA70004F9B2A8D2285EFD06FAE2A892285EFD089
:10BA80008FAC930705F893F7F70F1307E007AA8B1E
:10BA90006371F7062285EFD00FAB2A8C2285EFD099
:10BAA0008FAAAA8C5285032B0400EFB04FFF29E523
:10BAB00083574400231101008144F11793B7170005
:10BAC000A300F1000544034711008356210093872A
:10BAD00084005685DA8822885286CE85EFE03FE6DC
:10BAE000A167E90748003EC42302810026C6EFD0C3
:10BAF0009FD641016F606FA513061100A285EFE08C
:10BB0000FF9EAA8409E52311010009446DBF930536
:10BB100021006A85EFF06FA12A8455F58355210035
:10BB20009356C9001316490185486688E2875E87E7
:10BB3000858A51822685EFF07FCA2A8469B7EF6231
:10BB40004F9D83C7950041112A8B93F7F707A38474
:10BB5000F5003285AE893284EFD04FA093170501EE
:10BB6000C1876352F0082A8A2285EFD02F9FAA8AC4
:10BB70002285EFD0AF9E2A892285EFD0CF9C9307F4
:10BB800005F893F7F70F1307E0072A8C637DF70496
:10BB90002285EFD04F9BAA8C2285EFD0CF9A2A8D99
:10BBA0005285832B0400EFB08FEF29E183574400C7
:10BBB00085440144F11793B71700A301F10003472F
:10BBC0003100930784005A85DE882688D6865286FF
:10BBD000CE85EFE0DFD68D4748003EC423029100BA
:10BBE00022C6EFD05FC741016F602F96A285130672
:10BBF0003100EFE0BF8F2A84894471D19356C90088
:10BC00001316490185486A88E6876287858A5182CA
:10BC1000D685EFF0BFBCAA845DB7EF626F902A892A
:10BC200081440144617A916A17ABFF1F130B8B1A91
:10BC3000EFC0EFBE63C5A40022856F60AF9183277C
:10BC4000090093991400CE9703D5070033074501E7
:10BC5000420741836362570311CD03270B0009C7D5
:10BC600085453E85EF30E04A832709000504CE97DD
:10BC70002390070085046DBFEFF0BFB28327090052
:10BC80000504CE972390070075D58145EFE09FF816
:10BC9000D5B7EF62EF8883C7950041112A8A93F7E1
:10BCA000F707A384F50032852E893284EFD00F8BFD
:10BCB00093170501C1876354F004AA89832A0400FD
:10BCC000EFB0EFDD21E18357440085440144F117D3
:10BCD00093B71700A301F10003483100D6875285BE
:10BCE0000147CE862686CA85EFD01FE3A167F507F8
:10BCF00048003EC42302910022C6EFD0DFB54101C7
:10BD00006F604F85A28513063100EFE02FFE2A8475
:10BD1000894479D197A7FF1F9387C70B9C4381CB99
:10BD20000449EFC0CFAFAA852685EF30803E1305CA
:10BD30000401EFF09FEE2285EF609079814469BFA6
:10BD4000EF523FFD83C795004111AA8A93F7F70789
:10BD5000A384F5003285AE89328423110100EFC03F
:10BD6000FFFF93170501C187635CF0042A8AC14570
:10BD70002285EFC01FEBAA8B5285032B0400EFB086
:10BD80000FD231E18357440085440144F11793B742
:10BD90001700A300F1000348110003572100DA87C0
:10BDA0005685D2862686CE85EFD01FD7A16793878A
:10BDB000270248003EC42302910022C6EFD0BFA94B
:10BDC00041016F509FF8A28513061100EFE00FF2BA
:10BDD0002A84894469D197A7FF1F9387A7FF9843B7
:10BDE0003E8901CB0449EFC08FA3AA852685EF3099
:10BDF000403213050401EFF05FE2EFC04FA295441B
:10BE000059D9930521005E85EFE03FF2AA8441F500
:10BE10001C480357210022852390E700EF60506BF8
:10BE200083270900ADDB03552100EF30E026A5B7DD
:10BE3000EF523FEE83C795004111AA8A93F7F707A7
:10BE4000A384F5003285AE893284EFC03FF19317A9
:10BE50000501C1876359F0042A8A2285EFC01FF0CB
:10BE60002A895285032B0400EFB06FC321E1835769
:10BE7000440085440144F11793B71700A301F10072
:10BE800003483100DA8756854A87D2862686CE85D2
:10BE9000EFD09FC8A167F90748003EC42302910074
:10BEA00022C6EFD05F9B41016F503FEAA285130687
:10BEB0003100EFE0AFE32A84894479D19167CA97D2
:10BEC000C2071167C1831307F7EF8544E36AF7FAE6
:10BED00097A7FF1F938707F09843BE8B01CB0449B8
:10BEE000EFC0EF93AA852685EF30A0221305040149
:10BEF000EFF0BFD2EFC0AF92954459D11C482285D4
:10BF0000814423902701EF60B05C83A70B00ADDB79
:10BF10004A85EF306018ADB7EF523FE22A84410501
:10BF2000B284EFF09FCF01C52285EF60705A814641
:10BF30000146A6852285EF70C00B1C4C89C7DC47E3
:10BF400099C3228582976F509FE197A7FF1F938720
:10BF500067C99C43014599C313850701828097A750
:10BF6000FF1F938727C888438280EF521FDD9317F6
:10BF7000C600DD8DC2054111C1812A8432C6EFC0E1
:10BF80007FD33246228511829375F60FEFC05FD1C1
:10BF900041016F50DFDCEF52BFD879713C083ED2CF
:10BFA000B7070C003ED43C083ED683C79500AE844C
:10BFB0002A8993F7F707A384F500A16593853504D3
:10BFC0004810EFB0EFB7C165FD15014417AAFF1F78
:10BFD000130ACAE1930A400EAE892E8B2EC6EFC01B
:10BFE0000F874205931704014181C183B24563E382
:10BFF000A702C167FD176385F5004810EFC09FCB0E
:10C00000501001478146A6854A85EFB0EFD34561C0
:10C010006F505FD43307540383270A0BBA9703D6B4
:10C02000C70163083601638835014810EFF0FFF35C
:10C03000DA85050465B7B285EDBFEF529FCD797102
:10C040007C083EC8B70711003ECA7C083ECC83C7B7
:10C050009500AA89328593F7F707A384F5002E8906
:10C06000EFC0DFCF8567637EF502A165AA848905ED
:10C070000808EFB0EFAC2685EF30E052133415001E
:10C080000A04A2850808EFC0BFC1A6850808EFC052
:10C090007FC235C0014781461008CA854E85EFB082
:10C0A000AFCA45616F507FCAB30754030327CA0A5A
:10C0B000BA9703D70700631A970003D62700638A4D
:10C0C00065030808EFF07FEADE8505042EC6EFB0B1
:10C0D0001FF94205931704014181C183B245E3E58D
:10C0E000A7FCC167FD17E387F5FA0808EFC09FBCFE
:10C0F00055B7B285D9BFC165FD15014417AAFF1F09
:10C10000130ACACE930A80022E8BAE8BC1B7EF52B0
:10C11000DFC218418347170083460700A207D58F67
:10C12000D207D1832390F5008347270003471700E8
:10C130008D45A207D98F91832310F600EFC03FAD44
:10C140006F50FFC1EF52DFBDC164014417A9FF1F4B
:10C150001309C9C993098002FD14EFB05FF063456C
:10C16000A40001456F501FBF330534038327C90A5C
:10C170003E9583570500E38797FE0504F9BFEF520C
:10C180003FBA2A8AAE89B284B68AEF30C04109E547
:10C1900091473E856F501FBC2A894E85EF90105005
:10C1A0002A84638A0A048D476DD503570500C54765
:10C1B000E31147FF0347F9018546AD47E31BD7FC71
:10C1C0008347450091CB4146A6855D05EFC0D0224F
:10C1D000814761D1AD4775BF130965012302E500B1
:10C1E000CA852685EF10202D15CDA547E3830AFAD1
:10C1F0002302040079BF11CD83570500E39A47F964
:10C200004146A6851905EFC0301F814759D199478E
:10C2100049B74E85EFF01FF32A8495473DD913099E
:10C2200055007DBF4146A6852310440123113401EA
:10C2300013051900EFC0B01E2285EF60B03C8147A6
:10C2400089BFEF529FAF79717C003ECCB7070A00DF
:10C250003ECE7C003ED083C79500B2842E8493F7F7
:10C26000F707A384F5001306A1002A892C00268570
:10C27000EFF0FFE9A16528088D05EFB06F8C9040C5
:10C280008355A100035581008546EFF05FEFAA8436
:10C29000AA852808EFC0DFA00356A10083558100BE
:10C2A0002808EFF09FCC300801478146A2854A85D7
:10C2B000EFB08FA9854748103ED42302910202D6E1
:10C2C000EFD06FD945616F509FA9EF521FA77971C9
:10C2D0007C003ECCB7070A003ECE7C003ED083C730
:10C2E0009500B2842E8493F7F707A384F500130614
:10C2F000A1002A892C002685EFF07FE1A16528089E
:10C300008D05EFB0EF8390408355A1000355810068
:10C310008146EFF0DFE6AA84AA852808EFC05F987F
:10C320000356A100835581002808EFF01FC4300890
:10C3300001478146A2854A85EFB00FA1481023022C
:10C34000910202D402D6EFD00FD145616F503FA1C8
:10C35000EF52BF9EEFF0BFE26F507FA097A7FF1F85
:10C360009387878888438280EF523F9D83572500BB
:10C370004111AE842A842307B10017F5FFFF13058E
:10C38000A5696C002316F100EFB0CFD581C42285DA
:10C39000EF60B02DFD572310F400130620028145F5
:10C3A00013055400EF507F9C41016F505F9BEF528B
:10C3B0003F9779717C003ECCB7070A003ECE7C00E7
:10C3C0003ED083C79500AA89AE8493F7F7073285DC
:10C3D000A384F5001306A1002C00EFF05FD30355F2
:10C3E00081001144EF30201C15C10355A100014408
:10C3F000EF90D02A01CD03570500835781004544B3
:10C400006316F7008545EFF03FF601442169930577
:10C4100039002808EFA0DFF2A2852808EFC05F8866
:10C420000356A100835581002808EFF01FB430089F
:10C4300001478146A6854E85EFB00F9148104AD43A
:10C440002302810202D6EFD00FC145616F509F9049
:10C45000EF521F8D9797FF1F9387C7782A848843D1
:10C460002E8915C1035745038357C401631DF70087
:10C4700023260502231805024105EFA0303E630480
:10C480000900EF60302F814497A9FF1F9389099617
:10C49000130A8002EFB0BFBC63CCA4029797FF1FC2
:10C4A0009387077D9C4389C70355C401EF104076ED
:10C4B000630509002285EF6050031306400E814595
:10C4C0002285EF509F8AFD57231EF4006F509F88EE
:10C4D0003385440383A7C90A3E9503570500835754
:10C4E000C4016315F700CA85EFF01FE885045DB746
:10C4F000EF521F8383C795004111AA8993F7F7076D
:10C50000A384F5003285AE84EFC05F8585676370D4
:10C51000F5042A89EF302009014411C983D70400AA
:10C520003144638627018545EFF09FF201444E8533
:10C53000A2864A86A685EFD02FBFA16793871704EE
:10C5400048003EC42302810002C6EFD0CFB04101B3
:10C550006F505F80EF52CFFC9797FF1F93878768DC
:10C5600080431DCC0145EFA0E05681470148C164DE
:10C570001CDC232E04032320040417A9FF1F130926
:10C58000E98601449309400EFD14EFB05FAC634BA4
:10C59000A40081451705000013054598EFB08FB43E
:10C5A0006F504FFB330534038327090B3E958357A8
:10C5B000C501638597008545EFF09FE90504F1B754
:10C5C0009357050113D78700A380F5009317050142
:10C5D000C183A1832380E5002381F500A381A50009
:10C5E0008280EF528FF52300050083C71500A3005A
:10C5F000F50083C725002301F50083C73500A3019B
:10C60000F50083C745002302F50083C75500A30248
:10C61000F50083C7650093059500A3030500230378
:10C62000F500230405003285EFF09FF96F502FF3DA
:10C63000EF520FEF4111E9541DC995C993F9C5FF98
:10C640002E842A89AA84338AA900B7EA04006314D5
:10C650009A020D88854401CCB7E704009C5F82975D
:10C660002AC622866C0033053901EFC0405B26855F
:10C6700041016F502FEE83A78A039104829793178D
:10C680000501C183A183A38EF4FE93570501238F77
:10C69000F4FEA183238EA4FEA38FF4FE4DBF63E0BE
:10C6A000D502EF528FE9B28741113686BE8536C674
:10C6B000EFC0E056B246410136856F504FEA8146E1
:10C6C00036858280838705001387F5003D05FD8749
:10C6D00093F77708834607007D158606B58FA3007C
:10C6E000F5006307B7007D17834717009D83DDB70B
:10C6F0008280EF528FE4B7E7040083A707093287EF
:10C700002A863A858297133515006F504FE501CD83
:10C71000814799C9EF526FE24146EFC040508547CB
:10C720003E856F50CFE381473E8582801DC5EF5225
:10C73000CFE0414681452A84EF502FE341468145B1
:10C7400013050403EF506FE20147C167232204047D
:10C7500038C87CC805456F508FE00145828081470D
:10C7600029CDA1CDEF526FDDB2842E89130680054D
:10C7700081452A84EF506FDFCA8524C42685EFF0F7
:10C780001FF9414681452285EF502FDE3044A285B6
:10C790002285EFF01FF693040401A2852685EFF0B1
:10C7A0007FF2A68513050402EFF0DFF12285EFF09A
:10C7B000FFF785473E856F508FDA3E858280EF52C6
:10C7C0002FD64111E9541DC995C993F9C5FF2E848F
:10C7D0002A89AA84338AA900B7EA0400639444032F
:10C7E0000D88814401CCB7E704009C5F82972AC67C
:10C7F00022866C0033053901EFC060422685410175
:10C800006F504FD583A78A03910482979317050130
:10C81000C183A183A38EF4FE93570501238FF4FEF9
:10C82000A183238EA4FEA38FF4FE4DBF71CDEF52E2
:10C830002FCFB28401E605456F50CFD12A842E89CF
:10C840000145FDD93C487848B3E6E700F5D6938624
:10C85000F7FFB3B7F6007D17032A4404BA9734C82C
:10C860007CC8630F0A04C14913050A03B38949410F
:10C870002295637B3601B2862E86A685EFF03FE2D5
:10C880007C40BE9464C045BFCE862E86CE85EFF038
:10C890001FE1C114D2944E9923220404A287930667
:10C8A000040103C7070003C607038507318FA38F61
:10C8B000E7FEE398F6FE3044A2852285EFF07FE3A1
:10C8C0002699C1493306994063EA9900ADD4A686FA
:10C8D000A68513050403EFF09FDC6DB78147B3060F
:10C8E000F4003307F6000347070083C506008507F9
:10C8F0002D8F2380E600E39437FF3044A285228504
:10C90000EFF03FDFC1147DBF0145828019C9EF52AE
:10C91000CFC2130680058145EF502FC505456F50E6
:10C920000FC40145828081473DC9B5C9EF52EFC0B0
:10C93000FC4141462E84AA846393C70413860501F3
:10C94000A2878146C14503C7070003C507038507C2
:10C95000298F3305D600034505008506298FA38F4F
:10C96000E7FEE392B6FE3044A2852685EFF07FD83D
:10C970002285EFF0BFF985473E856F504FBE138586
:10C9800007031D8E81452295EF502FBE7C40130773
:10C9900000F813060402A2972388E70255B73E85E4
:10C9A0008280EF528FB96D712E84B284AA85901067
:10C9B00028003689EFF0BFDA19E9D55705A05040B5
:10C9C0000C402800EFF09FE66DD9FD142104E5F836
:10C9D0002C004A85EFF03FF5814765D13E855161D6
:10C9E0006F50EFB7EF526FB541112EC432C62C0015
:10C9F0000546EFF01FFB41016F506FB6EF52EFB3EA
:10CA000001112A842EC602C802CA02CC02CEEFC08F
:10CA10006049B2462A86A2850808EFF0BFFC13756C
:10CA2000F50F05616F50AFB3EF522FB17971B28737
:10CA30002A8421462308B10013051101BE853AC49A
:10CA400036C6EFC0C01DB246930591013685EFF0A2
:10CA50003FB72285141035460C08EFF0BFF82A8442
:10CA6000224711E521460C103A85EFC0401B228574
:10CA700045616F50CFAEEF524FAC7171AE84AA8555
:10CA80000A853284EFF0BFC801C90A86A6852285CF
:10CA9000EFF03FC6814711E1C5473E854D616F50BC
:10CAA0000FACEF528FA61D712A8AB289BE8435461B
:10CAB0008547130511012E8CB68A3A8BC28C468DA0
:10CAC0002308F100EFC0A01510100C085285231F99
:10CAD0000100EFF05FFA2A842DE9A147631BFD06F0
:10CAE0009307900591E0E5473546E285130511016E
:10CAF00013990A012308F10013590901EFC020120C
:10CB00001357890093978A00D98F90080C08528593
:10CB1000231FF100EFF03FF62A8405E9A1E0938797
:10CB2000FA0091831379F9003EC663130900414965
:10CB3000668B8144C14B854DB2476397970C6A86DB
:10CB40008C0033855C01EFC0800D228525616F501C
:10CB50008F9F93079004C9F8A54779B783470105CC
:10CB60000947C14B2308F10083471105A58FA3088E
:10CB7000F10093872400814463EFFB02014714080E
:10CB80003386E6008C08B386E400BA95DA9683C64D
:10CB9000060083C505000507AD8E2300D600E3908F
:10CBA000E7FE41476398E70490080C085285EFF0D0
:10CBB0009FEC35D535A8B3069B00BA871008B3059E
:10CBC000F60090083E9603C506000346060085075A
:10CBD0008506298E2380C500E39277FF998F900800
:10CBE0000C085285BE94EFF01FE98947014749D5EB
:10CBF0002A84A1BF90083E96034606001408BE96FC
:10CC00002380C600850779BFB2478504638B9712DE
:10CC100081471808B306F70098083E973386F90055
:10CC200003470700034606008507318F2380E6008F
:10CC3000E39177FF90080C085285EFF0DFE34DF9A0
:10CC40003546E285130511012308B101EFB0307DAF
:10CC5000139704014183939784002183D98F10187F
:10CC60000C085285231FF100EFF0FFE051F18147DE
:10CC700010183387F9003E96034707000346060065
:10CC8000B306FB008507318F2380E600E39277FF30
:10CC900075A01808B306F70098083E973386F90088
:10CCA00003470700034606008507318F2380E6000F
:10CCB000E3E127FFCA876398770990080C0852853B
:10CCC000EFF07FDB15F581479800B306F700900879
:10CCD00018103E973E960347070003460600850757
:10CCE000318F2380E600E39177FF3546E285130517
:10CCF00011012308B101EFB0907213970401418331
:10CD0000939784002183D98F10180C085285231F14
:10CD1000F100EFF05FD6E31D05EC81471018338773
:10CD2000F9003E960347070003460600B306FB00E2
:10CD30008507318F2380E600E3E227FFC109410B1D
:10CD4000E5BB8147B5B79408BE9683C606001808B0
:10CD50003E972300D7008507B9BF638E062CEF42AC
:10CD6000DFFA59712A84BE89B28B8547354613058F
:10CD700011022E8B468C4289BA8A368A2300F10230
:10CD8000EFB0F06910180C10228523170102EFF0A4
:10CD90009FCE631E0510A1476319FC0693079005FB
:10CDA00063930900E5473546DA85130511029314AC
:10CDB0000A012300F102C180EFB0706693178A0068
:10CDC00013D78400D98F90080C1022852317F10205
:10CDD000EFF07FCA69ED639009049307FA00BD88FC
:10CDE000918391E0C144C207C183DE8C814A3EC673
:10CDF000414DB24763EAFA0C6286B3854B01881055
:10CE0000EFB0905F4DC53D555DA093079004E39C46
:10CE100009F8A54749BF834701050947C14C2300CD
:10CE2000F10283471105B3C7F900A300F10293870C
:10CE30002900814963EFFC02814618103306D700B0
:10CE40008C083387D900B69556970347070083C5EA
:10CE5000050085062D8F2300E600E390D7FE4147AD
:10CE6000639AE70490080C102285EFF0DFC035D5F7
:10CE70003DA8B3863A01BA871010B305F6009008B2
:10CE80003E9603C506000346060085078506298EE3
:10CE90002380C500E39297FF3387EC4090080C1085
:10CEA0002285BA99EFF03FBD8947014741D56561B9
:10CEB0006F407FE990083E96034606001410BE9628
:10CEC0002380C600850769BFB247850A93990A0186
:10CED000939D8A0093D909016399570D854735467B
:10CEE000DA85130511022300F10293D98900EFB00E
:10CEF0001053B3ED3D0190000C1022852317B103B0
:10CF0000EFF07FB74DF58147A68963E69706268641
:10CF10000C084A85EFB0B05081471810B306F700EF
:10CF2000100898083E973E96034707000346060000
:10CF30008507318F2380E600E3E197FE639DA90515
:10CF400090080C102285EFF01FB335F1814798103F
:10CF5000B306F700900818183E973E96034707005F
:10CF6000034606008507318F2380E600E391A7FF83
:10CF70004109C10CBDBD18089000B306F7003E96EC
:10CF80003387FC0003470700034606008507318FFF
:10CF90002380E60095BF98084E97034707001C10B2
:10CFA000CE972380E700850951BF85473546DA854E
:10CFB000130511022300F10293D98900EFB0304626
:10CFC000B3ED3D0190000C1022852317B103EFF063
:10CFD0009FAAE31E05EC814718089000B306F700EE
:10CFE0003E963387FC00034707000346060085078B
:10CFF000318F2380E600E391A7FF41460C084A8564
:10D00000EFB0F04181471810B306F70010089808F8
:10D010003E973E9603470700034606008507318F7B
:10D020002380E600E391A7FF90080C102285EFF023
:10D030009FA41DDDADBD7D558280EF421FD0011143
:10D040002A842E8593055100328902C002C202C48F
:10D0500002C693047400EFF0AFD61D46A6851305F3
:10D060009100EFB0D03B10088A854A85EFF0BFA051
:10D0700019ED93071400180883C60700034607003C
:10D0800085070507B18EA38FD7FEE397F4FE0561F0
:10D090006F40FFCCEF42DFC82E848C414111AA893A
:10D0A000838715003289914463D30700A144979781
:10D0B000FF1F9387670A9C43B1C3B5CE8D472310EA
:10D0C000F10083C725004A852301F10083C735009D
:10D0D000A301F10083C745002302F10083C7550077
:10D0E000A302F10083C7650093059100A30301002B
:10D0F0002303F10023040100EFF08FCC0C404A869B
:10D100000A85EFF00FCE0328040083564400A6885A
:10D110001D0881470147E51642868A854E85EFF056
:10D120005F982A8909E5A6852285EFB0FFB24A8576
:10D1300041016F403FC24A860A85EFF08FCA7DBF2A
:10D14000EF421FBE2E848C414111AA8983871500AE
:10D150003289914463D30700A1449797FF1F9387B7
:10D16000A7FF9C43B1C3A5CE8D472310F10083C711
:10D1700025004A852301F10083C73500A301F10092
:10D1800083C745002302F10083C75500A302F100C5
:10D1900083C7650093059100A30301002303F100F9
:10D1A00023040100EFF0CFC10C404A860A85EFF05E
:10D1B0004FC383564400032804008A85858EC20627
:10D1C0001D08C1822312D400A68881470147E516B5
:10D1D00042864E85EFF07FB841016F40BFB74A8667
:10D1E0000A85EFF00FC0C9B7EF423FB5B335B000C5
:10D1F000011185052A891315F601336515012308E8
:10D20000B1009305110136843AC632C03EC442C211
:10D21000EFF00FBBA2471248425593D68700230B6D
:10D22000F1009305910193578800A30AD100A30B45
:10D23000F100230C0101EFF0AFB83247024603289A
:10D240000400B337E000835644009207914411C2B2
:10D25000A1444A85A68842860C08EFF09F842A895B
:10D2600009E5A6852285EFB03F9F4A8505616F409D
:10D270001FAFEF42FFAA01113EC68647B335B0008B
:10D280008505AA891315F6015D8D2308B100930564
:10D29000110136843A89B28442C446C2EFF04FB2DB
:10D2A00022489248164593578800A30AF100930537
:10D2B000910193D78800230B0101A30BF100230CEC
:10D2C0001101EFF0EFAF3247104083564400B337FF
:10D2D000E000920703280900914891C0A1480C087A
:10D2E0004E85EFF09FA7AA8411E5835544004A8537
:10D2F000EFB09F96268505616F40DFA5AA9593073D
:10D30000F00F17F700001307278A6317B50013C53E
:10D31000F7FF1375F50F828005058346F5FFB58F7E
:10D32000BA9783C70700D5B7035745001441930741
:10D33000F00F17F600001306268736974207418341
:10D34000139506014181631BE500AD8FB29703C5BC
:10D350000700130515F3133515008280850603C5F4
:10D36000F6FFA98FB29783C70700D9BFEF42FF9C92
:10D37000B28736842E86BA86AA853E85BA84EFF0B7
:10D380006FE6634B05002285EFB0D0312A86A68672
:10D39000A2852685EFF00FE56F407F9CEF425F98F6
:10D3A0005D712A8BAE8A17E500001305657D2C00A0
:10D3B000B284368ABA893E89EFF04FE42A8459E56F
:10D3C00034104146DA852800EFF0CFE12A843DEDA4
:10D3D0008547A303F100A6C2930771002408BEC4C9
:10D3E000A68685470D462C18281002DC02DED6C022
:10D3F000BEC6EFF00FDB2A8431E983477102A686AF
:10D400000D4693F7F7072300FA00C1473EDE2C18BC
:10D410008947281026DCA303F100EFF08FD82A8477
:10D4200015E54146A6854E85EFB0607F8D47A686FF
:10D430000D462C182810A303F100EFF08FD62A8494
:10D4400011E54146A6854A85EFB0607D2285616180
:10D450006F405F90EF427F8E97D700009387070C55
:10D46000984383C7470079712A89AE8417E5000085
:10D47000130585710C083AC42306F100EFF00FD8AC
:10D480002A8415E514104146CA850808EFF08FD5A7
:10D490002A8411ED140815462C000810EFF08FD4E3
:10D4A0002A8411E521462C082685EFB04077228595
:10D4B00045616F40DF8AEF425F8897D7000093870E
:10D4C000E7059C477971AA842E8417E500001305AF
:10D4D000256C0C083EC6EFF06FD20DE514104146E6
:10D4E000A6850808EFF00FD011ED140811466C0066
:10D4F0000810EFF02FCF19E58347F10193F7F703F9
:10D500002300F40045616F409F85EF421F833688FA
:10D51000A14881470147E546EFF0AFD86F403F840F
:10D52000EF42BF813688A14881470147E546EFF0C9
:10D53000DF826F40DF82EF425F8001112A842E85F7
:10D540000C0832C6EFF08FCB19E9324797E600009E
:10D55000938686621008C1452285EFF03FE10561A0
:10D560006F40EFFFEF426FFD4111C1472EC032C443
:10D570008A8509463EC23EC6EFF0AFC241016F4008
:10D580000FFEEF428FFB4111AE8613061009AA85EC
:10D590000A8502C002C202C402C6EFF0AFC4410154
:10D5A0006F40EFFBEF426FF9328797E600009386FA
:10D5B000A65E2E8693050002EFF05FDB6F402FFA28
:10D5C000EF42AFF77971C1472ACC2ED032D42C0864
:10D5D0000D4628003ECE3ED23ED602C402C602C848
:10D5E00002CAEFF00FBC45616F406FF7EF42EFF4F6
:10D5F0000111AA842E8417E500001305655A8A8557
:10D60000EFF0CFBF05E514084146A6850A85EFF087
:10D610006FBD09ED8347E1010347F101A207D98FEF
:10D62000CA07C9836177D98F2310F40005616F4061
:10D630000FF305C9EF426FF09787FF1F9387475F8E
:10D6400090439785FF1F9385E55E1785FF1F1305A0
:10D65000255AEFB080091785FF1F130565596F40E4
:10D660000FF01785FF1F1305A55882809DC5EF4257
:10D67000CFEC9787FF1F9387A75B944301112E84FC
:10D680000A869785FF1F9385E55AEFB0800A0A85C1
:10D690000294014505616F408FEC7D558280EF4219
:10D6A000CFE9EFB080149787FF1F23A3A75817F582
:10D6B000FFFF130525F8EF90D0406F404FEA178722
:10D6C000FF1F130727599317150008433E95FD5771
:10D6D0002310F5008280EF424FE62A84084019E1CA
:10D6E0006F40EFE71C4158401CC06313E5005CC06D
:10D6F0008347550023200500F99BA302F500EFB0F6
:10D70000EFF9E9BFEF42CFE19787FF1F9387875675
:10D7100098432A8411CB8347350093F7070289C7C2
:10D72000035505008945029713054401EF90101336
:10D73000835504000355E400EF20701B485809C5C9
:10D74000EFB0CFF5232A040213058403EFF0BFF8EE
:10D750008144B149EFA0FF9A63C5A4028347340016
:10D760002320040493F727FCA301F4000048EFA052
:10D770005F9A1316150081452285EF400FDF6F4039
:10D780006FDDB38734030329040385043E994A857A
:10D79000EFF07FF42304090075BF8347350093F74A
:10D7A000070299E3014582808357E500E39CB7FEB9
:10D7B000C167FD176316F600054582800545B9A0CF
:10D7C000EF42AFD793170601C187B2842A8401497B
:10D7D0006359F002835705008DCB01456367F6005E
:10D7E000034584003E953325A6001375F50F39A82F
:10D7F0001C4813171900BA9783D70700E38097FCDA
:10D800000509EFA01F91E345A9FE01456F402FD503
:10D81000EF420FD1AE89AA84EFA07F852A84EFD092
:10D82000BFAAAA86014713068401970500009385C5
:10D8300045E91785FF1F13052542EFA0AFD52A89BB
:10D8400021CD8C441304C50022859E0593F505085F
:10D85000EFB00FC5CC4083877400E18163D107042A
:10D8600093E505082285EFB0AFC30D4693854400CC
:10D870002285EFB00FC183D504002285EFB0EFC53C
:10D8800083D524002285EFB04FC503D6490083A578
:10D8900009002285EFB0EFBE4A856F40AFCB93F50C
:10D8A000F507C9B7EF426FC901112A84328532C624
:10D8B000EFB06FB4EF903F91835704001787FF1FBD
:10D8C0001307C7523246231BF100930700F8A30D3C
:10D8D000F1001C471843231AA1008983858BB307E5
:10D8E000F740B28548083ECE231C0100230D0100FD
:10D8F000EFF01FF205616F408FC6EF426FC200412B
:10D90000014529CC9304C40026853289AE89EFB045
:10D910008FB295452A8A2685035B0401EFB02FAFAD
:10D920002685EFB02FC68D45AA8A2685EFB02FAE8B
:10D930002685EFB02FC55C48420A135A0A01D297D8
:10D940005CC423186401814763983A0146054D8100
:10D95000330625419337160013F5F70F6F408FBF3D
:10D96000EF422FBB89692A8BAE8B328AB68A8144FB
:10D970000144314CFD19EFA0CFF863C9A400EFA01A
:10D980004FFB018D33B5AA006F402FBC3389840350
:10D9900083270B003E9963170A008347890085049B
:10D9A0003E94D1BF03560A00DE854A8533F6C9008E
:10D9B000EFF0BFF47DD10545C1BFEF420FB80111B3
:10D9C0002A847C000355E5003ECAB70707003ECC19
:10D9D0007C003ECEEF10303D2A8985454808EFB0E7
:10D9E000EFC199454808EFB02FA7AA844A85EF10E8
:10D9F000B03D2380A4009787FF1F9387273F9C4358
:10DA00004166130606F09396870113D78701558F59
:10DA100093D68700F18E558FA207B706FF00F58FCA
:10DA2000D98F11462C00138514003EC4EFB0201F7F
:10DA30005008A382040089452285EFF0BFE609C99A
:10DA4000AA8513058403EFB0EFBB3C4085073CC0BB
:10DA500005616F40CFB0EF424FAEEFA08FED2A844B
:10DA60000504EFA00FEC3305A402F14791453305FF
:10DA7000F502EF10207B01E565556F404FAE9787AB
:10DA8000FF1F23A1A71EEFA0CFEA2A840504EFA061
:10DA90004FE93305A40289450605EF10A07869DD3A
:10DAA0009787FF1F23A8A71AEFA0AFE82A840504D1
:10DAB000EFA02FE73304A4029787FF1F239E871848
:10DAC000EFA02FE72A84EFA0CFE59307140033855A
:10DAD000A7029787FF1F2392A71897E70000938755
:10DAE000E7CF1787FF1F232DF716014579B7EF42C0
:10DAF0002FA3AA842E8901449789FF1F9389092F98
:10DB0000130A8006EFA0EFE16345A40001456F40D2
:10DB10006FA43305440383A709024A86A6853E9570
:10DB2000EFF0BFC719E10504F1BF0545CDB7EF42DE
:10DB30004F9EAA8A2E8BB28B368C3A8A814401443E
:10DB40008149978CFF1F938C6C2A130D8006EFA0E0
:10DB50004FDD63C7A40011E085494E856F40EF9EFD
:10DB60003389A40383A70C025E86D6853E994A8535
:10DB7000EFF0BFC219CDEFA0CFDB0544636B4501C9
:10DB8000D2866286DA8513050903EFF07FDD11C1C5
:10DB9000854985046DBFEF42AF98C16441112A8960
:10DBA00001449789FF1F93896924130A8006FD1495
:10DBB00036C632C42EC2EFA0CFD692452246B24618
:10DBC0006346A400014541016F40CF9833054403EB
:10DBD00083A709023E9509C683473500C18B9DC7BF
:10DBE00091C68347350093F707028DC363069900FA
:10DBF0008357E500639C27010357050001CB63E7CA
:10DC0000E50083478500BA97E3CFF5FA05044DB7E1
:10DC1000EF420F91C1642A8901449789FF1F9389BC
:10DC2000E91C130A8006FD14EFA0AFCF6344A400E3
:10DC30006F404F923305440383A709023E958357F3
:10DC4000E500638897006304990063942701EFF06F
:10DC50007FAB0504D1BFEF424F8B89692A8AAE8A18
:10DC6000328BB68B8144178CFF1F130C2C18930C2E
:10DC70008006314DFD19EFA0CFCA63C4A4006F40E8
:10DC80008F8C3389940383270C028355CA015A86EB
:10DC90003E994A85EFF07FB005CD814D05A03384D4
:10DCA000AD038327090303D60B00D68533F6C900DD
:10DCB0003E942285EFF07FC419E5850DEFA06FC477
:10DCC000E3CFADFC31A02285EFF0FFA023040400D8
:10DCD000850455B7EF42EF834169AA8A014A178B41
:10DCE000FF1F130BAB107D19C14B054CEFA06FC389
:10DCF0006344AA006F406F8593098006B3073A0317
:10DD000083290B02BE9983D7E900638C27016384C2
:10DD10002A016398570103A4890311E44E85EFF0AB
:10DD2000DFC9050AE1B783570401639977079304B4
:10DD3000C4002685EFA03FF085452A8D2685835CAB
:10DD40000401EFA0DFEC2685EFA0FFFF62056185EF
:10DD5000635F05028D452685EFA07FEB894526850B
:10DD6000EFA0FFEA89452685EFA07FEA8545268555
:10DD7000EFA03FEB83470500094793F7F707639848
:10DD8000E70099452685EFA0DFE9A3028501484811
:10DD9000337D2D01231894016A9548C40040B5BF16
:10DDA000EF32BFF937E404008327041D8297978779
:10DDB000FF1F83C7A7F01755FF1F1305A539A30041
:10DDC000F5008327441C82978327841C8146130611
:10DDD000F00F8145014582976F307FF81787FF1F4D
:10DDE0001307C7DD18439785FF1F83C525ED978768
:10DDF000FF1F938727EB83468703034697036397A9
:10DE0000D5009787FF1F238BC7EA828083C58701D0
:10DE10000347A7036317B6009787FF1F2380E7EA2E
:10DE2000828003C687016317C7009787FF1F238778
:10DE3000D7E8828083C68701130750026319D70091
:10DE4000930760021787FF1F230AF7E6828083C6C5
:10DE50008701130660026315D60093077002DDB7D1
:10DE600083C7870155BF9787FF1F9387A7E3D44BCD
:10DE700009476385E608EF325FEC1789FF1F130936
:10DE8000A9DF3E8483470900918B9DCFB7E404004E
:10DE900083A7041D829783A7441C1785FF1F1305C2
:10DEA00025DE829783A7841C81461786FF1F0346C1
:10DEB00026DF81450145829721C183470900ED9BFB
:10DEC0001787FF1F230AF7DA8347040093F7F70F3A
:10DED00085C791471787FF1F2320F7DEEFF05FEC20
:10DEE000EFF0DFEFB7E70400BC4F414691451785DF
:10DEF000FF1F0345A5DB82976F307FE68280EF32FC
:10DF0000DFE38D4741116304F504C5476306F5025D
:10DF100085476310F5029787FF1F2383A7DAB7E7CA
:10DF20000400BC4B930500101785FF1F034505D85F
:10DF3000829741016F30BFE285471787FF1F23019A
:10DF4000F7D8B7E70400BC4B93050020F1BF9787D3
:10DF5000FF1F938727D5D44B1147638DE600B7E7A2
:10DF6000040083A7071D8297B7E70400BC4B930505
:10DF700000045DBF05491787FF1F232F27D383C7E1
:10DF8000070032C62E8493F7F70FC5D7B7E4040015
:10DF900083A7041D7D141374F40F8297E37689FC24
:10DFA000B245994703C61500E3F0C7FCFC440906D7
:10DFB0001785FF1F130505D18297BC4893050008FC
:10DFC0001785FF1F034585CE829779BFEF32FFD6B5
:10DFD0001787FF1F130707CD4047184B1C40978634
:10DFE000FF1F23A7F6CC6316E4001787FF1F232328
:10DFF000F7CC130584FEEF907FF3035564FFEF9099
:10E000003FC6EFA0BFE96F309FD5EF321FD3978790
:10E01000FF1F938727C9D84BDC4799C3EFF01FFB3D
:10E0200085471787FF1F2329F7C89787FF1F938707
:10E03000E7B89C43930500021785FF1F034505C7FA
:10E0400083C787031787FF1F230AF7C6B7E70400B4
:10E05000BC4B82976F30BFD09787FF1F23A6A7C402
:10E060008280EF32FFCB37E404007C4CA14517855A
:10E07000FF1F0345A5C382977C48A1451785FF1F55
:10E080000345C5C29784FF1F9384C4C18297DC44B3
:10E0900089E7EFF05FDD6F30FFCB03D567FFEF90CF
:10E0A0003FBCAA897DD5D84891476310F7027C4CC4
:10E0B00091451785FF1F034565BF82977C489145B1
:10E0C0001785FF1F034585BE829703A9490103D425
:10E0D00009018947B7E904001787FF1F232EF7BC02
:10E0E00083A7091D21044204829783C78401175521
:10E0F000FF1F1305250661191757FF1FA30CF7040F
:10E1000083A7491C418082979787FF1F238A07BAFC
:10E1100083A7C91C814609469375F40F4A858297E7
:10E1200011E99787FF1F83C7E7C989C79740FF1F7A
:10E13000E7800074B7E70400BC4F2146A14517856E
:10E14000FF1F0345A5B68297B9B7EF321FBF93F7FC
:10E15000052001112E8481CBEFF03FEB1345042005
:10E1600005616F30DFBF93F70510A9CB9784FF1FC0
:10E17000938444B3DC48EFF07FC61787FF1F130773
:10E18000E7A3184383C78401034787036316F70097
:10E19000DC4499C3EFF09FE385471787FF1F232DCA
:10E1A000F7B0B7E70400BC4B930500021785FF1FCB
:10E1B0000345C5AF8297134504105DB793F7050873
:10E1C000ADC79787FF1F83C7F7AFE9171946978534
:10E1D000FF1F938545AF1305D10093F4F70F1789FF
:10E1E000FF1F034929AEEFA0902393970401C18339
:10E1F0001787FF1F130787AD231DF100231CF100B4
:10E200009787FF1F938707AA3ACE3ACAD8432306B7
:10E21000010009CBDC439315890154080D46E185C3
:10E22000680082971345040825BF93F72500B1CFF6
:10E230009787FF1F938707A7D84B89476306F70285
:10E240009787FF1F83C747A313F7270011EF918B11
:10E2500099CFB7E70400BC4F1306000A894517851C
:10E26000FF1F0345A5A4829713452400D5BD9787BA
:10E27000FF1F9387A7949C4383C787031787FF1FBC
:10E28000230EF7A2EFF0FFDDC5B793F7050291C7A4
:10E29000EFF03FDD13450402E1B593F7850091C728
:10E2A000EFF0BFD61345840065BD93F7150091C705
:10E2B000EFF07FBB1345140065B593F7450091C798
:10E2C000EFF07FBA1345440061BD93F7050485C3A1
:10E2D0009787FF1F83C7079D81CBEFF07FAC9147E6
:10E2E0001787FF1F232AF79C1345040495BD93F756
:10E2F00005010145E38607E69787FF1F9387879A05
:10E30000D84B91476310F7049787FF1F9387C796F1
:10E310009C4313D727008583D98F858B91E7B7E777
:10E32000040083A7071D8297B7E70400FC4F9145BF
:10E330001785FF1F03458597829785471787FF1F1E
:10E34000232CF7961345040121BD9787FF1F238BCC
:10E35000A7A68280EF327F9E9787FF1F23AA07948C
:10E360009787FF1F23A8079485471784FF1F13046F
:10E37000E4841787FF1F2321F7941C4083C787037A
:10E380001787FF1F230CF792EF90FFDF39C19757D4
:10E39000FF1F23A5A7DC1C4017050000130525DB84
:10E3A00083C787031787FF1F230AF7901757FF1F9D
:10E3B000A302F7DA9787FF1FA386078EB7E704004B
:10E3C00083A7070882979787FF1F2381A78E6F3047
:10E3D0001F99B7C7898E938767ED1757FF1F232FA4
:10E3E000F7D655BF1787FF1F0347C78B795555E3EE
:10E3F0009787FF1F9387078B03C71700050797862B
:10E40000FF1FA381E68A03C717008D463377D70223
:10E410009786FF1FA388E68883C617001777FF1F1C
:10E420001307C779184393F6F60FA9EA83478703C2
:10E430001787FF1F2304F78885471787FF1F2303CC
:10E44000F7869787FF1F938727839C430145998B06
:10E45000A9E3EF329F8E37E404007C48C14517855D
:10E46000FF1F0345A58482973C4885451785FF1FFC
:10E470000345C583829701456F307F8E83C71700A0
:10E4800085466395F600834797035DB78347A703E7
:10E4900045B782809787FF1F83C7C780A1CBEF3224
:10E4A000DF8937E404009777FF1F238D077E7C48C0
:10E4B00085451775FF1F0345657F82977C4C914505
:10E4C0001775FF1F0345857E82977C489145177518
:10E4D000FF1F0345A57D82973C48C1451775FF1F67
:10E4E0000345C57C829701456F307F8779558280CF
:10E4F000EF32BF842A84035565FFEF906FF697775C
:10E50000FF1F9387277AD847BE841DEBEFA05F9843
:10E510009C48232004008DEB9777FF1F23AC87785E
:10E520009777FF1F23A68778B7E70400BC4B894580
:10E530001775FF1F03458577829701456F303F822E
:10E54000630A87001843D1B780C39777FF1F23A3BF
:10E550008776D9BF7955DDB7EF322FFE9787FF1F3A
:10E5600093878786884323260500232405005105C9
:10E57000EF80D02E6F30AFFEEF322FFC1784FF1FDD
:10E58000130484841C40411189CF9C472302B500A9
:10E590002AC61CC1EFF05FFC1C409C4B99C332455E
:10E5A000829741016F30AFFBEF322FF94111444D9B
:10E5B000328532842EC6EFA00FF92AC42285EFA03F
:10E5C000EFF903A84400630C0800B24583574400E8
:10E5D0001840224683D54500AA8626850298410127
:10E5E0006F30EFF7EF326FF5404D1DC408C097054F
:10E5F00000009385E50213054401EF80901897779A
:10E60000FF1F9387677C9C43014589E79777FF1F2E
:10E6100023AC877A6F30AFF47D55EDBFEF32EFF169
:10E62000011168009305F00F02C602C802CA02CCAD
:10E6300002CEEFF07FF405616F306FF29777FF1F26
:10E64000938787789C43D847A1679D076311F7029A
:10E65000EF32AFEE01113285EFA0EFEE230AA100F9
:10E6600081456800EFF05FF105616F304FEF828008
:10E670009777FF1F938747759C43D847A167938778
:10E6800077036311F702EF324FEB01113285EFA0F0
:10E690008FEB230AA10081456800EFF0FFED0561D3
:10E6A0006F30EFEB82809777FF1F9387E7719C4372
:10E6B000D8479547631CF702EF322FE801113285E6
:10E6C0003284EFA04FE8230AA1002285EFA00FE9D2
:10E6D00083574400231BA10081453ECC1C406800A9
:10E6E0003ECEEFF07FE905616F306FE782809307E0
:10E6F00085FF89CF8327C5FF91CBDC4B81CBEF32E0
:10E70000CFE3032585FF82976F306FE58280EF327C
:10E71000CFE22A843285EFA00FE3BD4763EBA70069
:10E7200018449377F5000345B70041995D8DA30523
:10E73000A7006F30CFE2EF324FE001117C003ECAFC
:10E74000B70707003ECC7C003ECE5C4D8DCF2A84BF
:10E7500013858700AE84EF807004A1652A899D052A
:10E760004808EF80FFBD9305803EB345B9024808D5
:10E7700093F5F50FEFA0CFD2014781465008A6854B
:10E780002285EF807FDC05616F306FDDEF32EFDADD
:10E79000EFF07FFA6F30AFDCEF322FDA01117C003F
:10E7A000AE843ECAA165B70707002A843ECC48085C
:10E7B0007C00938575033ECEEF809FB81C444808CB
:10E7C00083C5B700BD89EFA0AFCD50080147814692
:10E7D000A6852285EF805FD705616F304FD8EF3275
:10E7E000CFD52A84AE84EFF09FF2A6852285EFF084
:10E7F000BFFA6F30CFD6EF324FD4EFF0FFF96F3062
:10E800000FD6EF328FD30329C501411163040902EA
:10E810002A843285B284EFA00FD32AC62685EFA0C2
:10E82000EFD3832749002A8691C7DC4781C7B245C9
:10E830002285829741016F308FD2EF320FD0444D45
:10E8400081CC2A843285EFA06FD1DC40AA8589C7AC
:10E850009C4799C3228582976F306FD0EF324FCC9F
:10E86000032AC501411163030A062E89AA8495452E
:10E8700032853284EF80DFAC85452285EFA0CFBDA5
:10E88000AA89CA852285EFA0EFC283274A009DC7C7
:10E89000DC438DC72285EFA0AFBA83274A00104022
:10E8A00083564400DC437115A307A100B2961307F9
:10E8B000F1004E86CA852685829701C5238009000E
:10E8C00031A08345F1002285EFA00FB941016F30DF
:10E8D0006FC8EF328FC665711C083EC2B707800152
:10E8E0003EC41C0832893EC62A84AE84EFF07FF114
:10E8F0004A85EFA0AFC68357A10089CFAA855000F3
:10E900002285EFF0BFF5014781465000A68522859C
:10E91000EF809FC359616F308FC4EF326FC0657154
:10E920001C088329C5013EC2B70780013EC41C08EC
:10E930002A84AE8432893EC6EFF03FF06384090238
:10E940004A85EFA0AFC18357A100AA8581CF5000AF
:10E950002285EFF0BFF0014781465000A685228551
:10E96000EF809FBE59616F30EFBEEF320FBD657112
:10E970001C083EC2B70780013EC42A841C083285A9
:10E980003EC6AE84EFA08FBD8357A10089CFAA8574
:10E9900050002285EFF09FEC014781465000A6858C
:10E9A0002285EF807FBA59616F306FBBEF32EFB8CD
:10E9B000444D91E88347450093B71700B307F040F3
:10E9C0003E856F30CFB91845FD577DDB97070000B6
:10E9D000938707032A845CCB97050000938565D154
:10E9E00013858400EF80E05980C0034744008147CD
:10E9F00061FB1777FF1F232B973CD9B7EF324FB23C
:10EA00008329C5014111032985008147638B0908CA
:10EA10000324090191452A8A2285EF807F9285454A
:10EA20002285EFA06FA38945AA8A2285EFA0CFA2F5
:10EA3000AA84EF809F9683A749002A8B9DC79C4399
:10EA40008DC72285EFA0CF9F83A74900A306A10011
:10EA50001040835644009C431307D100B296D685DC
:10EA60001306E1005285829709CD83570B0023805E
:10EA7000F400A183A380F40023800A00A306010010
:10EA800029A88357E10022852380F4008345D10023
:10EA9000A183A380F400EFA02F9C8347D100B3375C
:10EAA000F0000347B900920701453D9BD98FA305AC
:10EAB000F90041016F300FAAEF322FA841111DE973
:10EAC0009777FF1F93878730804305C80440130959
:10EAD00084009DC55C4099C79C4B89C726852EC67E
:10EAE0008297B2459307803EB385F5024A85EF8051
:10EAF000605521A0404DAA8479F841016F302FA6BE
:10EB00004A85EF80A0555C40EDDBDC4BFDD72685C8
:10EB10008297E5B7EF326FA22A843285EFA0AFA2C9
:10EB2000AA852285EFF05FF96F306FA3EF32EFA077
:10EB30002A84AE84EFF01FFEA6852285EFF0BFBFCA
:10EB40006F30EFA108413355B50005898280EF325F
:10EB5000CF9E1774FF1F130464291C5C0111231737
:10EB600001008D83858BA303F1008327040B2318F9
:10EB700001002319010003D7C7013ECA3C0023143A
:10EB8000E1007D572315E1000357C4023ECC02CEBD
:10EB90002316E100EF802FE38357E101231EA1003C
:10EBA00093F707E093E71710231FF1009777FF1FF4
:10EBB00083C7672685C305470145638AE700834706
:10EBC000840393E727001777FF1F230DF7240561C0
:10EBD0006F30EF98814717D700001307271C854631
:10EBE0001306710085454808EF70E04B6DF18347CF
:10EBF0008403F59B1777FF1F2306F72285471777B6
:10EC0000FF1F230AF720E1B7EF322F90977DFF1FF8
:10EC1000938DCD1D03A6CD0639712A898147814484
:10EC2000930600023357F600058B01C7850493F461
:10EC3000F40F8507E398D7FE83A70D0B2317010276
:10EC40002318010203D7C7013EDA3C102314E10266
:10EC50007D572315E10203D7CD023EDC23190102C3
:10EC60002316E10202DEEF800FD68357E103231E55
:10EC7000A102014593F707E093E71710231FF10264
:10EC80009777FF1F83C72719A9EF9777FF1F83C7C0
:10EC900077193EC69779FF1F938949150144014DA5
:10ECA0009D4A054B954B177CFF1F130C6C1B977CE3
:10ECB000FF1F938C6C1A03DAC90563090A00EA8501
:10ECC000631459036685EFF0FFE71DC1050DA147E9
:10ECD0008909E312FDFE2DE09777FF1F23A0071897
:10ECE000014521616F302F866285EFF0BFE579DD48
:10ECF0003247B3878400E3F0E7FE9C00130614005C
:10ED000006043E9413178A0093578A00D98FC207CE
:10ED1000C183A30EF4FCA183230FF4FC03A70D070A
:10ED2000B317AB01D98F1777FF1F2329F71263049D
:10ED30007601328461BF15449777FF1F83C7870D23
:10ED4000138717009776FF1F2386E60C931614008F
:10ED5000230EF10017D700001307470481478506EB
:10ED60007008CA854818EF700034E34705F68347FA
:10ED7000C10105451777FF1FA30EF7089777FF1FFF
:10ED8000238B2709B9BFEF22BFF90111AA892E846D
:10ED9000EFD0EF9C2A899774FF1F93842405639911
:10EDA000090A9C5C414793F707036393E70A1777C7
:10EDB000FF1F03479706894763ECE70883A7040B07
:10EDC000231701002318010003D7C7013ECA3C00E6
:10EDD0002314E1007D572315E10003D7C4023ECC84
:10EDE000231901002316E10002CEEF80CFBD231EC0
:10EDF000A100EFC06FCD8357C101230FA100914641
:10EE000013D78700A207D98F2312F1009777FF1F2E
:10EE100083D7670113D78700A207D98F2313F10087
:10EE200017D70000130707F781475000954548089A
:10EE3000EF70602705889317240003C484036D983E
:10EE40005D8C9777FF1F238F87FC05616F209FF0F4
:10EE5000EF70B0781775FF1F130545FDEF80002098
:10EE600083A7040B9775FF1F83D505FB03D5C70147
:10EE7000EF10E0279777FF1F83C7C7FA93F60702C3
:10EE8000014789E61777FF1F035707F99776FF1F9A
:10EE9000239CE6F81777FF1F130707F4184309CBE5
:10EEA000C18B99C789451775FF1F0355E5F6029772
:10EEB0009777FF1F23A207F69777FF1F238D07F48D
:10EEC0009777FF1F23AA07F89777FF1F23A807F854
:10EED0009777FF1F23A607F883D7840393F7270CA0
:10EEE00093E717001777FF1F231EF7F283572903B5
:10EEF000A18B99C3EF70E03F11C49777FF1F23A93F
:10EF000007F0A1B78D471777FF1F2323F7F0EF9086
:10EF10002FA59305803EB305B5021775FF1F130596
:10EF2000E5F0EF80201215B79777FF1F938707EC66
:10EF3000D85325C791C99777FF1F238E07EC977782
:10EF4000FF1F23AD07F08280EF223FDF83C7F70268
:10EF500041112EC685071777FF1FA300F7EC97779F
:10EF6000FF1F2394A7EC9D471777FF1F2322F7EA83
:10EF7000EF900F9E2A84EF90AF9DB24501E5EF9090
:10EF80002F9DAA85B305B4401775FF1F130505EA29
:10EF9000EF80400B41016F209FDC82809777FF1F3D
:10EFA0009387C7E4D85331C7EF223FD903C7F7028D
:10EFB00005079776FF1FA382E6E611CD8C5F0D470C
:10EFC0000145898185899776FF1F23A3E6E4EFF049
:10EFD0009FDB6F20DFD885479305C0441775FF1F5F
:10EFE0001305C5E41777FF1F2324F7E2EF808005A0
:10EFF000CDB78280EF227FD41777FF1F0347A7E1A9
:10F000008547631EF7009777FF1F938727DE83C727
:10F01000870393C787001777FF1F2305F7E017754E
:10F02000FF1F1305A5E0EF806003EF807FEF994796
:10F030001777FF1F232EF7DC9777FF1FA38F07DCBF
:10F040009777FF1F238907DCEF90AF8F9307400668
:10F050003305F5029777FF1F23A2A7DC6F203FD06F
:10F060009777FF1F83C707DCC18B99C7EF22FFCCBF
:10F07000EFF0FFAD6F20BFCE695582809777FF1FFD
:10F080009387C7D6DC5381CBEF223FCB8545EFF08A
:10F090009FCF6F20DFCC82801777FF1F130707D524
:10F0A00001468146BA852148631E06019DCA239008
:10F0B000A60083C7850393E717001777FF1F230375
:10F0C000F7D605A08357C705631DF502F859854794
:10F0D000B397C70093C7F7FFF98F1777FF1F232157
:10F0E000F7D89C5D9183858B85C79777FF1F83C772
:10F0F00087D299EFEF227FC41D45EFF0FFB06F205C
:10F100001FC681E699E39306C7050506090769BF8F
:10F110008280EF221FC08605AA84B309B500977AC2
:10F12000FF1F938A6AD3054B977BFF1F938B0BD3EB
:10F13000214C639434039777FF1F938727CB9C5F01
:10F140009183858B89CB9777FF1F83C7C7CC81E7D6
:10F150002145EFF07FAB6F205FBF03DA0400630B44
:10F160000A041779FF1F130969C80144CA8C835721
:10F17000C905639D4703A2855685EFF0BF9C11E545
:10F18000A2855E85EFF01F9C05C903A74C07B31746
:10F190008B00D98F1777FF1F2324F7CC83C78C03ED
:10F1A00093E717001777FF1F230EF7C60504090919
:10F1B000E31F84FB8904B5BF231E0904C5BF17776D
:10F1C000FF1F034747C58547631AF700EF22FFB6C5
:10F1D000EFF05FE2EFF0BF976F207FB8828081474A
:10F1E00085451306000293861700B397F500E98F53
:10F1F00013F7F60F89E7B687E397C6FE01473A850E
:10F200008280FD4785457D56B396F500138717002C
:10F21000E98E1377F70F89E6FD17E397C7FE0147DD
:10F220003A85828089E901473A85828001473A859B
:10F2300041016F20DFB2EF225FB041112AC62E8557
:10F240002EC4EFF0DFF9A2457D158547B397A700DF
:10F25000E39EF5FC32469377360099C3719A110606
:10F260009777FF1F938747B894433E871778FF1F10
:10F270001308C8B689EA832708009107F19B97769F
:10F28000FF1F23A3F6B6032588001843B307A70082
:10F29000B3F7B702B387F540FD15FD8D832748000E
:10F2A000AA95B306B600E3F3F6F8E371D5F82E9706
:10F2B0009777FF1F23A8D7B23DDB3A858145EF2022
:10F2C000DFAA2A87ADB718419777FF1F938707B149
:10F2D00023A4070098C35841D8C39777FF1F23A5DD
:10F2E00007B08280EF22DFA3AA8401441779FF1FB1
:10F2F0001309C9AF9309400EEF807FD56345A40081
:10F3000001456F203FA5330534038327090B3E9544
:10F310008357C501E38797FE0504F9BFEF227F9F5E
:10F320009779FF1F938989AC3E84BA84834706008E
:10F3300003A7090041119D83058B3D8F83C74401BD
:10F34000AE8A2A89F99BD98F238AF4001C44B6859A
:10F35000231204001CC02285328A36C6EF90DF8F4C
:10F36000B246D2853686EF90900BDC4883A5090023
:10F370000840858B56869D8DEFD03FCC61E91840C3
:10F380007D558347570003476700A207D98FC207FF
:10F39000C1872394F4006358F00A83C7440193F7AC
:10F3A0000703B5CBD0489377160003A609001D8E3E
:10F3B0009777FF1F938747DA9C43ADEB814641A0C7
:10F3C00003A70B0093172A00BA971840944383476A
:10F3D00057008345670033F65601A207CD8F6311AE
:10F3E000F602834737000346470003472700A2077A
:10F3F000D18F4207D98FBD82B3F76701638AF604C4
:10F40000050AEF80DFC3420593170A014181C183DA
:10F41000E3E8A7FA41BFA16A370B0200014A977BD4
:10F42000FF1F938B6BAAFD1A7D1BE1BF83C74401AD
:10F4300013070003854693F70703E391E7F8A285D6
:10F440004A85EFD0FFCF41016F203F906155E5BF66
:10F450007955D5BFEF22DF8C9774FF1F93844481C9
:10F460009C40D9EF9777FF1F9387C7969C4363997A
:10F47000070CEF80DFBE930780023305F502894554
:10F48000EFF05FDA41C99777FF1F23A7A7A0EF80AE
:10F490001FBC9307400E3305F5029145EFF09FD84E
:10F4A00035C99777FF1F23ABA79EEF805FB201CDD1
:10F4B000EF80FFB191450E05EFF0DFD621CD9777B4
:10F4C000FF1F23AFA79CEF801FCB11CDEF80BFCADA
:10F4D000D9473305F5028945EFF0DFD405CD97779D
:10F4E000FF1F23A9A79AEF809FB591450A05EFF06A
:10F4F0007FD30DC19777FF1F23A8A79C014521A8A3
:10F50000EF803FC2930780063305F5029145EFF087
:10F510007FD101E565556F20FF839777FF1F23A7F4
:10F52000A78E0144130A80061779FF1F1309098C5F
:10F53000B14AEF801FBF6364A4029C40E38407F2DA
:10F54000EF803FBE9307A0043305F5028945EFF035
:10F550007FCD69D19777FF1F23ACA79619BFEF80A6
:10F560005FBB89450605EFF0FFCB4DD5B3094403DA
:10F57000032709024E9708CBEF80BFB83305550328
:10F580009145EFF03FCA59D583270902050413744A
:10F59000F40FCE9788DB71BF9777FF1F938707859E
:10F5A000884705898280C167FD176319F500977741
:10F5B000FF1F9387A78303A5070B8280EF22EFF736
:10F5C000EFF05FD26F20AFF9814709C58347E501AE
:10F5D000B337F0001777FF1F1307478118470983D8
:10F5E000058B19C393E727003E858280EF22EFF455
:10F5F0002A84EFF07FFD8347E401AA851305940870
:10F6000099E3130504039766FF1F9386267E9442B1
:10F61000130615021307840213059504EFD0CFC01B
:10F620006F20EFF3EF22CFEF9764FF1F9384047CEA
:10F6300098442A892E840983058B9C4019C763143A
:10F64000F5006380050E014401A2E3FEA7FE1387C7
:10F65000A702E36AA7FE850763FCA70883A9440BFA
:10F66000EF80FF961316350081454E85EF20EFEFB2
:10F670009767FF1F23AC27779767FF1F23AA07769B
:10F6800049CC9C4493E747001767FF1F2324F77674
:10F690009767FF1F2388077C630F040C9767FF1F82
:10F6A00023A6277501440549EF807F926341A40A90
:10F6B000EF80FF9493050006B3C5A502B7F73600A7
:10F6C000938707E81765FF1F1305057A4169014411
:10F6D0009309400E7D19B385F502EF70B016EF80E7
:10F6E0001F97634FA4080145EF3040700544A9A857
:10F6F0006398A7029DE583A9440BEF805F8D1316E5
:10F70000350081454E85EF204FE69767FF1F23AFF9
:10F71000276D9767FF1F23AD076C9C44ED9BADB72A
:10F7200085C51767FF1F0347E7739307F005E3FCE1
:10F73000E7F021F8EF60F03C6DD19C4493E70702BD
:10F740001767FF1F2328F76A22856F20AFE083A782
:10F75000440B131534003E958357050081CB834736
:10F76000250099C721468145EF202FE005042DBFD4
:10F7700023012501E5BF9767FF1F23AB07660DBF78
:10F780003305340383A7040B3E958357C501638477
:10F790002701EFF0BFE5050499B7EF220FDAEF80FC
:10F7A0001F86130400063345A4029764FF1F938449
:10F7B000E46383C784073E951375F50F9767FF1FB2
:10F7C0002382A76A9307F00563E7A7020545EF3098
:10F7D000E061EF80DF823345A402B7F53600938500
:10F7E00005E8B305B5021765FF1F1305E567EF7060
:10F7F00070056F20CFD69C4405458983858B81CBCE
:10F80000EF904F8888408145EFF0DFE1DDB7EF30C2
:10F81000E05DC5B7EF22CFD0130495082A891306FF
:10F820009005A28513050503EF90603F1306900530
:10F8300081452285EF206FD34A85EF30C054814443
:10F84000176AFF1F130A8A5A930A8002EF803F81CA
:10F8500063C4A4006F200FD0338454038327CA0AE3
:10F860003E94035704008357C9016317F702834787
:10F8700044009DC3930964014546CE851305540099
:10F88000EF90E039454681454E85EF200FCE228529
:10F8900023020400EF30005785044DBFEF22EFC96B
:10F8A0009767FF1F9387C73C9C432A8491C70DC568
:10F8B0000355C501EFE00FC29777FF1F9387C789F4
:10F8C0009C4389CBEFB0DFD085476315F5002285D7
:10F8D000EF50C05D6F20AFC841657D15E1BFEF22DD
:10F8E000CFC51764FF1F130464504440938714006E
:10F8F0001767FF1F232EF74EEF30605E1C4489838D
:10F90000858B9DE75840B7E7B0009387075063F1B8
:10F91000E7020145EFF01F9D01CD0545EF809FF601
:10F92000084085450505EFF0FFCF0145EFF01FF7D3
:10F9300026856F20CFC2EF22AFBEA1642A89014481
:10F940009769FF1F93894958FD14338AA500EF80FA
:10F950000FEF6344A4006F20EFBF03A709009317C4
:10F960002400BA979843658F42074183634C27016F
:10F97000635A470123800700A38007002381070003
:10F98000A38107000504E1B7EF222FB88359450092
:10F99000C547411163F537310441C1E53385340171
:10F9A000834785FF034795FF0348B5FFA207D98F1B
:10F9B0000347A5FFC207220733670701D98F034713
:10F9C000C5FF0348D5FF2207336707010348E5FF5A
:10F9D0000345F5FF420722083365A800498FB98F18
:10F9E0001767FF1F1307074C1768FF1F1308884D81
:10F9F0003A85832807006384172B1107E31B07FF51
:10FA00001767FF1F1307074C184313182700429569
:10FA10001CC10507A1473367F7029767FF1F23A3A0
:10FA2000E74A93F735001397470083474601C16BB8
:10FA3000368993F7F7FCD98F32842E8A230AF60091
:10FA4000814A176CFF1F130C6C3AFD1B976CFF1F4C
:10FA5000938C0C22176DFF1F130D8D47EF802FDF46
:10FA600063C7AA00E154268541016F20CFAD13087A
:10FA7000400EB3870A0303280C0BB30DF800638E06
:10FA80000D2083D7CD01638A772183A70C00014B1A
:10FA9000639707169767FF1F9387C7339C4363904D
:10FAA000071683C7040003C70D0493F7F707631B0A
:10FAB000F71ACA872287CE86268693859D061385E8
:10FAC0001D04EFF0BF85631F051883D7CD01032701
:10FAD00009002320B4012312F400FD572313F4007E
:10FAE0008347170093F6F7078347D40093F707F887
:10FAF000D58FA306F40093F7F707B337F000B307E9
:10FB0000F0402307F400834717009D839396370046
:10FB100083474401DD9BD58F230AF40083473700D8
:10FB200083464700A207D58F83462700C206D58F9C
:10FB30001CC88347770003478700A207D98F231586
:10FB4000F4000D476304EA00BD5491DF938707106A
:10FB5000C207C1831307B00FBD54E376F7F0EF80FF
:10FB60000FC98144E31105F09766FF1F83C606366F
:10FB7000938716001767FF1F230AF7341767FF1FC5
:10FB800013078734231BD40093972600144303578D
:10FB90008400E175BE96A1671386F7FFB377C700AF
:10FBA00098426D8FD98F9CC21848F18F3E07D98F2C
:10FBB0009CC2EF80CFC89767FF1F83C7273133F5FB
:10FBC000A7029767FF1F2383A73071BD9307A00487
:10FBD000B308FB0283270D00BE9803D7080083D724
:10FBE000CD01631DF70083C7040003C7880093F7A6
:10FBF000F707630BF70083C7FD019DEB050BEF8053
:10FC00004FD2E345ABFC71BD9385980113859800F5
:10FC1000CA872287CE86268646C6EFF02FF0B248E6
:10FC200079F98347440193E74700230AF40071BD43
:10FC300083C7040003C7980293F7F707E310F7FCA4
:10FC4000CA872287CE8626869385A8031385A802B5
:10FC5000EFF0CFEC45F58347440193E72700230AF3
:10FC6000F400C1B783C7FD018DCB83C7040003C770
:10FC70009D0993F7F7076312F702CA872287CE869A
:10FC8000268693852D0C1385AD09EFF02FE911E53C
:10FC90008347440193E7270049BF850AC1B3FD5458
:10FCA000D9B3EF220F87797183544500AA8B2E8434
:10FCB000B28AEF80CFBB590563499504B7E40400CD
:10FCC00003A90407EF80AFBA5905420541810299A3
:10FCD0002A8905CD2AC623180100EF804FB959059E
:10FCE0002319A1006146814528089769FF1F938960
:10FCF000E90F4ACAEF206F872302810203A489001B
:10FD0000058819E4BC544A85829745616F20EF83CA
:10FD100074003008D6855E85EFF01FC765F5680072
:10FD2000EF807FF1176AFF1F130A0A4383270A0037
:10FD3000AA84035B010189CB89476397FA00835545
:10FD400001025E85EF50203003552102EF704FC84D
:10FD500019E503552102EF708FD43334A0009317B7
:10FD600064000344C1022C0868001374F4FB5D8C2A
:10FD700023068102EF60B056E9576314F5028356FB
:10FD8000E1029767FF1F938727149C431397260070
:10FD90006176BA979843718F98C39767FF1F23873F
:10FDA000D712831721026345F00085476396FA0056
:10FDB000B25793F7070C95E7D247C2040347C10235
:10FDC000C180BE9426C62318610113770703C1477B
:10FDD000631DF70083475102054793F7F7076390C8
:10FDE000E704B7E70400BC5739BF92570544A18325
:10FDF00093F7F707E377F4FE15C78347C1021307AC
:10FE0000000293F707036397E700EFB06FFC8547A5
:10FE1000E319F5FC8347C10293F7070389CFEFB0DD
:10FE2000AFCA21A8EFB08FD7E30985FCEFB04FFA36
:10FE3000E31985FAD9B7EFB0EFD8AA850146054591
:10FE4000EF707FF82A8451DD8347C102414793F761
:10FE500007036384E70232478347170093F707F8E5
:10FE6000A300F7003247925783461700A18393F708
:10FE7000F707FD17D58FA300F70003560101B24520
:10FE8000130BC4005A85EF80DFDFE24A13069005AA
:10FE90008347C10283C4EA01918BB384C4021385F2
:10FEA0001404569595C35444B3879A0083C7070436
:10FEB00003C70600137707F82380E60058448346FB
:10FEC0000700D58F2300F700B25703A6090081462B
:10FED000858B1D8EDA85EFD0EF9B15E9B25783A590
:10FEE0000900484413869406858B56969D8DEFD065
:10FEF000CF9411ED83270A0099EFB25705479183FC
:10FF00008D8B6387E7049DCF09476389E7042285CA
:10FF1000EF80DFF8F9B5EFB0AFEB85476309F50087
:10FF20008347C102414793F70703E398E7FC8355F2
:10FF300021025A85EF40907C69D183172102E35E4C
:10FF4000F0FAF1B7EFB08FC57D151335150061D10B
:10FF5000014681452285EF70FFEF55BFEFB04FE7B7
:10FF6000E5B7EF129FDD9764FF1F9384A4E9268510
:10FF7000EF809FEB2A8419E16F107FDE1305C40028
:10FF800005468145EFF0FFD12285EF803FF1C5B7EF
:10FF9000EF12BFDA4111AE842A8493079503130749
:10FFA00015019306F10005466C0026852306010025
:10FFB000EFD0CFBE1DEDA68541462285EF803046AD
:10FFC0008347F1009305140226852308F400EFD03F
:10FFD0006FC805E19767FF1F938707189C4389EF58
:10FFE0001306940497C500009385C5DB2685EFD0E2
:10FFF0008FD441016F10BFD61306940297C500003D
:020000040001F9
:100000009385C5DA2685EFD00FD379D9DDB7EF1206
:100010003FD19767FF1F938727EB8043AE84B28958
:10002000368AAA8AEF80AF81131625008145228582
:10003000EF10BFD39767FF1F238A07E89767FF1F5B
:100040009387C7DA03A4070B13F714003E89230F25
:10005000E400CE8525C713059408EFF07FF301C5B2
:1000600055556F103FCF8947A30FF4009767FF1FC7
:100070009387870E9C4303278900858093B71700D9
:1000800086072300F402231E54019767FF1F23AF46
:1000900047D585889377B7FF99C09367470017675F
:1000A000FF1F2329F7D42285930700061767FF1F38
:1000B000230AF7DAEFF08FD3014565B71305040380
:1000C000EFF01FED45D569BFEF123FC7FD57231075
:1000D000F500231105002312050023130500130664
:1000E000200481452105EF105FC86F105FC7EF1234
:1000F0003FC34111AA8401441769FF1F130949DD59
:100100009309A0042EC6EF80CF81B2456344A400BA
:1001100061550DA033053403832709003E958357AD
:100120002500639CB7008357050063989700EFF0A4
:10013000BFF9014541016F10FFC10504E1B7EF129E
:100140003FBE9767FF1F9387E7C89C434111AA846E
:100150002E84B28903592500C1C39767FF1F83D737
:10016000A7CB639B2707EF700F862A8903D524004E
:1001700093051002B305B40285472302F10093579B
:100180008900A302F10093578500A303F10083D7F0
:1001900044002304A100254613D787002305F1005E
:1001A00083D76400A304E1004E8513D78700A3051D
:1001B000E1002306F1001387950093879501A105BF
:1001C000B386B400A6974C00269723032101EFD0F5
:1001D000EF9C41016F101FB8EF60FFFE51BFEF129F
:1001E0003FB44111AA8401441769FF1F130949CE86
:1001F0009309A0043AC636C432C22EC0EF707FF213
:1002000082451246A24632476344A400615599A034
:10021000B307340303250900AA9703D8070003D5C1
:10022000C4016310A80495E91DEE91CA03C6E40158
:10023000930510023306B60225063E9690C201458C
:1002400011CB83C6E40113061002B386C602E5068D
:10025000B6971CC341016F10FFAF03D52700E3051C
:10026000B5FC050441BF83C5E40113051002B38545
:10027000A502BE9583C585002300B6007DB7EF12A9
:100280003FAA5C4141112A8403DA2700C167FD17A8
:10029000AE843289630CFA002685EF807F9A8D4701
:1002A00063EDA7007D5541016F10DFAA2E85EF8019
:1002B0003F999D47E3E2A7FEF5B75C40268583D5CD
:1002C0004700EF809F90835584002685EF80FF8F45
:1002D0008D452685EF803F8EAA89EFF04FE093573A
:1002E00005012380F90093578500A380F90023813D
:1002F000A9005840C167FD178345A7006314FA00A1
:1003000093E505082685EF801F8F9767FF1F93876A
:1003100067AC9C430840D9CF8347B400858BD9CBC9
:1003200078003400130671008145EFF05FEB1DC9C2
:100330008347B400184093069005F99BA305F40089
:100340008347E701B387D702B306F70083C60604E5
:10035000A303D1009386170493879706BA96BA979A
:1003600036C43EC61764FF1F130444A81C440C4047
:1003700026858983858B9D8D834771009E05DD8D44
:1003800093F5F50FEF803F871C4410402245898389
:10039000858BCA861D8EA685EFC0DFCFE31505F0DD
:1003A0001C440C40324689838840858B9D8DEFC06C
:1003B000DFC8D5BD8347B40013079005F99BA3059B
:1003C000F4008347E501B387E7023307F5000347ED
:1003D0000704A303E10013871704938797062A975E
:1003E0003E953AC42AC6BDBFEF129F93032A45002B
:1003F0009307F00FAA840347AA00AE893284368996
:100400006316F700EFB06FAB2305AA00938AC9000B
:100410000146D6852685EFF09FE62A8A21E51767F3
:10042000FF1F130767D31843DC4039C383C6A700F7
:100430000547638FE60283D547005685EF40102CB1
:1004400005C9DC40839747006354F00201CC1C408F
:1004500089C74A868145014582975C4081C7CA8524
:10046000014582974E85EF807FA352856F109F8E46
:10047000DC4003D54700EF60BFD501E9DC4003D580
:100480004700EF60DFE181471DCD19C41C4089C7DB
:100490004A868145014582974E85EF807F9FAA85D8
:1004A0001765FF1F13050596EF80DF9511C45C40AB
:1004B00081C7CA85014582971765FF1F1305C5933C
:1004C000EF60F0368547D84085460346A700E30B2A
:1004D000D6F8031747006353E000C9F74A86A285A0
:1004E0004E85EF703F97BDBFEF129F83AA840144F2
:1004F0001769FF1F1309C99D9309A004130A9508E2
:10050000EF703FC26344A400014535A033053403B6
:10051000832709003E958357250099E30504CDB74D
:100520000357050083D7C401E31AF7FE52868545B9
:10053000EFF0FFC065D56F10FF81EF126FFEAA8448
:1005400001441769FF1F1309A9989309A004EF70CC
:100550005FBD6344A4006F10EFFF330534038327AE
:1005600009003E958357250081CF83570500639985
:10057000970093059502130610022105EF80206A6B
:100580000504F1B7EF126FFB0347E5012A848347A7
:10059000F5016307B70089E781452E856F102FFCB1
:1005A000230FB400054781C9E398E7FE8947A30FED
:1005B000F4008545DDB7638BE7020947E39FE7FC5D
:1005C0002285EFF02FA59767FF1F9387A7809C4395
:1005D00099E79757FF1F9387A7699C4389C70355DE
:1005E000C401EFF09FF5A30F0400E1B755D6C9BFD2
:1005F000EF120FF3EFA0FFEE85476312F508EF80CF
:10060000EFCC1764FF1F130424B51C4081CBEFA06F
:100610003FFC89476304F5001C4082979757FF1FF2
:100620009387477B9C43B9CF82979757FF1F938748
:1006300027649C4391C382971754FF1F1304047BC4
:100640008327040B83D4C701EF60FFB78327040B14
:10065000AA85144003C6E7011C448983858B99C38E
:100660001366260026854169EF40C03D8144D94983
:100670007D19EF705FB063CAA4006F10AFEDEF801B
:100680000FCA41B7EF705F884DB7B38734030327B4
:10069000840ABA9703D527006308250103C64701DA
:1006A00083D50700EF40A03B8504E1B7EF124FE789
:1006B00001449754FF1F938464731309400EFD593E
:1006C000EF70FF98634FA40401449754FF1F938475
:1006D000E47113098002FD59EF707F98634CA40404
:1006E00001449754FF1F938464705949FD59EF707A
:1006F0009FA8634AA40497F5FFFF9385450A175501
:10070000FF1F13056576EF60D007970500009385FE
:1007100085851755FF1F1305256EEF6050056F1077
:100720006FE33307240383A7040B0504BA97239EC2
:10073000370179B73307240383A7C40A0504BA979E
:100740002390370151BF3307240383A7840A05048C
:10075000BA972391370161BFD4410387350085479C
:100760003356F5026377E600A54899E72380060033
:100770008280B387E702EDB73358F502038735006F
:100780003375F502B3D7E7021307000363DA0801F4
:1007900003C6050013077003118A19E213077005D9
:1007A00085064297A38FE6FEC9B718451C416376BC
:1007B000F7005C41BA972380B7001C4585071CC52C
:1007C0008280EF128FD74111AA872E85B285368697
:1007D00036C6829763480500B246158D3335A000B2
:1007E0003305A04041016F108FD7EF126FD3056919
:1007F00041112A8A2320060001448149975AFF1F8C
:10080000938A8A6F056B7D1932C62EC4EF703F85BF
:10081000AA84EF70DF832695A24532466346A40082
:100820004E8541016F100FD303A70A0093171400E0
:10083000BA9703D707003377670101E71CC20504A5
:10084000E1B703D707009356D700858AE39946FF9F
:1008500033772701E315B7FEBE89D5B7EF12EFCD89
:1008600001112EC6B2843689EFB02FEE2A8461556D
:1008700001C8B24589E9232E040023200402014562
:1008800005616F10CFCDA1463008CA852685EFF0EF
:100890005FF37DF5835781010357A101231EF40007
:1008A0008357C1012310E4022311F4028357E101AD
:1008B000D207D1832312F4028357E1011397370142
:1008C00063560700FD57231FF4005DBF231F04007C
:1008D00045BFEF12EFC41754FF1F130424518327A1
:1008E000040B03D7C701C167FD17630EF7109767A5
:1008F000FF1F9387A7869C4381C70545EF4060771C
:10090000C1690149930A400EFD19176BFF1F130BB4
:10091000AB84EF70CFF3634BA90E1757FF1F03474C
:1009200067549307F00563E4E702EF704FED93051A
:100930000006B3C5A502B7F73600938707E8175539
:10094000FF1F13056552B385F502EF60A06F814567
:100950001705000013058520EF60DFF8EFB0EFDE2C
:1009600001CD0357C50109CB0357E50111C78347E3
:10097000050299C3EF60A06BEFB06FDE31C517576A
:10098000FF1F0347E75A9757FF1F9387675A0DCFFB
:1009900003C717002304E50003C72700A304E500ED
:1009A00003C737002305E50003C74700A305E5009B
:1009B00003C757002306E50003C7670083C7770016
:1009C000A306E5002307F5001C4493E7170017571B
:1009D000FF1F2321F7425C4085E7EF708FEF0DC1C9
:1009E000EF702FEF44402A89EF70AFEE33F5A40289
:1009F0005C40FD17CA97898F1757FF1F232AF73EC0
:100A00000145EF70DF9F01456F10CFB4B304590368
:100A10008327040BBE9483D7C40163883703138AEA
:100A20000403D2855285EFF0AFD605E183C7F40108
:100A300099CF938594082E85EFF08FD509C91306B9
:100A4000900581455285EF104FB20509D9B583272E
:100A50000B00268593B7170086072380F402EFE08A
:100A6000FFB8E5B7854763F8A7009307F5FFBE9584
:100A70003305A040E98D2E8582809841C167BA97E1
:100A800013D707016304A7009CC182804207998F96
:100A9000E5BFEF128FAA41112EC63284B684EFB0A3
:100AA0000FCCE15701C9B24591E99757FF1F238148
:100AB000074881473E8541016F106FAA9D46175632
:100AC000FF1F1306F646A6852285EFF09FCFAA8763
:100AD00075F105479756FF1F238CE644E1BFEF12DF
:100AE0002FA4411191E99757FF1F23A30730014419
:100AF000228541016F100FA6B68532858D467000A4
:100B0000EFF03FCC2A846DF58347D1000347E10025
:100B10001759FF1F1309892DA2074207D98F0347D1
:100B2000C100D98F1757FF1F2324F72CEF706FDAFE
:100B300061D1EF700FDA83244900AA89EF706FD971
:100B400033F5A40283274900FD17CE97898F1757E5
:100B5000FF1F232FF72869BFEF122F9E1C45AA8481
:100B600091CFD84B01CF83D7470089CBEF601F923D
:100B7000AA8509C588446105EF60C04C9757FF1FDF
:100B8000938747259C43014489EF6F104F9D9C48F4
:100B900013171400BA9703D5070019C1EFE0CFCFA0
:100BA0000504EF70CFC7E344A4FEC5B7EF12EF987A
:100BB000011185E9EF605FDA01449757FF1F23A316
:100BC000072C9757FF1F23A1072C9757FF1F23AF11
:100BD000072A9757FF1F23AD072A228505616F104B
:100BE0000F98B6873285C9467000BE85EFF07FBD8D
:100BF0002A8465F541469305E1001755FF1F13054B
:100C00006528EF80C0010355C100EF608FD7F1B7B1
:100C10008DE19757FF1F23AB071C9757FF1F938743
:100C2000E71C9C470145ED9B1757FF1F2324F71C2A
:100C30008280EF128F904111B68532859546300043
:100C4000EFF03FB815EDA2471757FF1F2320F71A03
:100C50009757FF1F938787199447B24713F7B6FF3B
:100C600013F6170019C213E74600858393F7F707B9
:100C70009756FF1F23A0E6181757FF1F2304F71EE0
:100C800041016F10CF8DEF12AF8903841500DC4155
:100C90002A89AE8485070387F7FF19C36340800C58
:100CA0008387240091C7635580007D1462046184AA
:100CB0009C40370700FF0907F98F37070010090725
:100CC0006392E70A6355800079146204618483C7E4
:100CD0000400858B95E39379F40F4E8A93178A016C
:100CE000E187634AF008A287635304008147338495
:100CF000F9407D14620461848385240081C54A859E
:100D0000EFF0BFAA9C40370700FF0907F98F3707AC
:100D100000100907639AE706930500034A85EFF080
:100D2000DFA883C7040093058005918B99E39305A1
:100D300080074A85EFF07FA783C70400858B81CBAE
:100D40001374F40F93178401E1876347F004C040E4
:100D500005048305F4FFA1E96F00DFFF7D14620441
:100D600061840DBF370700080907E392E7F6E350F7
:100D700080F67D1499BF930500024A857D1AEFF035
:100D8000DFA2137AFA0F99BF370700080907E39526
:100D9000E7FA9305000371BF930500034A85EFF05E
:100DA000DFA07D1471BF4A85EFF03FA055B7EF0279
:100DB000DFF8EF70CFAA2A84EF706FA922958945DA
:100DC0000605EFE02FC6E55711C59757FF1F23A56E
:100DD000A71281473E856F009FF8930700026306C4
:100DE000F5005D1513355500828005458280EF02C0
:100DF0003FF34111AA892A89130419008304F4FFDF
:100E000032C62EC42685EFF05FFDA245324659E179
:100E10009307D0026392F408830404000548130486
:100E200029009377F6FEC9E793070003639FF40E4A
:100E3000830704001307800593F7F7FD6399E7061E
:100E40008304140041460904B706008063140800B7
:100E500093C6F6FFB3FEC6028147254F654EFD5F80
:100E600033D3C602138704FD6368EF06BA8463D5E3
:100E7000C408630DF5017D55636AF3006394670050
:100E800063C69E000545B307F602A69705048304D2
:100E9000F4FFC9BF22898DB79307B0020148E392DE
:100EA000F4F8830404002A88130429009DBF01CAB2
:100EB0008947E31BF6F893070003E397F4F88307E9
:100EC00004001307200493F7F7FD639BE7048304F2
:100ED0001400094609048DBF13E704021307F7F94C
:100EE000636CEE009388F4FB1307700363741E01B8
:100EF00013077005998CA5BF7D576300E502630455
:100F00000800B307F04091C519C19309F4FF23A06D
:100F100035013E8541016F00FFE3B687FDF5D5BF82
:100F20009304000315F2214605B719FE294629BF8F
:100F3000EF021FDF011161540DC53284AE894146B5
:100F400081453689EFF0BFEA93140501C180639EA5
:100F500009002685EF30102B014401C58145EF20A3
:100F60005016228505616F00FFDE2285CD46700098
:100F7000CA85EFF01F852A846DF52685EF3090280D
:100F800009E90356C1008345E1012685EF20500B96
:100F900001C941469305E1001105EF705048D1B7F2
:100FA0005D54C1B7EF02DFD70111E15401CDB28426
:100FB000AE89414681453689EFF07FE32A84639705
:100FC00009008144268505616F00DFD82685D1465A
:100FD0007000CA85EFF0EFFEAA846DF58357C1005B
:100FE000EDD3EF700F8E4205931704014181C18349
:100FF00063F9A702EFB08FB64204E14741803304A2
:10100000F40241460C082A9413054400EF70304165
:101010008357E1002311F4008357C1002310F4002B
:1010200055B7E55445B7EF02BFCF7971E15415C507
:101030003284AE8941468145B684EFF05FDB1319F7
:10104000050113590901639E09004A85EF401065A7
:10105000814401C58145EFB02FB1268545616F0000
:101060007FCFA6859306300270002285EFF06FF5E2
:10107000AA8465F54A85EF4070622A8411E54A85A5
:10108000EFB04F8C2A8431C58357C100231124014E
:10109000930964002310F4008347E1009305F100F5
:1010A00041462302F4004E85EF7070371309740136
:1010B00041469305F1014A85EF707036930554005F
:1010C0004E85EFC04FBF930564014A85EFC0AFBEA8
:1010D00069B7DD5459B7EF02BFC4797111E5E15426
:1010E000268545616F001FC7B284AE8941468145A0
:1010F0003689EFF0DFCF131A0501135A0A01528522
:10110000EFE06FCA2A846398090071D98145EFB076
:101110002FB48144F1B72685930610027000CA856A
:10112000EFF02FEAAA844DFD31C8B2479305D100F4
:101130004146858B230FF400B247130504038583D2
:1011400093F7F707A30FF400EF70702D4146930556
:10115000D10113059408EF70902C59B7330469033B
:1011600083A70A0B3E948357C401638337030509A1
:10117000EF60FFEDE344A9FEDD549DB7C16901496D
:10118000975AFF1F938A8AC6130B400EFD19CDB7DD
:10119000231E440159BF49CDEF029FB84111B289C6
:1011A000AE8441468145368AEFF07FC4931A05012B
:1011B00093DA0A010149175BFF1F130B2BC3EF6082
:1011C0001FE1634AA9000145ADCC81441759FF1FB7
:1011D0001309C9C181A883274B0B131439003E940E
:1011E00083570400638857050509D1BF8327490B3E
:1011F000139434003E948357040085E72310540170
:1012000091467000D2854E85EFF0AFDB1DE9B24705
:1012100013978700E1832183858B58C02301F40055
:101220000DA08504EF60BFDAE3C2A4FC5D5511A8F0
:1012300061558280F1F4214681452285EF00FFB29D
:10124000014541016F001FB11971D2C4130AC106D3
:1012500086CEA2CCA6CACAC8CEC6D6C2B6D6BAD880
:10126000BEDAC2DCC6DE52C463810524FD151C1043
:101270002ACC2ECA02CE3EC89304B0021549A94911
:1012800083050600130416009DE1F2465247E2472B
:1012900063FBE620B697238007007245F64066445C
:1012A000D6444649B649264A964A09618280930740
:1012B00050026386F5004808EFF02FCFF5A883575A
:1012C000C10023070100014593F7C70F2316F10062
:1012D000814501480147014681469308D002130326
:1012E0000003130E300205048307F4FF99C7638CD3
:1012F000970463C3F404638BC70501CA0346C100A6
:10130000858A799AD18E2306D10063090800834625
:10131000C100098BF59A558F2306E10019C12307F7
:10132000B100138707FD1377F70FA54663E2E606C2
:101330008146A545294535A0E38717FBE39F67FA5A
:101340000546FD564DB70545854571BF05487D5796
:1013500059BFB386A60205048307F4FFBA96E206D6
:10136000E18613F7F70F130607FD1376F60F63E513
:10137000C500138707FDF1BF1306F7F91376F60FC3
:10138000636EC902138797FAE30537FDA306D10000
:10139000130790066385E704634BF7061307800580
:1013A0006384E70A6345F702E38107EE13075002FF
:1013B00093055002E381E7F02286D9B51307F7FBC6
:1013C0001377F70FE364E9FC138797FC75BF1307E6
:1013D00030066386E70A13074006E39FE7FC032510
:1013E0000A00A947A307F100930A4A0063580500C1
:1013F0009307D0023305A0402307F1006C00EFF003
:10140000AFB56C004808EFF01F88568A75B7130710
:101410003007638EE7066341F7021307F006638E19
:10142000E70413070007E399E7F80347C1001367D0
:1014300027002306E10009A813075007638BE70282
:1014400013078007E39AE7F6938787FA414793B734
:101450001700A307E100139727008347C100ED9B06
:10146000D98F2306F100930A4A006C0003250A0075
:1014700079B7A947A307F100FDB7A147E5BF8305E9
:101480000A004808930A4A00EFF02FB2BDBF832735
:101490000A006C0048083EC8EFF0EFFE1C10930AEB
:1014A0004A003EC89DB7BA97FDB30145C5BBEF02E0
:1014B000DF882A88368583464800BA870347580064
:1014C000A206D98E328717B600001306669089E50A
:1014D00017B6000013068690BE85EFF0FFD66F00AA
:1014E0001F889757FF1F938727A49C4381CFEF0244
:1014F000DF84D843B2862E861847AA853E85029798
:101500006F00FF8561558280EF023F83835705009E
:1015100039712A84231EF100834745009305650035
:1015200041461305F101230FF100EF70406F930561
:10153000740141461305F102EF70606E835624007A
:1015400017B600001306C691E5450A85EFF0DFCF18
:101550006C08130630020A85EFF0BFF821616F00B6
:101560001F80EF028FFD39712A84930505034146E0
:101570001305D101EF70A06A930594084146130545
:10158000D102EF70C0698347E4010347F401835639
:10159000C401858B0607D98F17B600001306068D88
:1015A000E5450A85230EF100EFF01FCA6C0813060B
:1015B00010020A85EFF0FFF221616F004FFAEF028F
:1015C0002FF637040001B70400FF0111814A1759B3
:1015D000FF1F1309A9817D149389F4FF17BA000036
:1015E000130A4A8DEF60BF9E63C5AA0005616F00B4
:1015F0006FF68327490B13973A003E9783473700CE
:1016000095CF5C43A30107005286B3F6870082475B
:10161000E5454800E58FD58F3EC083462700B3F7E8
:101620003701858AE206D58F835607003EC0EFF06A
:10163000BFC111468A854800EFF0BFEA850A5DB751
:10164000EF02AFEF01468145EFF0BFE96F002FF1E8
:1016500083576500638E071A1D71A2CCA6CACAC83B
:1016600086CECEC6D2C4D6C2DAC05EDE801013F7F4
:1016700017003289AA8431CBF99B2313F500EF6060
:101680001F9906053D0541990A8BC16A3301A140A6
:101690008A8B8149014AFD1AEF607F97634CAA0C3F
:1016A0007947930604FB17A600001306A67FCA8598
:1016B0002685EFF0DFDF638F090C13961900DE85B6
:1016C000130504FBEFF0FFE15A8183D7640013F7A1
:1016D000270021CBF59B2393F400EF605F94060570
:1016E0003D0541998A8A3301A1400A8B8149014A0B
:1016F000EF60FF926345AA0A6547930604FB17A6AD
:1017000000001306A67ACA852685EFF05FDA6387A4
:10171000090A13961900DA85130504FBEFF07FDC44
:10172000568183D7640013F7470005CBED9B2393C5
:10173000F4006547930604FB17A6000013064677DE
:10174000CA852685EFF0BFD69C4481C703D74700E2
:101750003DEB130504FBEFF0BFEE130104FAF64076
:101760006644D6444649B649264A964A064BF25B39
:1017700025618280DC4413171A00BA9703D707004B
:101780006308570193971900DE972390E7008509B6
:10179000050A19B7130504FBEFF09FEA35B79C481B
:1017A00013171A00BA9703D7070019C793971900A0
:1017B000DA972390E7008509050A1DBF130504FB8E
:1017C000EFF01FE8B1BF2314E4FA03D767008326C4
:1017D000C4FA2146520751832315E4FA370700F073
:1017E000758F9447930584FA130504FB9206918242
:1017F000558F2326E4FA83C7770013F70701834741
:10180000F4FABD9BD98FA307F4FAEFF09FCDB1B7DF
:101810008280EF020FD01744FF1F1304245D04449D
:10182000797193F7F4FB1747FF1F2325F75C93F7B4
:101830000404A1C78588A1E097A90000938989675E
:10184000EF60EFF863DBA4028327440B13993400A5
:101850003E998356090091CE4E86E5454808EFF043
:10186000BF9E4808EFF0DFDD214681454A85EF0045
:10187000CFCF8504F1B7EFF09FD41C4413F7F7F7EF
:101880009746FF1F23A8E65693F707086397071E9E
:101890001C4413F7F7EF9746FF1F23ADE65413F7E9
:1018A00007106318071E18449377F7DF9746FF1F4A
:1018B00023A2F6549376072095C6058B630A07206A
:1018C00018408983858B3ACA0347840715464C081C
:1018D0000607D98F17A500001305855A230CF100C0
:1018E000EFF03FC01C4413F7F7BF9746FF1F23A339
:1018F000E65093F707408DC3835744000D464C08CC
:10190000231AF1008357640017A5000013058557BB
:10191000230BF100EFF0FFBC1844FD749387F47FB4
:10192000F98F9746FF1F23A7F64C9317470163DFF4
:101930000700EFA08FE119C98356C5016391061A0C
:1019400017A5000013058554EFF09FCF1C447D7749
:101950007D177D8F9746FF1F23AEE648139737010B
:10196000635A0702858B6388071CEFA04FDF1DC1F8
:1019700018458347E5001D463ACA0357C5004C0881
:1019800017A5000013050551231CE100230DF100EC
:10199000EFF03FB51844F977FD17F98F9746FF1F11
:1019A00023AAF6449317270163D907008145170539
:1019B0000000130525CAEF50FFF21844E177FD1728
:1019C000F98F9746FF1F23A7F6429317070163D3AA
:1019D0000702EFA0BF982A84814417A900001309C9
:1019E000E94BEF600FEE939704014205C1834181FB
:1019F00063EAA71445616F004FB583A70A009314EB
:101A00001900BE9483D7040033F767011DCF1396E6
:101A1000170133F77701B3F637016352060417A6AF
:101A200000001306E64309E717A600001306064464
:101A3000E5454808EFF05F814808EFF07FC083D7A5
:101A40000400B3F747012390F4000509EF602FE18C
:101A5000AA84EF60CFDF2695E341A9FA15BD36854C
:101A600019C7EF40A04361DDEFF01FAAC9BFEFD057
:101A70009FB371D5EFF0FFAED9B785697D7A014983
:101A8000974AFF1F938A4A47056B896BFD197D1A98
:101A900075BF858B9DC7EF500FF3231AA1004146F8
:101AA0009745FF1F9385053E13056101EF702017D1
:101AB00049464C0817A500001305053CEFF07FA22E
:101AC000DDB317A500001305253BEFF07FB7E1BBA1
:101AD00017A500001305C53AEFF09FB621B50357CF
:101AE000E501C17785073E978357A101FD141337A0
:101AF00017003207E58FD98F231DF100231AD1007B
:101B000083560502035725022146231BD100231CBF
:101B1000E100035745028566FD16758FFD76F58F4A
:101B2000D98F4C0817A5000013054536231DF10079
:101B3000EFF03F9B21BD17A500001305A535EFF081
:101B40003FB089BD5C4813F7E7FF58C8858B89CF44
:101B5000A6864A86C9450A85EFF00FEF8357040031
:101B600099E70A85EFF0DFAD850461049DBD231A76
:101B7000F100835724009305440041462808231BA5
:101B8000F100EF70C00951464C080A85EFF07F95CF
:101B9000E1BFEF028F9A85473395A7009747FF1F54
:101BA0009387C7249C47411181455D8D9747FF1F4F
:101BB00023A2A7249377057085E393576500858B4F
:101BC000A1CBC167938707887D8D05EDEF606FD14D
:101BD0009305803EB305B5021745FF1F1305053277
:101BE0002EC6EF50A03BB24519C16349B50085C56B
:101BF0001745FF1F13058530EF50C04441016F00AA
:101C00000F96EF600FCE2A84EF60AFCEE360A4FCA6
:101C1000EF602FCE75BF0145EFF0BFBFC5B7EF0234
:101C2000CF917971AA8601441749FF1F1309091C36
:101C300036C6EF60CFB9B246635CA4028327490B76
:101C400093143400BE9483D704006396D70285C6EC
:101C500017A6000013060626E5454808EFF0CFDE7C
:101C60004808EFF0FF9D214681452685EF00EF8F64
:101C700045616F00CF8E050465BF19C223200600A1
:101C8000814701C59306D00389E53E85828085059D
:101C90000505838705000307050099CF6394E700D6
:101CA000E397D7FE8147D5B79306D0038547E30E68
:101CB000D7FC93371700D1BF9307F002E316F7FE66
:101CC000854761D6050508C2C9B799C123A005009B
:101CD00081470DC11308D0031306F0023307F50046
:101CE0008306070081CA638706016397C60099C10E
:101CF000050798C13E8582808507CDB731C9EF02BF
:101D00004F8141112E8A6C002A89368BB28A97A4A2
:101D100000009384E40DEFF05FFB2A8C0144A68958
:101D2000B14B88406286CA85EF70E01801ED0E0461
:101D30004E945C403245DA865686D28582974101C0
:101D40006F00AF800504A104E31D74FD6155C5BF9C
:101D50007D55828099E561558280615505616FF0FE
:101D60007EFFEFF2FEFB2E8A2A8401118145B284A8
:101D700052854146BA893689EFF06F879315050180
:101D8000C1811376F50FA1812285EF507FB12A849E
:101D900069D552854C08EFF05FF3524A2A8BE30E67
:101DA0000AFA2A8697A500009385C50F5285EF7021
:101DB0008010AA8A0DED7D5AEF606FA563C5AA0059
:101DC00099E8014561BF5C4413971A00850ABA97E8
:101DD00023904701D5B74C442EC6EF604FA3B245C0
:101DE000131615004E850299E34DA0FC85BF5A8657
:101DF00097A500009385850B5285EF70C00B0DE110
:101E0000032A0401EF60AFA1131615008145528526
:101E1000EFF0BEF5DDD40C482EC6EF604FA0C1B781
:101E20005A8697A500009385A5085285EF70A008F3
:101E300041E11C44A5CF81ECD443370700E0758F06
:101E40009447D8C33707001F758F98C701BFA146B5
:101E50003008CE854A85EFE0DF96E31105F018449F
:101E6000835781017D762312F7008357A101939652
:101E7000470183576700D182F18FD58FF2467D7677
:101E80007D16F182858AB206F18FD58F2313F70074
:101E90008347E1018356C1012305F7008347B7005B
:101EA0002314D700FD8BA305F7004DBD7D557DB5EF
:101EB0005A8697A50000938525F35285EF60B07F81
:101EC000E31D05E81C4CE38A07E89C43E38707E829
:101ED000CE864A86A6852285829749B5EFF2FEE531
:101EE0003687B2862E86AA850545EFF0BFE66FF0ED
:101EF0001EE7EFF29EE43687B2862E86AA8501455C
:101F0000EFF05FE56FF0BEE5EFF29EE1411199C1A0
:101F100023A005009747FF1F938707008043814454
:101F20001DC82E89AA8931141DC40C4070004E852D
:101F3000EFF0BFD419CD81E8A284630C0900B24749
:101F40002320F90039A08C4008400146EFF0FFD271
:101F500065F5404869F8268541016FF0BEDF1841FC
:101F600011CBEFF29EDDAE873E85B28536860297B5
:101F70006FF0FEDE35558280EFF23EDC8357C50000
:101F800013D70501C205B387E7021841C18148494B
:101F9000BA95BE95EFF0BFFC6FF07EDC584111CBD7
:101FA000EFF2BED9AE873E85B285368602976FF0D6
:101FB0001EDB35558280184509CBEFF21ED8AE875F
:101FC0003E85B28502976FF09ED9355582805C457B
:101FD00099C7EFF29ED62E8582976FF05ED8355561
:101FE0008280EFF2FED383290500035AC5002A84BC
:101FF0004849AE848145EFF09FFD2A890DE193D5D4
:102000000401B38545030356C4004848CE95EFF05C
:102010009FFA2A8909E548488545EFF05FFB4A8524
:102020006FF05ED3EFF2DECF2A890441035BC50077
:10203000484979712E848145B28A368AEFF03FF99A
:1020400041E193590401B389690342044180269414
:10205000A29903440901330480403374440111CC34
:1020600003254901A2865686CE85EFF03FF3AA8468
:1020700031E1330A8A40A299A29A8144630C0A0290
:102080005286D685080803244901EF6050398346FB
:1020900009011C089305F00F33864641338547013B
:1020A00036C6EFF09ECCB2461008CE852285EFF002
:1020B000FFEEAA84032549018545EFF05FF12685EF
:1020C00045616FF03EC9EFF25EC72E864C41A146D6
:1020D0002A84EFF03FF5AA8403450401A145EFE00F
:1020E0007F985C403385A74048C026856FF03EC787
:1020F000814797A600009386A6CC6393C700828091
:102100003387F500034707008507398D13574500CE
:102110003697034707001205398D1375F50F1357CE
:1021200045003697034707001205398D1375F50FE3
:10213000E9B7EFF29EC02A84AA851D461305F00F69
:10214000EFF01FFB834774003385A7403335A000B1
:102150006FF0FEC0EFF27EBE4111A1463000EFF0FD
:10216000BFE109ED03578100C167FD1705456317FE
:10217000F7002800EFF0FFFB3335A00041016FF0BE
:102180001EBEEFF2FEB9AE848C414111A1462A89F0
:1021900003440501EFF05FDEAA8939E9A1452285F4
:1021A000EFE05F8C9C400357C9002A8AAA97939658
:1021B00007019CC0C182098F639CE602C16513D7E9
:1021C0000701B385B74011E78355E900FD15C20546
:1021D000BE958CC0A1460A864A85EFF0FFD9AA8930
:1021E00001E90A85EFF0FFF401C9832749009CC08B
:1021F0004E8541016FF01EB60357C9008357210079
:1022000080403307474163DBE70033FA4703631736
:102210000A004177798C3E9480C0D9BF03450901FB
:10222000A145417AEFE01F84098CAA8A80C0337AE5
:102230004401417B63648A0081495DBFA14630004F
:10224000A2854A85EFF05FD3AA895DF12800EFF0FF
:102250005FEE11E98357A1000357C100337A6A0189
:1022600080C0BA973E9A33045441E9B7EFF2FEAC0E
:102270002A84AA851D461305F00FEFF07FE7A3031C
:10228000A4006FF0DEADEFF2DEA82A84034505015D
:102290005D71A145EFE00FFD5C402A8B0355E40022
:1022A0004179B3F727016C003EC6EFE00FFD83557F
:1022B000C400B247A1463008BE95B385654122856A
:1022C0002EC8EFF07FCBAA84634B05002808EFF0FF
:1022D0005FE611C9B2452285EFF0BFD0AA842685FA
:1022E00061616FF09EA6C2470357A101417C338B09
:1022F0006741B3F72701BA973EC810100C08228532
:10230000C24BEFF01FE8AA8479F90810EFF07FE2E2
:102310002DE95C403ECA30104C0822855249EFF04E
:102320005FE6AA844DFD03578102835701026316BD
:10233000F7002810EFF0FFDF09C55840D247E31C33
:10234000F7FC63902B058357410285CF8357210209
:10235000B3FA8B010810BE9A1C442311F102EFF06E
:10236000FFF083490401035A4102B309304193F954
:102370000902631B0A000C102285EFF0DFD4AA8447
:1023800039FDE31C7BF7B9B74E8963733A01528973
:10239000CA861018D6852285EFF01FBEAA8421F1C7
:1023A000630909000C44CA8610182285EFF09FC704
:1023B000AA8403450401CA85EFE0CFEA1C443E9598
:1023C00008C4E39E04F0330A2A41CA9A5DB7EFF2CB
:1023D0003E95411191E5FD54268541016FF09E9790
:1023E000C44983D725014CC904C12316F50003C78E
:1023F00005012A842317E50003C51501931607017B
:10240000130700022308A400C182E366A7FCE1D7FA
:10241000B3E4F402E9F08547E3FFD7FAA145EFE022
:102420006FE4AA89014A01498357C4009315090141
:102430002285BE95B38535412EC2EFF0BFD119ED8F
:102440000355E4004C00050AEFE02FE39245420AF1
:102450002285135A0A01EFF0FFCF09E905098357D6
:10246000E400420913590901E360F9FC8357E400D1
:1024700063944701D1548DB7639427039245A146D5
:102480003000B38535412285EFF01FAF35E12800DC
:10249000EFF03FCA11C50355E4004C00EFE0EFDD5B
:1024A0009247C17A3387374158C04177F98F1CC4AE
:1024B0004C401C4463EEF500A14630002285EFF04D
:1024C000BFAB1DE52800EFF0DFC6032A44001DC1A5
:1024D0005C400355E4004179B3F727014C003EC24C
:1024E000EFE0AFD992452285EFF0DFC6635C0502CD
:1024F000AA84DDB512450359A100035BC10033F581
:10250000AA002A9903450401DA85EFE0AFD54A9580
:1025100008C46314450163130B04330A3A412322B0
:10252000440179B709C58547A308F40075B54C4047
:102530002285EFF01FAB4DFD48408357C40086094C
:102540003375A9003E953305354148C033752501E3
:1025500008C42285EFF03FD379D559BF4D5549BF07
:1025600083471501C9CFEFF2CEFA2A84034505014E
:1025700041112E8AA145BA893689328BEFE08FCE80
:102580008357C4000605898F7D5563E727075C40A4
:1025900081443EC230004C002285924AEFF07FBE5B
:1025A00021ED835B810063994B012800EFF07FB838
:1025B00001E58504C204C18058409247630BF702CD
:1025C000E3FA99FC8356C10061559DC663E6340366
:1025D000C175B3FABA006373D900CA868355A100E6
:1025E0005A862285D695EFF03F9919E50355C1002B
:1025F00021A06155E3884BFD41016FF00EF549556F
:102600008280EFF28EF30147EFF09FF56FF02EF529
:10261000EFF2AEF23284B2862E8683554500084131
:10262000EFF03FFE635385002A8422856FF02EF37E
:10263000EFF2AEED834715013971C954BDC7034BA5
:1026400005012EC62A84A1455A853689328AEFE0D3
:102650006FC10D473307E5028357C400AA8DFD54AF
:10266000998F63E427056304090063000A045C4052
:102670003ECA30084C082285524DEFF09FB0AA891F
:1026800045ED8357810132476397E7002808EFF053
:102690005FAA630605105840D247E31CF7FC81444B
:1026A000631B090019A0814499E7268521616FF019
:1026B0008EE9E35CA0FE5A85CA85EFE0AFBA014B14
:1026C00011C5330BB501420B135B0B01014D7D5C52
:1026D000C17B930C44008357E4006380A70D1C4426
:1026E00044403307FB0063EBE40432472311F1025B
:1026F0000810FD572310E102231221032303F102E6
:10270000EFF0DFB6630909000C44CA8652862285C1
:10271000EFF05F91AA8903450401CA85EFE08FB409
:102720001C443E9508C4639909000C102285EFF003
:102730009F99AA89CA8435D9CE8485BF03450401EF
:10274000A145EFE02FB2B387A4002311F102835714
:10275000C400B3F4740123108103BE94898C44C077
:10276000081023120102EFF07FB00C102285EFF069
:102770009F95AA840355E400E685EFE00FB05C4026
:10278000B3F777011CC4E39204F22285EFF0BFAFE8
:10279000AA84E31C05F0050D3DBFC15439B783572A
:1027A000C101E30209F0E39827F1C177034C04016A
:1027B000B377FD00035DA101330C8041137C0C0253
:1027C0003E9DD28ACA8CE28B63F38C01E68BDE8657
:1027D0001010EA852285EFF02FFAAA84E31B05EC9E
:1027E0005E860C105685EF602041AA84E31505EC47
:1027F000B38C7C415E9DDE9AE3970CFC7DB5EFF2D5
:10280000CED381460146EFF0BFE26FF04ED5638C28
:10281000050EEFF20ED05D71054D19C213BD160005
:1028200003590502B68B328B050942091359090178
:102830002E8A2A84CA89216C930A8500E15C93045C
:10284000F9FFC204C180638F84059306A004500081
:10285000A6855685EFF0FFDA6357050063139501EF
:10286000A6892689E9BF9C083E95230A05FA4C00F3
:102870005285EFF00EDA75F563040D0883570402F4
:10288000639597089387F4FF2310F4028946130693
:102890000402A1655685EFF0BFD963580506616152
:1028A0006FF0AECA0145E31C0DFE0549B1675D55E9
:1028B000E387F9FE9165CE9593048400C205DE8618
:1028C0005A86C1812685EFF0BFD6630D0900528577
:1028D000EF60405DAA865286CE852685EFF05FD5F3
:1028E000E34F05FA8357040263FF370323103403D1
:1028F000894613060402A1652685EFF07FD325A043
:10290000A689014965B77D558280A6855685EFF079
:102910001FEFE34605F89165FD15CA95C205C18113
:102920005685EFF0DFEDE35CA0F601458DBFEFF2D9
:102930004EBE03540502916A1D71050442042A89A2
:10294000AE894180A16B130A8500FD1A130B0502A5
:102950009304F4FFC204C180639D7405916B2164EC
:10296000130A8900850B170C0000130CACCA83579F
:10297000090293041400C204C18085076383F40E26
:102980005E949306A0045008A68552854204EFF099
:102990005FC74180AA8A854613067100A2855285C9
:1029A000EFF03FC62A8B634750076347A006268493
:1029B0007DBF56949306A0045008A6855285420414
:1029C000EFF03FC441802A8C854613067100A28532
:1029D0005285EFF01FC3634C8003E351A0F8835787
:1029E0000902E39D97F69387F4FF2310F9028946C5
:1029F0005A86A1655285EFF0BFC3A6855285EFF0D8
:102A00001FE0A2855285EFF09FDF268491B7E3583F
:102A1000A0FCA9B7634BA000A6855285EFF03FDE6E
:102A2000A2855285EFF0BFDD59B79C10BE9A238A6C
:102A30000AFA639109022C004808EFF0EFCC25D97F
:102A40001C45224552C62318810074006286DA852F
:102A50008297B1BF0146CE854808EFF00FA261FD15
:102A6000B9B7014525616FF04EAEEFF20EAD973765
:102A7000FF1F9387674A8043814409C42A89311420
:102A8000814401E426856FF08EAD631809005C4433
:102A900081EF404865D83114EDB708400146CA853A
:102AA000EFF0AF9D6DF5F5B78297E5F4AA84D5B741
:102AB000EFF2AEA89737FF1F938787468043AA841B
:102AC00009EC2685EFF07FFAAA840144EF502FD05D
:102AD000636CA40026856FF08EA85C402285A685D5
:102AE0009C4382970040E9BF05041374F40FF9BFBB
:102AF000EFF2AEA40145EFF0BFFB6FF04EA69737A3
:102B0000FF1F9387E74123A0070023A207008280CD
:102B1000EFF2AEA29737FF1F9387074023A007006D
:102B200023A20700EFF0BFFD6FF06EA3EFF2EEA05F
:102B30004111130985002A84EF50CFE5AA854A8503
:102B4000EFF0FF88AA8419ED89461306E100A1651C
:102B50004A85EFF01FABE177634405008357E1003E
:102B60002310F402268541016FF06E9F9737FF1FF7
:102B70009387073B90430147B28691EE05E3DC4320
:102B800010C11737FF1F232DA73885EF9737FF1F79
:102B900023AAA738828036879442C5B7144385E2BA
:102BA000DC432320050091EB9737FF1F23ACA736AA
:102BB0009737FF1F23A6A736828088C3C1BF14C1E1
:102BC00008C38280EFF26E971734FF1F130484301E
:102BD0002285EFF0BFF5AA8405E5179900001309D7
:102BE000292722859737FF1F23A8272FEFF01FF8EB
:102BF0009737FF1F23A2272F9737FF1F23A6873260
